:020000040000FA
:06000000020B260201F3D1
:03002B000207C009
:030043000206555D
:0300530002012D7A
:03006B000207E9A0
:1000830002018401010105030101FF0F10FEFF7B43
:100093002D00000000B12C00000000FF000000FF55
:1000A300000196511800020000041D0000B61C74E4
:1000B3001C941DD41C4C1DB01CA41C00000000008B
:1000C300000000000000000000000000000000002D
:1000D30000000006FFFFFF00081001010400561B8B
:1000E300000000E8030000FFFF251C03E8030000F5
:1000F30064006400B801A0BB0D00A0BB0D000202A8
:10010300000800000502070401051E02051E020A7D
:100113000A01080803B80B02803E0102FEFFE80350
:100123000A050001FFFF0A1401E0C0E074F21204A3
:1001330072A2AFE433F508D2AFAFA7AEA1EE5F541E
:100143001060061219E675A1EFEE5F5408600812FD
:1001530019EC75A1F78023EEA2E092F0EFA2E08202
:10016300F05017906198E0F8900B52E0C398A2D238
:1001730065D0335002E8F075A1FE751A00E50880DA
:1001830066C0E074F2120472A2AFE433FED2AF9001
:1001930061A4E0F8759B00E59158540860087591D7
:1001A300F7121A348023E59158541060087591EFC3
:1001B300121A3A8014E591A2E092F0E8A2E082F0EC
:1001C3005007E0C2E0F0121BA29061A3E0F8E5E95A
:1001D300585404600E121B7875E9FB906193E0A2FA
:1001E300E640F2751A00EEA2E092AF7F010204D15D
:1001F300C0E074F2120472A2AFE433FED2AF906196
:10020300A5E0F8E5BF585404600675BFFB121BBA9E
:1002130080D1C3E498F8E499F91202568026C3E426
:100223009AFAE49BFBE920E7E9120256E498F8E422
:1002330099F922C3E498F8E499F9120256E498F87C
:10024300E499F9C3E49AFAE49BFB22EB20E7CFE9B4
:1002530020E7E0B90010BB0008E88AF084F8AAF0B0
:1002630022E4FBC8FA22EB70227B10C833C8C933DF
:10027300C9335007C39AC3DBF280069A50012ADBC5
:10028300EAC833F4C8C933F4C9FA2275F008E4C8DC
:1002930033C8C933C933C99AC99B5004C92AC93B56
:1002A300D5F0ECFBC833F4C8E4C9FA22080808EA1D
:1002B300C0E0EBC0E086F0E7A4FA180986F0E7A4F3
:1002C3002AFA180986F0E7A42AFA180986F0E7A49F
:1002D3002AFA1986F0E7A4FBE5F02AFA190886F052
:1002E300E7A42BFBE5F03AFA190886F0E7A42BFB09
:1002F300E5F03AFA18180986F0E7A4C5F02BFBE4F9
:100303003AFA1908E7C5F0C6A426F6E5F03BFBE484
:100313003AFA1886F0E7A4F6E5F00826F6E43B0877
:10032300F6E43A08F6D0E0FBD0E0FA22E4CFC0E0EE
:10033300E4CEC0E0E4CDC0E0E4CCC0E075F020E65C
:1003430026F608E633F608E633F608E633F6181819
:1003530018EC33FCED33FDEE33FEEF33FFC3EC97C4
:1003630009ED9709EE9709EF97191919400FFFEC5B
:1003730097FC09ED97FD09EE97FE191906D5F0BF15
:10038300ECF709EDF709EEF709EFF7191919D0E0C2
:10039300FCD0E0FDD0E0FED0E0FF222518C582C0EE
:1003A300E0E51934FFC583C0E0E518C3958224F85E
:1003B30010AF088583198582188008858319858283
:1003C30018D2AFCEF0A3E520F0A37808E608F0A397
:1003D300DEFAEFF0A3E58124FAF8E608F0A3E608D5
:1003E300F0A3E608F0A30808E608F0A3E608F0A3E4
:1003F30015811581D0E0FED0E0F8158115811581B6
:10040300E8C0E0EEC0E022120BB8B9000302045CBE
:10041300E49004D1780A791A8002F0A3D8FCD9FABF
:10042300781A9000867A01BA00028007E493A3F653
:1004330008DAF97ADA7B1D90008778A779018015AD
:10044300E493A3AD82AE838A828B83F0A3AA82ABAB
:10045300838D828E83D8E9D9E77582407583CD7405
:10046300061208B17582AE75832A74001208B1C0F2
:10047300D02518C582C0E0E51934FFC583C0E0E587
:1004830018C3958224F310AF0885831985821880D9
:1004930008858319858218D2AFC8F0A3E9F0A3EACF
:1004A300F0A3EBF0A37908E709F0A3D8FAECF0A3E3
:1004B300EDF0A3EEF0A3EFF0A3D0E0F0A3D0E0F0D3
:1004C300A3D0E0F0A3E520F0A3E5F0F0A322851983
:1004D30083851882E0C0E0A3E0F9A3E0FAA3E0FB80
:1004E300A37808E0F608A3DFFAE0FCA3E0FDA3E0AD
:1004F300FEA3E0FFA3E0C0E0A3E0C0E0A3E0F5D0EB
:10050300A3E0F520A3E0A3F5F010AF0885831985D8
:1005130082188008858319858218D2AFD082D08350
:10052300D0E0F8D0E032E4730375F0108E218F220F
:10053300858226858325851882851983E0CEA3E0ED
:10054300CF852682852583EBC9EAC8EDCBECCAC3E8
:10055300E833C8E933C9EA33CAEB33CBC3EA9EF5C0
:1005630024EB9FF523B35004AB23AA24EC33CCED47
:1005730033CDD5F0DAAE21AF2222D083D082ECC0C6
:10058300E0EDC0E0E493A3FCE493A3FDED4C600D28
:10059300120698EC24FFFCED34FFFD80EFE493A3F7
:1005A300FCE493A3FDED4C600D12076BEC24FFFC00
:1005B300ED34FFFD80EFD0E0FDD0E0FCE493A3C079
:1005C300E0E493C0E022D083D082E9C0E0E493A3C7
:1005D300C386F0C5F095F0F908E493A386F0C5F05F
:1005E30095F0700BE493A3C3994005E9048002A33B
:1005F300E475F002A42582F582E5F03583F583D016
:10060300E0F9E493A3C0E0E493C0E0228519838575
:100613001882E0A3FEE0A3F5207808E0A3F608DF44
:10062300FAE0A3FFE0A3C0E0E0A3C0E0E0A3C0E0E2
:10063300E0A3C0E0E0A3C0E010AF08858218858383
:10064300198008858218858319D2AFD083D082029E
:1006530008B7C0E074F2120472A2AFE433FED2AF63
:10066300C2C0901CD2E0700BE5D1A2E4501D121958
:10067300448018E5D1A2E3500675D1F712191AE5A3
:10068300D1A2E4500675D1EF121920EEA2E092AF89
:100693007F010204D1C0E0C3E493960874019396EA
:1006A30018400FE49366700808740193661870008D
:1006B3007019A3A3C3E49396087401939618A3A394
:1006C300400DD0E0D0E0D0E00205B9A3A3A3A3A3DB
:1006D300A3D0E022D083D082C5F0E493A3C5F0C3B6
:1006E30095F0F5F0E493A3C395F04005E5F004809D
:1006F30001E475F002A42582F582E5F03583F583E4
:10070300E493A3C0E0E493C0E02274048004740281
:100713008000CCC0E0EDC0E0E518C39CCCAD19501F
:10072300011D10AF068C188D1980068C188D19D2F7
:10073300AF120833D0E0FDD0E0FC2274028000CC7D
:10074300C0E0EDC0E0E518C39CCCAD1950011D100D
:10075300AF068C188D1980068C188D19D2AF12082C
:1007630011D0E0FDD0E0FC22C0E0C0F088F0E493BB
:100773006670080874019366187000A8F0A3A3704C
:100783000BD0F0D0E0D0E0D0E00205B9A3A3D0F0C5
:10079300D0E022D083D082CCC0E0E493A3600612E1
:1007A30008541470FAE493A360061209831470FAD0
:1007B300D0E0FCE493A3C0E0E493C0E022C0E0C037
:1007C300D0E8C0E0E9C0E0A9A8D2AFC2C7751A005B
:1007D300E9A2E7E433F8E9A2E792AFD0E0F9D0E089
:1007E300F8D0D0D0E032C0E074F212047275890000
:1007F300C2C5901CD2E0700E7A007B10900BEEE025
:10080300F9121ECC80031229107F010204D1CAC041
:10081300E0E493A3C582CCC582C583CDC583F0A391
:10082300C582CCC582C583CDC583DAE5D0E0CA22B3
:10083300CAC0E0E0A3C582CCC582C583CDC583F021
:10084300A3C582CCC582C583CDC583DAE6D0E0CA11
:1008530022C0E0E493A3D39C5010E493A3C39C4031
:100863000AD0E0D0E0D0E00207B3A3A3A3D0E022F4
:10087300C008C3E096F50808A3E096420808A3E081
:1008830096420808A3E09645087001D3D008227069
:1008930009080808226016181818C6C333C608C604
:1008A30033C608C633C608C633C6D5E0EA22C09F9E
:1008B300F59FE473D09F22D083D082C09FE493C07E
:1008C300E0740193C0E0740293F59F2200C0D02529
:1008D3001810AF08F518500C05198008F5185002C8
:1008E3000519D2AFD0D0222518F58210AF08F5181C
:1008F300400C15198008F51840021519D2AF851957
:1009030083227404800A74038006740280027401D3
:10091300C0E0F4041208EAD0E0120B6322BB010228
:10092300E722C082C08389828A83BB0003E08002FE
:10093300E493D083D082226016080808C6C313C686
:1009430018C613C618C613C618C613C6D5E0EA22BE
:100953002518F8E43519F9222518FAE43519FB228C
:100963002518FCE43519FD22C3E0C696F608A3E07A
:10097300C696F608A3E0C696F608A3E0C696F62246
:10098300C0E0E493A36C7009D0E0D0E0D0E00207AC
:10099300B3A3A3D0E022251810AF08F518400C1517
:1009A300198008F51840021519D2AF22E0667010BD
:1009B30008A3E066700A08A3E066700408A3E06673
:1009C30022C3E09608A3E09608A3E09608A3E09666
:1009D300A2D265D03322E76670100809E766700A71
:1009E3000809E76670040809E76622C3E697F60874
:1009F30009E697F60809E697F60809E697F622C38B
:100A0300E49396087401939608740293960874030A
:100A1300939622C3E096F008A3E096F008A3E0962D
:100A2300F008A3E096F022E657F60809E657F60821
:100A330009E657F60809E657F622E026F608A3E08A
:100A430036F608A3E036F608A3E036F622E493F67A
:100A530008740193F608740293F608740393F6225C
:100A6300E056F608A3E056F608A3E056F608A3E01E
:100A730056F622E056F008A3E056F008A3E056F03D
:100A830008A3E056F022E647F60809E647F6080908
:100A9300E647F60809E647F622700422600D18C6F9
:100AA300C333C608C633C6D5E0F41822E627F608D2
:100AB30009E637F60809E637F60809E637F622E0CD
:100AC30026F008A3E036F008A3E036F008A3E036EA
:100AD300F022E4C396F608E496F608E496F608E4F2
:100AE30096F622600D08C6A2E713C618C613C6D52C
:100AF300E0F322C6F4C608C6F4C608C6F4C608C6A0
:100B0300F4C622C3E7960809E7960809E796080999
:100B1300E79622C3E09608A3E09608A3E09608A30D
:100B2300E0962275D00075813F7518D175190400C0
:100B330002040AE6F008A3E6F008A3E6F008A3E639
:100B4300F022600C08C6C313C618C613C6D5E0F45A
:100B530022E0F608A3E0F608A3E0F608A3E0F622F5
:100B6300CAC0E0E6F0A308DAFAD0E0FA22E8F0A37C
:100B7300E9F0A3EAF0A3EBF022E0F8A3E0F9A3E0A5
:100B8300FAA3E0FB22ECF0A3EDF0A3EEF0A3EFF069
:100B930022E0FCA3E0FDA3E0FEA3E0FF22EAF0A332
:100BA300EBF0A3ECF0A3EDF022E0FAA3E0FBA3E06B
:100BB300FCA3E0FD22E5C754F84401F5C7790122FF
:100BC3002518F582E43519F58322C2AF75D69F0245
:100BD3000000221208BA7EA0031208BA8BA00312E7
:100BE30008BA94A0031208BA76A2031208BAA2A301
:100BF300031208BAB2A3031208BAEDA4031208BA87
:100C030061A5031208BA9BA5031208BACCA6031266
:100C130008BA2DA7031208BA69A7031208BA43A991
:100C2300031208BA00AD031208BA14AD031208BACE
:100C33001EAD031208BA28AD031208BA32AD03126F
:100C430008BA3CAD031208BA55AD031208BA5FAD3A
:100C5300031208BAD6AD031208BAE1AD031208BAFB
:100C630010AE031208BA38AE031208BA43AE031229
:100C730008BAA8AE031208BAB2AE031208BABDAEE0
:100C8300031208BAE1AE031208BA05AF031208BA99
:100C930077AF031208BAC0AF031208BADCAF03126E
:100CA30008BA4DB0031208BA99B0031208BAE2B0F9
:100CB300031208BA20B1031208BAA1B1031208BA89
:100CC30048B2031208BA0DB4031208BA72B403127D
:100CD30008BAA0B5031208BAC6B5031208BA0EB70C
:100CE300031208BA48BA031208BA46BC031208BA78
:100CF30011BE031208BAAABE031208BAABC003128C
:100D030008BA60C1031208BA99C1031208BA09C22A
:100D1300031208BA13C2031208BA3CC4031208BA76
:100D23003FC5031208BA7CC6031208BAD3C603121E
:100D330008BA7EC7031208BA2EC9031208BA7BCABF
:100D4300031208BA9BCA031208BAF0CA031208BAFC
:100D5300F1CB031208BA19CC031208BA78CC0312E8
:100D630008BA70CD031208BAE7CD031208BAFACE57
:100D7300031208BA68CF031208BA67D0031208BA7D
:100D8300C1D2031208BAEAD2031208BA50D403122A
:100D930008BAD2D5031208BA29D6031208BAD7D68D
:100DA300031208BA7CD7031208BADFD7031208BAB2
:100DB3009DD8031208BA2FD9031208BA8ED9031289
:100DC30008BAD0D9031208BA01DA031208BA58DBF9
:100DD300031208BA0080021208BA3280021208BA5B
:100DE3006B80021208BA3482021208BA78820212A5
:100DF30008BA4E83021208BAAD83021208BAC3843A
:100E0300021208BA0F85021208BA9D87021208BAA5
:100E1300818A021208BAC88B021208BA608C0212C5
:100E230008BA6C8C021208BAB58C021208BAF78D94
:100E3300021208BAED8E021208BA178F021208BA0C
:100E43006D8F021208BAC68F021208BA39900212C5
:100E530008BA6F92021208BAF193021208BADC942C
:100E6300021208BA2696021208BA5E98021208BA4B
:100E73005B9B021208BA6A9B021208BAFE9B02121B
:100E830008BAA99C021208BAEC9C021208BA359D52
:100E9300021208BA859D021208BAE99D021208BA25
:100EA3005B9E021208BA779E021208BAA69E02122D
:100EB30008BAE59E021208BAE09F021208BA8FA090
:100EC300021208BA0CA3021208BA3EA4021208BA0C
:100ED30016A5021208BA98A5021208BACDA90212E1
:100EE30008BAFCA9021208BA57AA021208BA8AAAB7
:100EF300021208BA02AB021208BA35AB021208BAE0
:100F030096AB021208BAE6AB021208BAB3AC0212ED
:100F130008BA6CAD021208BA30AE021208BAAAB00F
:100F2300021208BA0CB2021208BA5DB3021208BA6E
:100F330081B4021208BA84B4021208BAB3B402121A
:100F430008BAABB6021208BA6AB7021208BA99B75E
:100F5300021208BAB7B8021208BA7FB9021208BA65
:100F630040BB021208BAB0BB021208BAE2BB0212BB
:100F730008BA02BC021208BA71BC021208BA6ABDEE
:100F8300021208BA8EBD021208BA01BE021208BAD2
:100F93002AC0021208BA89C0021208BADDC00212BE
:100FA30008BA0CC3021208BAEFC3021208BA77C414
:100FB300021208BA5BC5021208BAE5C5021208BAE2
:100FC300F9C5021208BA0DC6021208BA21C60212E6
:100FD30008BA35C6021208BA62C6021208BA92C625
:100FE300021208BA4DC8021208BA23C9021208BA7B
:100FF300C7C9021208BA1CCA021208BA7FCA02126F
:1010030008BAC8CA021208BAE3CA021208BA34CB31
:10101300021208BAFCCB021208BAA2CC021208BA16
:1010230028CE021208BAB3CE021208BAF6CE0212C2
:1010330008BA8FD0021208BAD6D0021208BA48D121
:10104300021208BA9DD2021208BA46D3021208BA93
:101053007AD3021208BA92D3021208BA35D4021212
:1010630008BAB1D6021208BA59D8021208BA77D808
:10107300021208BA95D8021208BA61D9021208BA44
:10108300AFDC021208BACB81011208BA0D82011239
:1010930008BA7A87011208BAC687011208BA0C88FF
:1010A300011208BA5D89011208BAC289011208BA8D
:1010B300068A011208BA6C8B011208BAC78E011294
:1010C30008BAFA8F011208BA899B011208BA199C4F
:1010D300011208BA039F011208BA68A0011208BAE4
:1010E300CBA0011208BAE7A1011208BA51A3011259
:1010F30008BA30A4011208BA9EA6011208BA30A891
:10110300011208BAC1A8011208BAE0A9011208BA6B
:101113006DAA011208BA77AA011208BA9FAA01128E
:1011230008BA42AB011208BA2DAC011208BAF5ACE9
:10113300011208BA82AD011208BA98AD011208BAB9
:10114300B5AD011208BADEAD011208BA0BAE011239
:1011530008BA4FB0011208BA22B1011208BA66B137
:10116300011208BAE8B1011208BA89B2011208BA29
:10117300BBB2011208BA02B3011208BA35B30112A5
:1011830008BA79B3011208BAC8B3011208BACDB3C9
:10119300011208BA29B4011208BA6DB4011208BACF
:1011A30052B5011208BA9CB5011208BA01B6011270
:1011B30008BA5FB6011208BADEB6011208BA56BA07
:1011C300011208BA59BB011208BAEFBC011208BADE
:1011D30032C0011208BAD4C0011208BA1DC30112E9
:1011E30008BAD8C3011208BA17C4011208BADBC57A
:1011F300011208BAF8C5011208BA01C6011208BAE9
:101203000AC6011208BA15C6011208BA34C6011279
:1012130008BA58C8011208BAB5C8011208BABFC83B
:10122300011208BAC9C8011208BA2CC9011208BAB6
:1012330088C9011208BA95CA011208BAF6CA01127E
:1012430008BA07CC011208BA50CC011208BA1ACD59
:10125300011208BA31CE011208BAF5CE011208BA4A
:1012630041D0011208BA45D1011208BA3ED2011287
:1012730008BA56D2011208BA8DD2011208BA97D20F
:10128300011208BAA1D2011208BAACD2011208BAEB
:10129300CAD2011208BA12D3011208BA70D30112CA
:1012A30008BA97D3011208BAA9D3011208BA52D4C3
:1012B300011208BA8BD4011208BABCD5011208BABC
:1012C30019D6011208BA0AD7011208BA40D7011277
:1012D30008BAB0D7011208BA2CD8011208BAADD98E
:1012E300011208BAD4DA011208BA96DB011208BA5D
:1012F30064DC011208BAE9DC011208BA98DD0112B4
:1013030008BA80DE011208BA19DF011208BAF5DF44
:10131300011208BA5DE0011208BA1CE1011208BA11
:1013230078E1011208BADCE1011208BAA2E2011263
:1013330008BAC5E2011208BA7FE3011208BAA1E3B1
:10134300011208BA02E4011208BA32E6011208BA1D
:101353002BE7011208BAD7E7011208BAF4E9011220
:1013630008BA3DEA011208BA88EA011208BAE4EAA7
:10137300011208BA42EB011208BA66EB011208BA6D
:101383008AEB011208BABFEB011208BAE7EB0112AC
:1013930008BA2CEC011208BA8AEC011208BAE3EC81
:1013A300011208BADDED011208BA89EF011208BA79
:1013B300CEEF011208BAF7EF011208BA80F001125A
:1013C30008BAF3F0011208BA01F1011208BA25F1C3
:1013D300011208BA7BF1011208BA96F1011208BA98
:1013E30051F2011208BA7DF2011208BAC0F20112D9
:1013F30008BA23F3011208BA33F5011208BA5FF5EC
:10140300011208BA1AF6011208BAFEF6011208BA56
:1014130092F7011208BA78E6051208BAB0E6051287
:1014230008BAD1E6051208BA13E7051208BA77E736
:10143300051208BA81E7051208BA91E7051208BA3E
:10144300C8E7051208BA71EB051208BA39ED05129F
:1014530008BA1DEF051208BABFEF051208BA49F022
:10146300051208BA6931001208BA1232001208BA1A
:10147300F132001208BAFD33001208BA1D3400120B
:1014830008BA3F35001208BAEF36001208BA5C37C3
:10149300001208BA2D38001208BA3339001208BAFC
:1014A300AB39001208BAE639001208BA3F3A001203
:1014B30008BA7A3A001208BAC33A001208BA573B7C
:1014C300001208BAED3B001208BAC23C001208BA77
:1014D300953D001208BA233E001208BA493E001295
:1014E30008BA763E001208BAA73E001208BA743F43
:1014F300001208BA843F001208BAD73F001208BA94
:10150300E43F001208BAF13F001208BAFA3F001292
:1015130008BA5E40001208BABC40001208BA07417C
:10152300001208BA2241001208BA4941001208BA4F
:101533006641001208BA7241001208BA034300124E
:1015430008BA1C43001208BA9843001208BAAB4306
:10155300001208BABB43001208BA5F44001208BA6B
:10156300CB45001208BADE46001208BA7E470012C5
:1015730008BA8847001208BA0748001208BA184880
:10158300001208BA5748001208BA8548001208BA70
:101593005249001208BAA949001208BAE2490012D6
:1015A30008BA384A001208BA564A001208BAA44ABE
:1015B300001208BA6F4B001208BABD4B001208BAEA
:1015C3000A4C001208BA8D4C001208BAB74C00122C
:1015D30008BAED4C001208BAFC4C001208BA5B4D75
:1015E300001208BAD34D001208BA144E001208BAFA
:1015F300644E001208BA8F4E001208BAA94E0012A8
:1016030008BAC34E001208BA984F001208BAA24F84
:10161300001208BADD4F001208BAED4F001208BAE3
:10162300F64F001208BA4750001208BA5B50001276
:1016330008BA7D51001208BA9051001208BAA75196
:10164300001208BABC51001208BA4F52001208BA6D
:10165300C352001208BA6853001208BA7353001237
:1016630008BAD654001208BAF254001208BA3E550A
:10167300001208BAAC55001208BADE55001208BAB7
:10168300F855001208BA5856001208BAF756001255
:1016930008BA4257001208BA9559001208BA2D5ACF
:1016A300001208BAA45A001208BA015D001208BA5F
:1016B300195D001208BA1C5D001208BA285D0012F9
:1016C30008BA3C5D001208BA445D001208BA7B5D9B
:1016D300001208BA6F5E001208BAF95E001208BA67
:1016E3007B5F001208BAFB5F001208BAD2600012D7
:1016F30008BAF460001208BA8D61001208BAEA61F0
:10170300001208BAED61001208BA1A62001208BA90
:101713002F62001208BA9E62001208BAEA6300122E
:1017230008BAFD64001208BA8865001208BA9B66FD
:10173300001208BA6267001208BA9367001208BA67
:10174300B967001208BAC267001208BAF16700123B
:1017530008BAA168001208BA5169001208BAC4692C
:10176300001208BA676A001208BADA6A001208BAE5
:10177300196B001208BA626B001208BA976B001259
:1017830008BAFCF1041208BA7DF2041208BAC4F2D2
:10179300041208BA3AF3041208BA9EF3041208BA00
:1017A30052F4041208BA96F6041208BAC7F80412DF
:1017B30008BA9CFC041208BA1CFD041208BA57FDAF
:1017C300041208BA75FD041208BAD5FD041208BA4A
:1017D300FDFD041208BA2DFE041208BA5EFE0412BF
:1017E30008BA8BFE041208BAE8FE041208BA33FFE3
:1017F300041208BA4ACD051208BAC6CD051208BAB2
:10180300F2CD051208BA24CE051208BA86CF051206
:1018130008BAA2CF051208BAE0CF051208BA6DD0F4
:10182300051208BAC9D0051208BA8FD1051208BA31
:101833004ED2051208BA93D2051208BAF4D2051291
:1018430008BA69D3051208BAA3D3051208BAFBD3A1
:10185300051208BA1DD4051208BAB5D4051208BA80
:101863005CD5051208BAA9D5051208BAD2D5051256
:1018730008BA13D6051208BAC0D7051208BAA4D8F5
:10188300051208BA55D9051208BAACEF061208BA00
:10189300BDEF061208BA5BF0061208BAEF7F00121A
:1018A30008BAC5FF031208BA75F0061208BA85F024
:1018B300061208BA9AF0061208BA2BF1061208BAF1
:1018C300E2EC061208BA66ED061208BACCED06126F
:1018D30008BAF27F001208BAE1FF011208BAF1FF59
:1018E300011208BAF4FF011208BAF7FF011208BA8D
:1018F300F87F001208BAD8E1061208BAFAE1061214
:1019030008BA65E3061208BAE9E3061208BAB8FF93
:10191300011208BAC1FF011208BACAFF011208BABC
:10192300D8FF011208BAF89D061208BA659E06127E
:1019330008BA2D9F061208BA24A0061208BA1DA2DF
:10194300061208BA84A2061208BADCA2061208BA62
:10195300EDA2061208BAFDA2061208BA70A3061277
:1019630008BA86A3061208BA91A3061208BA9FA35F
:10197300061208BAB1A3061208BAC4A3061208BA1B
:10198300F0A3061208BA96A6061208BAEDA6061226
:1019930008BA29A7061208BA3DA7061208BA56A71D
:1019A300061208BA47A8061208BA23A9061208BAEB
:1019B30037A9061208BAECE3061208BA10E40612B5
:1019C30008BA29E4061208BA67E4061208BA9DE4C5
:1019D300061208BAD0E4061208BADAE4061208BA04
:1019E30046E5061208BA49E5061208BA53E5061297
:1019F30008BA60E5061208BA297D001208BA4C7DC0
:101A0300001208BA977D001208BAB57D001208BA11
:101A1300D07D001208BA367E001208BA427E001248
:101A230008BA9F7E001208BAC37E001208BA897FE3
:101A3300001208BA967F001208BAA77F001208BAEC
:101A43006AFF041208BA82FF041208BAAEFF041236
:101A530008BA93FA051208BAE9FA051208BA47FC5C
:101A6300051208BA55FC051208BA69FC051208BA32
:101A730086FC051208BA5D9A031208BAAEFC051279
:101A830008BA30FD051208BA95FD051208BA1DFE05
:101A9300051208BA95FE051208BA6EFF051208BAB8
:101AA3007EFF051208BA8DFF051208BA52F306121B
:101AB30008BA76F3061208BA9EF3061208BAC6F3FA
:101AC300061208BAC9DA061208BAF0DA061208BA18
:101AD3000FDB061208BA84DB061208BAC2D7061255
:101AE30008BA819F031208BAF2D7061208BAFBD7C5
:101AF300061208BA19D8061208BA23D8061208BA69
:101B03002DD8061208BA40D8061208BAD1D8061240
:101B130008BA40D9061208BA6ED9061208BAC2D951
:101B2300061208BA0EDA061208BA29DA061208BA39
:101B330033DA061208BA59DA061208BABEDA0612FE
:101B430008BAD2EE061208BAF4EE061208BA82EF09
:101B5300061208BAD57F001208BAF8F0051208BABF
:101B630024F1051208BA47F1051208BA5AF1051211
:101B730008BA75F1051208BAD5F1051208BA03F2CD
:101B8300051208BA0BF6051208BA48F7051208BA87
:101B93007AF7051208BAE1F7051208BA84F90512B3
:101BA30008BAACF9051208BAC1F9051208BAD1F995
:101BB300051208BA11FA051208BA53FA051208BA3F
:101BC30063FA051208BA33E8061208BA43E80612A4
:101BD30008BA67E8061208BA90E8061208BABAE823
:101BE300061208BADEE8061208BAF5E8061208BAC1
:101BF30023E9061208BA46E9061208BA3BF10612AF
:101C030008BA81F1061208BAF0D0061208BA00D158
:101C1300061208BA1ED2061208BA52D2061208BA1F
:101C230074D2061208BA9CD2061208BAB5D20612AA
:101C330008BAF1D2061208BA57D3061208BA9CD3CF
:101C4300061208BAE1D3061208BA0ED4061208BA6D
:101C530046D4061208BA5FBD061208BAC1BD061201
:101C630008BA6EBE061208BAA5BE061208BA3EBF6F
:101C7300051208BAEDBF051208BA1FC2051208BA49
:101C8300F0C4051208BA80C6051208BAB9C605120F
:101C930008BA44C7051208BAC4CA051208BA0CCC5C
:101CA300051208BAADEA061208BAF8EA061208BA2B
:101CB30028FF021208BA6197061208BA339A06126D
:101CC30008BA459B061208BA459C061208BAFE9C40
:101CD300061208BA73AE061208BA32B1061208BA6F
:101CE300CFB1061208BAFBB1061208BA29B206121E
:101CF30008BA5EB2061208BA86B2061208BAE6B28B
:101D0300061208BA42DA051208BA36DE051208BA14
:101D1300CDDF051208BAFBE0051208BAD7E10512B8
:101D230008BA85E3051208BA3AE5051208BA06E6C9
:101D3300051208BA5AE6051208BA55DD061208BAA2
:101D430060DD061208BA81DD061208BA026C0012C1
:101D530008BA0672001208BA6B73001208BA477504
:101D6300001208BA2576001208BA1C77001208BAC6
:101D73005978001208BAA279001208BABA7A001286
:101D830008BACC7B001208BA987C001208BAD5D2E4
:101D9300041208BA0DD3041208BAECDD041208BA0F
:101DA300E5DE041208BA34E0041208BA95E104121D
:101DB30008BA6EE2041208BA40E3041208BAA5E4B2
:101DC300041208BA83E5041208BA88E6041208BAB2
:101DD3003AE7041208BA6AE7041208BA23E90412BC
:101DE30008BA99E9041208BAB2E9041208BA13EB63
:101DF300041208BAD1EB041208BA70EC041208BA40
:101E030011ED041208BA76ED041208BA14EE0412A6
:101E130008BA97EE041208BAB5EE041208BACCEF6A
:101E2300041208BA9AF0041208BA49F1041208BA63
:101E33006AE5061208BA94E5061208BAA8E606127D
:101E430008BAABE6061208BAEFF1061208BA42F274
:101E5300061208BA84F2061208BA94F2061208BAF5
:101E63007F90061208BAB790061208BAFF900612BE
:101E730008BA6891061208BA8991061208BAA291A3
:101E8300061208BA5492061208BA5D92061208BAEC
:101E9300AE92061208BAE492061208BAFB92061230
:101EA30008BA6893061208BAF893061208BA2E9471
:101EB300061208BA7794061208BAD894061208BA1A
:101EC3001295061208BA7A95061208BACD9506122B
:101ED30008BA1096061208BA4D96061208BA5F960B
:101EE300061208BA7196061208BAAB96061208BA19
:101EF300F796061208BA3597061208BA9AB306126D
:101F030008BAE0B4061208BA09B5061208BA1AB537
:101F1300061208BA32B7061208BA52B7061208BA3E
:101F230096DF061208BACADF061208BA19E00612CB
:101F330008BA75E1061208BA429C051208BA809DD8
:101F4300051208BABC9D051208BA8B9F051208BA80
:101F5300B59F051208BA4CA2051208BA8CA2051245
:101F630008BA22A4051208BAB7A4051208BA15A51F
:101F7300051208BA9BA5051208BAD3A5051208BA1B
:101F830015A6051208BA86A7051208BA0AA90512EA
:101F930008BA33AB051208BA61AB051208BA8DABA8
:101FA300051208BA96AB051208BAECAB051208BACB
:101FB3007CAC051208BA7FAF051208BA01B005124E
:101FC30008BA9EF2061208BAB4F2061208BABEF2B2
:101FD300061208BA1AF3061208BA67FB031208BA04
:101FE30080FB031208BA25FC031208BA65FC03122E
:101FF30008BA7EFC031208BAB1FC031208BAFEFC4D
:10200300031208BA32FD031208BA74FD031208BAA8
:102013004DFF031208BAB8FF031208BA7EE906128D
:1020230008BAD8E9061208BA32EA061208BACFEBA0
:10203300061208BA41EC061208BA7FEC061208BA77
:10204300C0EC061208BA7C88061208BA8288061207
:1020530008BAC988061208BAD58A061208BA058BC7
:10206300061208BA6F8B061208BA2A8C061208BA2F
:102073006D8C061208BA9E8C061208BA288D0612B9
:1020830008BA3F8D061208BA4C8D061208BA568D4F
:10209300061208BAF68E061208BAE88F061208BAB4
:1020A3004690061208BA0080061208BA1680061275
:1020B30008BAC880061208BAF281061208BAE78283
:1020C300061208BA8483061208BABF83061208BA36
:1020D3003184061208BA8F84061208BA9F84061246
:1020E30008BAC684061208BA1885061208BA80868A
:1020F300061208BA8586061208BAA786061208BA17
:102103005EB0051208BA68B0051208BAFBB0051232
:1021130008BA3DB1051208BAF5B1051208BA6CB296
:10212300051208BAE1B2051208BA65B3051208BA76
:10213300ABB3051208BAB7B5051208BA56B60512FD
:1021430008BAB7BB051208BAB3BC051208BA43BD37
:10215300051208BA68BD051208BA36BE051208BAD8
:10216300BCBE051208BADBBE051208BA05BF0512CC
:1021730008BA69AB041208BA93AB041208BAAEAB3F
:10218300041208BACCAB041208BAFEAB041208BAA4
:1021930080AC041208BAD4AC041208BA96AD041287
:1021A30008BAD8AD041208BA17AE041208BA4CAE76
:1021B300041208BA15AF041208BAC9B0041208BA57
:1021C30006B3041208BAE8B4041208BAC5B5041277
:1021D30008BA29B7041208BAC2B7041208BA11B868
:1021E300041208BA56B8041208BA54B9041208BA49
:1021F300E2B9041208BA49BA041208BAF8BA0412C6
:1022030008BA8CBB041208BADABB041208BA06BCBB
:10221300041208BA29BC041208BAB3BC041208BADF
:102223008BBD041208BA7CBE041208BA5ABF04124A
:1022330008BA5CC0041208BAA9C1041208BAF9C1E9
:10224300041208BA2CC2041208BA6AC2041208BAE9
:10225300C0C3041208BA9DC4041208BAC0C504124C
:1022630008BA99C6041208BAA2C7041208BA40C928
:10227300041208BA20CA041208BA74CA041208BAAB
:1022830034CB041208BA4FCD041208BA63CE041239
:1022930008BA4BCF041208BA5BCF041208BA60D055
:1022A300041208BACCD0041208BAD6D1041208BA60
:1022B300CDDC021208BA25DD021208BAC5DD02120E
:1022C30008BA42DF021208BA2EE0021208BAEBE0A3
:1022D300021208BA02E1021208BA53E1021208BA62
:1022E300C7E1021208BA22E2021208BA35E2021268
:1022F30008BA99E2021208BA08E3021208BAB7E56B
:10230300021208BABCE6021208BA17E7021208BAA8
:102313006BE7021208BA1FEA021208BA6FEA021246
:1023230008BAF0EA021208BA32EB021208BA0CEC4D
:10233300021208BA45EC021208BA64EC021208BA97
:10234300AFEC021208BAC5EC021208BA80ED021211
:1023530008BA67EE021208BA72EE021208BAC0EEA9
:10236300021208BA15EF021208BA61EF021208BA94
:10237300BCF0021208BAE6F0021208BA7EF30212A7
:1023830008BAA8F3021208BAB3F4021208BAE2F4C4
:10239300021208BA5AF5021208BA35F6021208BA3E
:1023A30077F6021208BAEBF6021208BA05F802121F
:1023B30008BA52F8021208BA65F8021208BA68F8A5
:1023C300021208BA71F8021208BA8CF8021208BA9B
:1023D30004F9021208BA3DF9021208BA59F90212B5
:1023E30008BA86F9021208BAADF9021208BAD1F98D
:1023F300021208BA4AFA021208BABDFA021208BA5D
:1024030000FB021208BA0AFB021208BA39FB0212D5
:1024130008BA4FFB021208BA6BFB021208BA9AFB06
:10242300021208BABAFB021208BA03FC021208BA73
:102433003EFC021208BA4AFD021208BAADFE0212AD
:1024430008BACCFE021208BAE3FE021208BAF5FE7D
:10245300021208BAE5ED061208BAF6ED061208BA3A
:1024630081EE061208BA4BA9061208BA89A9061208
:1024730008BA22AA061208BA2DAB061208BA75AD1D
:10248300061208BAF2AD061208BA53F8011208BAD6
:10249300A2F8011208BA60FA011208BA34FC011258
:1024A30008BA72FC011208BA53FD011208BA5DFEA4
:1024B300011208BA7FFE011208BADBFE011208BA44
:1024C3005CFF011208BA0080041208BA22800412C9
:1024D30008BA9181041208BADA81041208BA4C824C
:1024E300041208BACE82041208BA4383041208BA4B
:1024F3009483041208BAFB83041208BAA684041254
:1025030008BA1B85041208BA5A85041208BA9589B9
:10251300041208BAB08B041208BAE98B041208BA81
:10252300288C041208BA3C8F041208BACC8F041208
:1025330008BA5D91041208BAA292041208BAB293BF
:10254300041208BA2194041208BAF894041208BABF
:102553007C95041208BA9095041208BA5C9604128A
:1025630008BA9197041208BAB199041208BABC9B2D
:10257300041208BA9C9C041208BA199F041208BAE0
:10258300EF9F041208BAFBA0041208BA4DA4041268
:1025930008BA5DA4041208BA04A6041208BA94A6E1
:1025A300041208BAC5A7041208BA3BA8041208BA51
:1025B300BFA9041208BAFEA9041208BAA5AA0412F4
:1025C30008BA0080051208BA9B80051208BA0E816A
:1025D300051208BA2881051208BAC781051208BA7C
:1025E3000F82051208BA4A83051208BA89830512B5
:1025F30008BA0084051208BA5184051208BAB084D7
:10260300051208BA5C85051208BA3188051208BAA2
:102613003789051208BAAC89051208BA878B0512E7
:1026230008BA2A8C051208BAE38C051208BA488D39
:10263300051208BAB78D051208BADA8E051208BA60
:10264300CF8F051208BA0A90051208BA2190051215
:1026530008BAE490051208BA2391051208BA9E91AC
:10266300051208BA1593051208BACF94051208BAD1
:102673002296051208BA9097051208BABC9805125B
:1026830008BA4999051208BAB999051208BACB9A3A
:10269300051208BAB4DB031208BA1DDC031208BA28
:1026A30065DC031208BAA9DC031208BA1CDD0312A5
:1026B30008BA76DD031208BAB1DD031208BA4BDE9D
:1026C300031208BAA5DE031208BA11E0031208BA0E
:1026D3008AE0031208BAB4E0031208BAC8E103128D
:1026E30008BADCE2031208BA04E3031208BA02E4EC
:1026F300031208BA13E4031208BA2BE4031208BA4C
:1027030031E5031208BA54E5031208BA23E60312AB
:1027130008BA4DE6031208BA64E6031208BA8AE659
:10272300031208BAC9E6031208BAE9E6031208BAA3
:1027330010E7031208BA28E7031208BA0BE80312DA
:1027430008BA65E8031208BACCE9031208BA4AEAE0
:10275300031208BA6EEA031208BA85EA031208BA2A
:1027630059EB031208BAF2EB031208BA18EC03127E
:1027730008BA68ED031208BA87ED031208BA06EE29
:10278300031208BA3DEE031208BA7BEE031208BA2D
:1027930011EF031208BA86EF031208BA6AF00312A4
:1027A30008BA48F2031208BA1DF3031208BA69F310
:1027B300031208BA74F4031208BA92F5031208BAA2
:1027C300B0F6031208BABEF6031208BABAF7031238
:1027D30008BA5CF8031208BAA2F8031208BAB7F8E9
:1027E300031208BAC9F9031208BA6AFA031208BA3B
:1027F300C6FA031208BA4EC9061208BA09CB061262
:1028030008BAD1CB061208BA26CC061208BAACCC49
:10281300061208BA58C1061208BA7DC1061208BAD0
:10282300C1C1061208BAE7C1061208BA0EC20612DF
:1028330008BA26C2061208BA3EC2061208BA56C21F
:10284300061208BA00C3061208BA42C3061208BA2F
:1028530057C3061208BA5EC4061208BA79C4061230
:1028630008BA82C4061208BA8BC4061208BA94C402
:10287300061208BA9EC4061208BA1BC5061208BA85
:10288300A6B8061208BAD2BC061208BAEEBC0612E3
:1028930008BAF3BC061208BAC1CD061208BA3BCF78
:1028A300061208BA53C5061208BA69C5061208BA51
:1028B30030C7061208BA7BC7061208BAE7C7061262
:1028C30008BAEEC8061208BA1DC9061208BA2FC9FB
:1028D300061208BAD8E6061208BA9AD4061208BA3B
:1028E300F7D4061208BA37D5061208BA39D6061233
:1028F30008BA51D6061208BA63D6061208BA8FD69A
:10290300061208BAC6D6061208BAD6D6061208BAEE
:10291300ECD6061208BA11D7061208BA9FD70612C8
:1029230008BA8CFF011208BA7999031208BA95986C
:10293300031208BAAB95031208BA6894031208BAD3
:10294300CF91031208BA8A91031208BA3091031285
:1029530008BA9190031208BA3C90031208BA698F1F
:10296300031208BAA38E031208BA678E031208BAB9
:10297300FA8D031208BAF28D031208BA678D031297
:1029830008BAF78C031208BA488C031208BA3D8CB4
:10299300031208BA2E8C031208BA0D8C031208BA5C
:1029A300D98B031208BAAD8B031208BA7F8A0312BC
:1029B30008BA7388031208BAF99E031208BA448846
:1029C300031208BAEA9E031208BA779E031208BAE2
:1029D3005B9E031208BA3D9E031208BA259D03129B
:1029E30008BA009D031208BA109C031208BA9C9BF4
:1029F300031208BA2888031208BAD287031208BA46
:102A03009987031208BA1187031208BA059B0312A8
:102A130008BAC586031208BA7E86031208BAB185BE
:102A2300031208BA3585031208BA939A031208BA37
:102A33008D84031208BADBD7061208BAE6830312A1
:102A430008BA8883031208BA5D83031208BA0E8397
:102A5300031208BAD082031208BAAE82031208BA6C
:102A63008B82031208BA7282031208BA4D820312D0
:102A730008BA0582031208BA4F81031208BAC38049
:102A8300031208BA5780031208BA0080031208BA67
:102A9300DCFF031208BA829A031208BADAFF0312A0
:102AA30008BAD8FF031208BA9BFC0500000080FB9C
:102AB3008F000100C61C87000100C51C35000400FF
:102AC300421E25000200461E26000200481E270063
:102AD30002004A1E28000100541E29000100551E51
:102AE30084000400561E860001005A1E2A000100BD
:102AF3005B1E2B0001005C1E2C000100601E2D00DC
:102B03000800A71C2E000100611E2F000100621E99
:102B130030000100631E31000100641E3200010019
:102B2300AF1C33000100B01C34000100651E3600E9
:102B33000100B11C38000100661E390001005F1E50
:102B4300830002007A1E63000100C21C64000100BE
:102B53005D1E650001005E1E6D000100C31C710057
:102B630008009F1C66000100791E430001006A1ED5
:102B7300440002006B1E450001006D1E460002006A
:102B83006E1E47000800BA1C48000100701E4B006F
:102B93000100711E040001007C1EA10001007F1EC4
:102BA300370001007E1E880001007D1E3C000100ED
:102BB300B21C3D000100671E49000200721E67003F
:102BC3000100C41C4D000200741E4E000100761E5D
:102BD3004F000200771E3E000100B91C51000100A6
:102BE300B31C52000100681E53000100691E54000B
:102BF3000100B41C00000000000000013636010192
:102C0300000102010001030100010401060605029F
:102C13000000070100340801000F090401010D0140
:102C230000FF0E08000017020000190100FF1A013F
:102C330000011B0100FE1C0100081D0200001F0112
:102C4300000120010001210200002301000F2402E2
:102C530000002601000127010008280200FF2A01C5
:102C630000072B0102402C0100002D0100012E0161
:102C730000012F0100FF30010B1D310800003A0154
:102C830000083B01000F3C0100013D0100FF3E0431
:102C9300000042040000460400004A0400004E0401
:102CA300000052040000560400005A04000001030F
:102CB300710301030103010301030103220302035F
:102CC30001031003000300030003000300030003D8
:102CD3000003420300032403060300030003040369
:102CE300120325032303250323030403040300031F
:102CF30000030003440300030003230300036503ED
:102D030021003503810300030503000300030003CF
:102D13000003250323030304710402046004110464
:102D23007004020402040104020410046104000498
:102D3300140463047304720462044304000413045C
:102D43000604000400040404120400040004000444
:102D5300000451046400000400040004440400045B
:102D630000040004000465040004350481046400C5
:102D730005040004830400040300710030016000B3
:102D83001100700031022003500480001000610024
:102D9300000014006300730072006200430000002F
:102DA30013000600000000000400120000000000F1
:102DB3000000000004000400370037003C02440018
:102DC30000000000000000006500000035008100E5
:102DD30000000500000083000000010171010101F2
:102DE3000101110101013101010101018001100102
:102DF30061013B001400630173017201620143012D
:102E03000001130106013D01350004011201000117
:102E130000010001000104010401330133013C01FD
:102E23004401320136000001000165010001350053
:102E33008101000105018201830100010302710286
:102E430030016002110270020102020202028002DA
:102E5300100261023A0041006302730272026202CD
:102E630043020002130238000002000204021202AD
:102E730000020002000200020402040237003700CD
:102E83003C02440200023900000200026502000213
:102E9300350281020002050282028302000236002B
:102EA3000100060000000F00000000000000000009
:102EB3000000000003FFFF00000403FFFF0000FF0A
:102EC300FF0FF4010005C4040320000100000B0000
:102ED3000000000000000003010F000000000000DC
:102EE30000000000000000000000000000000000DF
:102EF30000000000000000000000000000000000CF
:102F030000000000000000000000000000000000BE
:102F130000000000000000000000000000000000AE
:102F230000000000000000006C21122100000000DE
:102F3300000000000000000000000000000000008E
:102F4300000000000000000000000000000000007E
:102F530000000000000000000000042613006225AA
:102F63001F0068251F806E25010004260200EA2445
:102F73000300F0240400F6240500FC2406000825C1
:102F83003000262531002025320032253300382534
:102F930035003E253400442536004A2511005625C8
:102FA30014005C2515001A25FFFF00000A0000002D
:102FB30002000000040000000800000010000000F0
:102FC300200000004000000080000000000100001D
:102FD30000020000000400000008000000100000D0
:102FE300002000000040000001CE1006041108FE7E
:102FF300100B1C1110860D0A2E1102D41005F210AD
:1030030007DA100CB6100DC210645229FF00000736
:10301300ECFDFDFDECDCDCCCBCACAC9C9C8C7C7C8A
:103023006C6C5C5C5C4C4C3C3C2C2C1C1C00160FEC
:1030330000000B150B020002220F3300000E6B0081
:103043006A00690016001500300016001E005A6958
:1030530067426565416C6C69616E63653039010374
:103063000507090B0D0F00020406080A0C0D140ACC
:10307300E5D5C5B5A5A595858575650A0901070536
:103083000001ED3001ED30303016181920231A1CE1
:103093001E3000011916181616182303000C0E0211
:1030A3000B040B0A0708000F303017181921301BC7
:1030B3001D1F3000393D3F373C3C362C442D000367
:1030C3004A49434E181A250502020402010101016F
:1030D3000902000800003101141B0A061B7E3000A0
:1030E300E803000000BE040A12300008FA060E00CE
:1030F3007130000000007F00E8031509000400039D
:10310300FF1E1E0A050C100404081000FF0C2809FA
:1031130003010C050808E004123999A2E792AF22D3
:10312300E4F0A3F0A3F022A3123123A3F0227F0C37
:1031330002060FE0F508E4F509F50AF50B22740120
:10314300F0900B6AE0640F2274091208CF7F040227
:10315300060FA3A3E024F5C3941322900B8A125CF9
:10316300BC7A147B0022C082C0839005E374C4F050
:10317300A37414F0A374D6F0A37414F09005E77449
:10318300ACF0A37414F0A374A6F0A37414F0A374A6
:10319300E2F0A37414F0A374E8F0A37414F0A3741E
:1031A300DCF0A37414F0A37494F0A37414F09005EA
:1031B300F374B8F0A37414F0A374BEF0A37414F002
:1031C300A374B2F0A37414F0A374EEF0A37414F018
:1031D30090060412524960061254B3121F3290062D
:1031E300011249427408F0A3E4F0A3F09006A4F09E
:1031F300900606F07C0BFDF97A077B06121E727CA3
:103203000B7D0079007A127B06121E7202494B7401
:10321300F712039E74F7120999EAFEEBFF1247694E
:1032230074051232DF7403F0EE2402FAE43F123223
:10323300B9242DFCE43FFD8C828D831233F71232C7
:10324300C86008123B4174FFF0A3F0EE242BE43F67
:103253001C1CFD8C828D83A3E0C0E08A828B8312C9
:10326300477AD0E01232C888828983124F722403CE
:10327300125A861220407408120BC37403F0900B89
:103283007F12071174021209637903EEFAEFFB123E
:10329300169274021208CFE9F5087007EEFAEFFBF5
:1032A300121566A9087409023B51F582E43FF583C0
:1032B300126733124F67FB8A828B831232D7E8F08F
:1032C300A3E9F0EE22125CDA1232D7E8F0A3E91296
:1032D3006298E0221233C28A828B8322F0A3E4F045
:1032E3001232E722EE240DF582E43FF5832274F1D6
:1032F30012039EEAFEEBFF8C088D09890A1233CC78
:103303008A828B831233C2740F120BC31233E5E824
:1033130024FF18E934FFF988828983E50A1233D739
:10332300900B841233D4900B831233D47411120B89
:10333300C31233E5EE2404FCE43FFD880B8A828B41
:1033430083E0F50C8C828D83E0250CC3950B125C16
:10335300D6E8F0A3E91246D6A3A3A3A3A3A3A3A3EA
:10336300E064037008124A32F0A3E480031236D8F3
:103373001232E27409F0750C07750D06750E0078AC
:103383000C1209091236CC121E6074031208CF7591
:103393000CFF750DFF780C12090DAC08AD0979030C
:1033A300EEFAEFFB12169274021208CFE9F50870D9
:1033B30007EEFAEFFB121566A9087F0702060FE076
:1033C30024FFF8A3E034FFF922EE2402FAE43FFBE2
:1033D300221233F71233DB22F0E824FF18E934FF1B
:1033E300F922E0F50CA31233F71233DB88828983C9
:1033F300E50CF022E08882898322C082C083900694
:1034030023E0C39408400474078001E08A828B831D
:10341300F033333354F8F902494B74F012039EEA44
:10342300FEEBFF890C8C0E8D0F750A00A2AFE433FF
:10343300F50BC2AF90061D803F123505503712358C
:103443001664037030EE24F9FEEF34FFFF85088223
:10345300850983A3A3E02405FCA3E03400FDEEFA71
:10346300EFFB122040EE24FF1EEF34FFFF74102504
:103473000AF50A150C1246A312672FE50C6006E540
:1034830008450970B4E50BA2E092AFA2AFE433F5AF
:103493000BC2AF90061D802C2402FAE43509FB8A87
:1034A300828B83125CC52406F582E438F5831235DA
:1034B300238A828B8312350BA3A3123523050A15A6
:1034C3000C1246A31246B86022123516640270F13C
:1034D300123505E50840C1123806A2E550E3850E12
:1034E30082850F837401F0E50C70D6E50BA2E092A0
:1034F300AF8E828F83E50AF0EE24FFFAEF34FFFBF1
:103503008035123811A2E62212350F221260BAA3B7
:10351300A3A3228508828509831260B41256EE2282
:10352300E08E828F83F0EE24FF1EEF34FFFF221222
:10353300176A74041208CF7F0802060F74EC120393
:103543009E74F512099989138A128B0F8518828547
:103553001983E4F00412095B121476E9F8900B69FD
:10356300E0292434F508FA7B00121E8A8A0A8B0BA1
:10357300AE0AAF0BEE4F70030236C0EE2402F50A1B
:10358300E43FF50BA808EE28F8E43FF9850A8285A5
:103593000B831232C12404F510E43FF51185108228
:1035A300F583E4F0900B69E0FCF8C3E498F895E048
:1035B300F9850A82850B83E028F508A3E039F5092C
:1035C300900B6712597E750E00780C1209097D0065
:1035D300AA08AB09121E6074031208CFAC18AD1908
:1035E3007401120BC3E0F9E50824FFFAE50934FF7F
:1035F300FB12147C8A828B83E4F0EA24FFF508EB48
:1036030034FFF509E50FC454F0F99006A5E0C4337F
:103613003354C0F8900B63E0A2E0E433131348493A
:10362300440F1236E0E512C454F045138508828531
:103633000983F0A808850A82850B83E0FA85108246
:10364300851183E02AC398F0850A82850B83E8F00D
:10365300A3E509F01236D81232E2E4F0740A120B31
:10366300C3E4F0750812750906F50A78081209090A
:103673001236CC121E6074031208CF851882851986
:1036830083E06009EE240E1247FF4408F012167A15
:10369300E9F9E4F508F509780812090D740412092B
:1036A30063EEFAEFFB12169274021208CFE970066A
:1036B300EEFAEFFB800BEEFAEFFB121E907A007B23
:1036C30000740B1208CF0231317C0B7D00EE2418FD
:1036D300FAE43FFB2212476DE4F0A322E08508825F
:1036E3008509831236EA22F01259522274F3120327
:1036F3009E8A0A8B0BA2AFE433F50CC2AF750800A8
:1037030075090090061D802C12392D5024850A82DC
:10371300850B83A3A3126B5C8E828F83A3A31254A6
:10372300B6121680E9600A123753C2E6F08E088F8C
:1037330009123922123BDB70CFE5084509600612F6
:10374300380DD2E6F0E50CA2E092AF7F0502060F3A
:103753001237572212596BE02274F012039EEAFECD
:10376300EBFF8C0C8D0D750E00A2AFE433F50FC289
:10377300AF75080075090090061D8020850A08852D
:103783000B0912380DD2E4F0E508123806D2E7F03F
:10379300E50A24FBF582E50B34FFF583E0F50AA384
:1037A300E0F50BE50A450B6043E50A12458E350B40
:1037B300F583E0A2E750D9850A82850B83A3A31280
:1037C3000711AC0CAD0DEEFAEFFB12168674021264
:1037D30008CFE960BBE508450960A1E508240D129F
:1037E300381964017006123822D2E4F0E50FA2E022
:1037F30092AFE50845096006121560750E01A90E22
:1038030002353A1245B812381C2212381122E50843
:10381300241112381922F582E43509F583E0228553
:1038230008828509831260B4E02274F212039E7445
:10383300FE120999750C00750D0085188285198390
:10384300E4F0A3F0A2AF33F50AC2AF90061DE0FE89
:10385300A3E0FF8035EE24FBF582EF34FF12672DE2
:10386300780C12090DEEFCEFFD7A1D7B06121EC0CB
:1038730074021208CFEEFCEFFDAA18AB19121EAEAC
:10388300AE08AF09900623E014F0EE4F602712391B
:103893002D501DEE240BF8E43FF988828983E02440
:1038A300FFF0A3E034FFF08882898312524960A5B8
:1038B30012391E8099E50AA2E092AF900623E060D8
:1038C30031900B6AE0640F60069006A4E070237ADF
:1038D300FB7B0512177690818212070D7AFB7B051D
:1038E30012176A74041208CF800874F0124B69121D
:1038F3001554AA18AB19121EB48A0A8B0BAE0AAF61
:103903000BEE4F6013121488123753A2E28E828F8C
:1039130083A350D674E980D4023BE38E0C8F0DEE63
:1039230024FBF582EF34FFF58322123757A2E722F7
:1039330074F712039EEAFEEBFF1214881247771204
:103943000529E96401900B86700AE02401F8A3E0DD
:1039530034008004E0F8A3E0F9124DC512517790CA
:103963000623E07021900B6AE0640F70197AFB7BE9
:103973000512177690818212070D7AFB7B051217C9
:103983006A74041208CFA9A8C2AF900623E00412F8
:103993003999A2E7800DF0E9A2E7E433F8E922E5DB
:1039A30008A2E092AF024C0574F712039EEAFEEB05
:1039B300FF1239E0F0121488EEFCEFFD7A1D7B064E
:1039C300121EBAA9A8C2AF900623123119900B6A2E
:1039D300E0640F70057908121626024C051237575A
:1039E300C2E42274F712039E74EA120999EAFEEB09
:1039F300FF900B63E060408518828519837401F0A2
:103A0300120BC3E4123AB8120BC3AA82AB8312207F
:103A1300408E828F83123828C0E0740A120BC3D001
:103A2300E0125CEB740B120BC3AA82AB831216AACF
:103A3300AA18AB191228807416023B5174F71203AB
:103A43009EEAFEEBFF12146AE9F974DC69601E74E6
:103A5300DD69601974E469601474F369600F74DEDE
:103A630069600A74DF69600574DB697007EEFAEF59
:103A7300FB12162C024C0574F712039E74EB120909
:103A830099EAFEEBFF8518828519837406123AB80A
:103A9300120BC3AA82AB83122040125CF0740A1289
:103AA3000BC3AA82AB831216AAAA18AB19122880D9
:103AB3007415023B51F0EE2413FCE43FFD74022223
:103AC30074F712039E74F7120999EAFEEBFFEE24D2
:103AD3002D1247FF6065124390AA18AB19122040BC
:103AE3007408120BC37403F0900B7F120711123B7F
:103AF30041120711900B92E0F97404120963EEFA74
:103B0300EFFB12147074041208CFE9F974DC6960D6
:103B13002374DD69601E74E469601974F3696014C9
:103B230074DE69600F74DF69600A74E869600574A4
:103B3300DB697007EEFAEFFB12162C0232A8EE12C5
:103B43003B4622242BF582E43FF5832274031208BB
:103B5300CF024C0574F212039E8A088B09750C0080
:103B6300750D00750AE7A2AFE433F50BC2AF9006FB
:103B73001D800312391E123BDB603512392D50F3C1
:103B83001247FC640170ECEE242FF582E43F123DF2
:103B93008AE06870DE780C12090DEEFCEFFD7A1DE9
:103BA3007B06121EC074021208CF900623E014F0A5
:103BB300E50BA2E092AFEE4F6013EEFAEFFB1214A7
:103BC3008879F0EEFAEFFB12162C750A00A90AAAFF
:103BD30008AB0912162C800DE0FEA3E0FFEE4F2286
:103BE30074021208CF7F0602060F74F412039E7448
:103BF300F7120999EAFEEBFF8E828F83A3E064F349
:103C03007003023C978E828F83A3E064DF7003020C
:103C13003C978E828F83A3E064E860788E828F83E3
:103C2300A3E064DB606E1214CAE9F508705EEE244B
:103C33000E1247FF6056123CA1121512EA4B604C5C
:103C43007408120BC3123CAB1207117508FF7509F8
:103C5300FF780812090D8E828F83A3A3A3A3A3A3C6
:103C6300A3A3E0F974041209631214707404120814
:103C7300CFE9F50874F36508601274DF6508600C1A
:103C830074E86508600674DB6508700F8E828F83A5
:103C9300A3E508F0EEFAEFFB1214D602314BEE2443
:103CA3000FFAE43FFB79092274021264F574FFF002
:103CB300A3123CB822123CBC22124F7BA3A3227452
:103CC300F512039E8A088B097E008A828B83A3A345
:103CD300A3A3A3A312315540027EE88A828B83A358
:103CE300A3A3A3A3A3A3A3A3A3E0C3941040047E0D
:103CF300E880138A828B83A3A3A3A3A3A3A3A3A371
:103D0300A3E0640F600A900681E0540870027EE825
:103D1300EA240BF582E43509123D8AA3A3A3A3A3E6
:103D2300A3A3A3E0C398500CEA240B123819640F21
:103D330060027EE8900B83E0F47003A3E0F470026A
:103D43007EEC7A237B00121F2C9006041254C6903B
:103D530006041252496029850882850983A3A3A911
:103D630082AA8389088A09750A0078081209097CDE
:103D7300237D001254B3121E6074031208CF800215
:103D83007E1AEEF9026696F583E0F88A828B83A3A6
:103D9300A32274F512039EEAFEEBFF8E828F83A3A8
:103DA300A3A3A3A3A3A3A3E0900B6A1263D8900BCE
:103DB300851263BE900B651263DD9006A5F0F912C0
:103DC3001AEE9006A5E06018EE2404FAE43FFB79AE
:103DD30050121AD6EE2406FAE43FFB79E1121AD602
:103DE3009006A412314160047401800274009006AD
:103DF300061263C41209097C0B7D007A077B061245
:103E03001E6074031208CFEE2418F508E43FF50989
:103E130078081209097C0B7D007A127B0602668EF4
:103E230074F712039EEAFEEBFF8E828F83A3E0708A
:103E3300061254B31214D08E828F83742C124B69E2
:103E4300121644024C0574F712039EEAFEEBFF9030
:103E53000604125249600D1254B3900604E4F0A311
:103E6300F0121F328E828F837408124B69122880DE
:103E7300024C0574F612039E9006A4E060139006AC
:103E830006E0700D123E97121482EA4B600312157E
:103E930066025FF6900B65E0FB900B85E0FA900BF2
:103EA3006AE0F92274F412039E74E7120999EAFE98
:103EB300EBFF750B018E828F83A3A3A3A3A3A3A3FD
:103EC300E0A2E25068EE242BF582E43F126B5A1213
:103ED3003F6512148EE97055908100E0640170050E
:103EE300750B008048123F6D1209097C0B7D00742D
:103EF3001112095B121E6074031208CF12167AE9BD
:103F0300FA740E12095388088909780812090D7585
:103F13000830750900780812090D123B4112071188
:103F2300125C8C790112169874061208CF851882D8
:103F33008519837410123AB8120BC3AA82AB831289
:103F43002034123B41125CB8740B120BC31251772D
:103F5300740D120BC3E50B1249DC1228807419028D
:103F6300314DEE2413FAE43FFB22EE24081263CC16
:103F730022C082C0839006A5E060031216EC0249BA
:103F83004BC082C08390069C74E3F0A37405F0A336
:103F930074E7F0A37405F0A374F3F0A37405F09031
:103FA3001DED7419F0A3742DF09006867464F0A3CC
:103FB3007414F0900628749AF0A37414F090062AEF
:103FC30074A0F0A37414F0900681E044028001E42D
:103FD300F002494BC082C083EAFCEBFD7903024F38
:103FE300E7C082C083EAFCEBFD7905024FE7C0829C
:103FF300C0837908026187C082C08374FE12099965
:10400300900630744EF0A37415F09006327448F0A5
:10401300A37415F0800D7A1D7B06121EB41249D2CB
:1040230012166890061D12524970EB90061F125229
:1040330049600F7A1F7B06121EB41249D21216680A
:1040430080E990061DE4F0A3F09006231231247456
:1040530002800274111208CF02494B74F612039EB8
:10406300E9FF74B629F582E43430F583E493FEFA6C
:104073007B00121E8AEA4B6011EA2E12516D8A826E
:104083008B83A3A3A3A3E4F0802C7A027B00121EEC
:104093008AEA4B601D74AB2FF582E43430F583E478
:1040A300938A828B83F0A3741AF090067CE0F91252
:1040B3001E967A007B00025FF6E9FC740629F8EA93
:1040C300A2E0501EE875F00A84E5F0F96014740A62
:1040D30028C399F8E9C394054004740A28F8740BBB
:1040E30028F8ECC3941340047A1480027A06EA2871
:1040F30079002409F85001097A0A7B0012024EE87C
:10410300F90208B7C082C083900681E05402600AB6
:10411300122886E9600479018002790002494BC0C4
:1041230082C083900681E054026016900623E070FB
:104133000C125246600BE0C81246B050047901805D
:1041430002790002494BC082C0839080FDE0F89061
:104153000625E0C3985005121E8A80047A007B006E
:1041630002494BC082C083121668790002494B741E
:10417300F712039E74FE120999851882851983EA42
:10418300F0A3EB1242E1A3A3A3A3A3E0600A14608C
:104193006024FE6069024262900B6AE0640F60185B
:1041A30012163EE970128518828519831254B6904F
:1041B300062C12477A120529900B92E0C0E085186D
:1041C30082851983124F45D0E01242E174141264C0
:1041D300F1126B5C7A1F7B06121EAEA8A8C2AF90C9
:1041E3000625E0041254CC79201216267402023BF1
:1041F300518518828519831260BC741580D0851887
:10420300828519831242C4A3A3E060538518828573
:104213001983E02402F8A3E03400F9888289831229
:10422300692FE0C0E0851882851983E0FCA3E0CC08
:104233002406F582E43CF583D0E0125CF888828999
:10424300831254C68518828519831245AC8518825A
:1042530085198360131242C960051242D14043AAF3
:1042630018AB1912166880841242C960F21242D147
:10427300501C1246C0FA8518828519831242CBF866
:1042830074CB1251683430F583E4936A6014851853
:10429300828519831242C9640870C41246C0640837
:1042A30070BD1246C0141242E9240AC0E085188288
:1042B30085198312477AD0E01242E9040241D1E022
:1042C300F8A3124F9222E0F8A3E01242F0228518DD
:1042D30082851983125CC91242F1C3940A221242E5
:1042E300FBF5838882221242FB1242F022C8240685
:1042F300F582E438F583E0221264F5E0F8A3E022C6
:10430300C082C08390063412524960081260BD1205
:1043130005298002790002494B74F712039EEAFED5
:10432300EBFF1232E77401F0EE2430F582E43FF53F
:1043330083125A261232C124321247FFC0E0EE2400
:1043430013F582E43FF583D0E0F0EE24331247FF08
:10435300C0E0EE2414F582E43FF583D0E0F0EE24D0
:104363002CF582E43FF583120711124390EE242EBD
:104373001247FFF912169274021208CFE9F508707A
:1043830007EEFAEFFB121566A908024C05EE24238B
:10439300FCE43FFD22C082C08312163EE96004792B
:1043A300208002790102494BC082C083EA12458E04
:1043B30012444FD2E0023FD3C082C0831244496407
:1043C300017011124454400C8A828B83A3E0F912CA
:1043D300162C806FEA241012444CA2E650128A82F3
:1043E3008B83A3E0F990062E12477A120529805396
:1043F3001244496401700D12445450088A828B831D
:10440300743080368A828B83A3E0641B8A828B8319
:10441300700474228024A3E0700D124449F8748A56
:104423001251683430800B124449F874AB1251684E
:104433003430F583E4938A828B83F090067CE0F931
:10444300121E9602494BEA240DF582E43BF583E004
:1044530022EA1245B83BF583E0A2E32274F7120384
:104463009EE9FE1252467003024585EE6011741BED
:104473006E7013E0C812458864057003024550123C
:1044830060ACE402455474E96E70621245A4700B8B
:1044930012288CE960051245BE606279EE121A4C4F
:1044A3009006261245A1900626603B1245C1900650
:1044B30026700B1245A114F0121C260245851245E5
:1044C300ACC2E71246CC1245886403700C125CC27E
:1044D30012458E1242F6D2E2F079ED121A4C1245D1
:1044E3009412052980751260AF74E9806474E16EDB
:1044F300703E12288CE960551245BE7050900B8CAB
:10450300E0C0E0125CC22412F582E438F583D0E007
:10451300F0900B7BE0C0E09006261242C21242C22A
:10452300D0E0F0900B7BE004F07901121C0E805276
:10453300741C6E70189006261254B69006361247F5
:104543007A120529900626E4F0A3F080351260ACB8
:10455300EEF09006261254B6121554125CC2125C89
:1045630094E054806010900B92E0F9121B12900BB0
:1045730091E0F9121B06900626E4F0A3F0791012DD
:104583001626024C05240D1242F3222411F582E46F
:10459300229006261254BA90062A1260B622E0F838
:1045A300A3E0C824121242F322E0F8A3E0C81245A4
:1045B300B81242F6222410F582E422900626125CF9
:1045C300C9125C98E054042274F412039E750A0025
:1045D300750B00A2AFE433FFC2AF12524660030271
:1045E3004688124777120529E94410F890061D8082
:1045F3000985080A85090B1246A31246B8700302FF
:10460300468812380D586870E8780A12090DAC080C
:10461300AD097A1D7B06121EC074021208CF9006E4
:1046230026E508F0A3E5091246CC1246B0405D909A
:104633000624E014F0EFA2E092AF900626E0240EE9
:10464300F8A3E03400F9880889098882F5831254B5
:10465300B69006261246C6F9121518E9900621F0FF
:104663001246D4E054809006266026125CC52413BB
:104673001242F3F9121B12125CC224141242F3F910
:10468300121B068018EFA2E092AF801190062380E0
:10469300A11245ACA2E1B3E433F9121C0E0231506E
:1046A300E50824FBF582E50934FFF5832224111282
:1046B30042F3A2E722126733E508450922851882EF
:1046C30085198312350FA3E022F0900626125CC9E8
:1046D30022A3E4F08508828509832274F712039EDE
:1046E300EAFEEBFF121662EE24101247FFA2E3402C
:1046F3000C1247FC640170059080FB80039080FCE2
:10470300E0F9EEFCEFFD7A1D7B06121EC6E960465A
:10471300EEFAEFFB90063012477A120529EE240ECB
:104723001247FF54047020A8A8C2AF900624E004E7
:104733001254ACFAE8A2E792AF124769A3E054011E
:104743007021121560801CEEFAEFFB9006281247C9
:104753007A120529800D8E828F83A374F1124B691F
:10476300121554024C0512476D22EE240EF582E415
:104773003FF583229006321260B622C082C08312B4
:10478300156002494B74F712039EEAFEEBFF7900B2
:10479300900681E05402700CEE24301247FF54045B
:1047A300600279E8900681E05460700CEE243012C8
:1047B30047FF5402600279E88E828F83A3A3A3A3E9
:1047C300E0F8908101E0C398500279E8EE242E12BC
:1047D30047FF700CEE242B1247FF700479F5800B12
:1047E300E97005121542E9F9E96007EEFAEFFB12E9
:1047F300162C024C0534FFF509EE240DF582E43F37
:10480300F583E022C082C0838A828B83740DF01209
:10481300288002494BC082C0838A828B83E4F0A341
:10482300F0EA243012444C54049080FB7012E0F8F8
:10483300900624E0C398401279F112162C02494BDA
:10484300E0F8900623E0C39850EE90067CE0F9125E
:104853001E9680E974F612039EE9FE244CFAE434B2
:1048630000FB121E8AEA4B6012EE8A828B83A3A39B
:10487300A3A3F0EA244C12516D80047A007B00025A
:104883005FF6C082C08390063874AEF0A37415F04F
:10489300A374DEF0A37415F0A374B4F0A37415F03D
:1048A300A374BAF0A37415F0A374D8F0A37415F02D
:1048B300A374CCF0A37415F0A374C6F0A37415F01D
:1048C300A374E4F0A37415F0A374EAF0A37415F0D1
:1048D300A374F0F0A37415F0A374FCF0A37415F0A3
:1048E300A374C0F0A37415F0A374A8F0A37415F017
:1048F300A374A2F0A37415F090065474D2F0A374B9
:1049030015F0A374F6F0A37415F0A3742EF0A3743A
:1049130017F0A37402F0A37416F0A37408F0A37441
:1049230016F0900678E4F090067BF0900664124946
:10493300427402F090066D1249427401023FD3742F
:1049430026F0A37416F0A322D083D0820208B77492
:10495300F512039E74F112099985188285198374DF
:1049630002F07401120BC3E9F060047AFF7BFF7459
:1049730002120BC31254C6750870750906750A0036
:1049830078081209097C0B7D007407120BC3AA82F5
:10499300AB83121E6074031208CFAA18AB19122836
:1049A30080740F02669374F712039E74FD120999C3
:1049B300851882851983740AF07401120BC3E9F018
:1049C3007402120BC3EA1249DC122880023B4F85A2
:1049D3001882851983EAF0A3EBF0AA18AB192274A5
:1049E300F612039E74F7120999EAFEEBFF124A329C
:1049F3001232DF7402124B5AAA18AB19122034EE8A
:104A0300242E1232AD2430125A9312090D7402125D
:104A1300096379831A1AEFFB12169274021208CFF4
:104A2300E9F5087007EEFAEFFB121566025FEF1265
:104A3300476D74012274F012039E12657C120B54AD
:104A43007808790C1202AF78081209057A677B0699
:104A530002353274F412039E74C6120999900B6ADC
:104A6300E0640F6010851882851983742E1249DC67
:104A730012164480277A5E7B0612177612315E1275
:104A8300025688088909E4F50AF50B780812090526
:104A93007A5E7B0612176A74041208CF743A0231E5
:104AA3004D74F512039EEAFEEBFF8E828F83A3E023
:104AB300F86003024B43EE242D1247FF64026007A4
:104AC300E06403600278E8EE2423F582E43FF58393
:104AD300123157400478E8806AE87064EE2423FAC0
:104AE300E43FFB79E1121AD6EE242EFAE43FFB7978
:104AF30050121AD6EE242D1247FF6402700E125C78
:104B030082125CB8900B791251778012900B7974F2
:104B1300FEF0A304124B5A7A707B0B122040EE2452
:104B230018123F701209097C0B7D007A707B061204
:104B33001E6074031208CFEEFAEFFB12159CE9F81E
:104B4300E86011E88E828F83A3125EE47417124B20
:104B530069121644026696F0EE2425FCE43FFD221A
:104B63008E828F837429F0EEFAEFFB2274F6120320
:104B73009E74F712099990067BE0703B7401F0F97B
:104B8300121BD2AA18AB1912167475087075090690
:104B9300780812090D750801750900780812090DC6
:104BA300900B7F12071174061209637A03790512B9
:104BB300169874061208CF025FF174F712039EEA87
:104BC300FEEBFF7901121BD88E828F83E064207085
:104BD30004A374EBF090067BE0A2E25003C2E2F080
:104BE300E0A2E15008124E07121596800C8E828FB8
:104BF30083742A124B691216448007EEFAEFFB12F4
:104C030016E07F0102060F74F412039E74FE12096C
:104C130099EAFEEBFF7901121BD87A5E7B06121725
:104C2300767A677B06121776124F5185188285199B
:104C330083124F85E0F50B700FAA18AB1979531245
:104C43001AD6126723121AD6123F6D1209097C0B6A
:104C53007D007A707B06121E6074031208CF8518DC
:104C6300828519831254B6A90B12159090067BE026
:104C7300A2E1500C7A008E828F83A3E0F91215967D
:104C830090067BE4F0740202314D74F712039EEA3E
:104C9300FEEBFF8E828F83A374EBF090067BE0A282
:104CA300E150077A0079EB121596EEFAEFFB121535
:104CB300CC024C0574F712039EEAFEEBFF79011256
:104CC3001BD87A5E7B061217767A677B06121776F5
:104CD300900678E4F090067BF07AFF7BFF8E828F5C
:104CE30083A3E0F9121590024C0574F712039EEAB0
:104CF300FEEBFF1215C6024BFE74F712039EEAFE8B
:104D0300EBFF7901121BD88E828F83A3A3A3A3E0A9
:104D130060047400800274EB124D4E5003C2E2F043
:104D2300E0A2E15008124E501215968014A2E050F2
:104D3300108E828F83742AF0A374EB124B691216C0
:104D430044EEFAEFFB121578024C058E828F83A393
:104D5300F090067BE0A2E22274F612039EEAFEEBD9
:104D6300FF90067BE0D2E1F07901121BD28E828F95
:104D730083A3E0703C12167AE9FAEE240DF508E4F9
:104D83003FF509780812090D7508017509007808BF
:104D930012090D124DC5120711EE2402FCE43FFD6A
:104DA300790512169874061208CFE98E828F83A3B1
:104DB300F08E828F83A3E060067A00F912159602C3
:104DC3005FF6124DC922EE240BF582E43FF58322F0
:104DD30074F712039EEAFEEBFF7901121BD88E8251
:104DE3008F83E064207004A374EBF090067BE0A251
:104DF300E25003C2E2F0E0A2E15006124E071215A0
:104E030096024C05C2E1F07A008E828F83A3E0F90B
:104E13002274F712039EEAFEEBFF7901121BD87A84
:104E23005E7B061217768E828F83A3A3A3A3E06013
:104E3300047400800274EB124D4E5003C2E2F0E0A2
:104E4300A2E15006124E50121596024D44C2E112D1
:104E53003CB8A3E0A2E4E433FA8E828F83A3E0F9A3
:104E63002274F712039EEAFEEBFF7901121BD88E20
:104E7300828F83A374EB124D535003C2E2F0E0A27E
:104E8300E15006124E07121596024C0574F71203F1
:104E93009EEAFEEBFF7A5E7B06121776EEFAEFFBD5
:104EA3001215F0024BFE74F712039EEAFEEBFF7A33
:104EB3005E7B06121776EEFAEFFB1215F0024C0535
:104EC30074F712039E74EF120999EAFEEBFF125C6A
:104ED3008C7A707B0B12202EE9606285188285190B
:104EE300837409F07401120BC374EFF0124F51F87D
:104EF3007402120BC3E8124F85A3A3E0C0E074044D
:104F0300120BC3D0E0124F72640870158E828F8328
:104F1300A3A3124F45E0C0E07405120BC3D0E08099
:104F2300067405120BC3E4125CEB7406120BC3AADE
:104F330082AB831216AAAA18AB1912288074110225
:104F43003B51125CC92407F582E438F58322124FE2
:104F530067FB8A828B83125CBC88828983E0FCA313
:104F6300E0F9EC22EE2402F8E43FF9E8FAE9221230
:104F73004F7622124F7BE022F08E828F83A3A3A36E
:104F8300A322F0A3E9125CDA124F8F22E0F8A312F6
:104F930060BDA3A322C082C0831216EC02494BC09A
:104FA30082C0839006987438F0A37406F0A37454F7
:104FB300F0A37406F0901DE774DDF0A3742DF0A345
:104FC300743FF0A3742EF0900684748AF0A37415D2
:104FD300F0900681E04401023FD3C082C083EAFC23
:104FE300EBFD790212165002494BC082C083790649
:104FF30002618774F612039E74FE12099990067D6E
:1050030012524960077A7D7B06121668900683E484
:10501300F0901AF812524960268007AA18AB1912A9
:10502300166890067CE0F9121EA28A088B09A8086C
:10503300A909851882851983125177E84970DC74B0
:1050430002025FF374F712039EE9FA7B0090067C79
:10505300E0F9121ECC024C0574F712039E74F01291
:105063000999EAFCEBFDE9FE8C828D83E0F874A0DC
:105073001251683430F583E493C0E07401120BC31A
:10508300D0E0F0640B700DEE8C828D83A3F01216CA
:10509300CE02515BE0700302515B640C600302516A
:1050A3004C741A6E700B7404120BC3E4F0A3025118
:1050B3004B7404120BC3ECF0A3EDF0EC242F12514C
:1050C30060C0E07403120BC3D0E012628F120B7C3A
:1050D3007406120BC3120B708C828D83125CAF7437
:1050E3000A120BC3125177EC240E12516054106054
:1050F30009851882851983E48013EC241212516008
:10510300F8900B8CE0C398851882851983F0E0C072
:10511300E0740C120BC3D0E0F0EC2415125160C004
:10512300E0740D120BC3D0E0F0EC2416125160C0F2
:10513300E0740E120BC3D0E0F0EC2417125160C0E0
:10514300E0740F120BC3D0E0F07402120BC3EEF045
:10515300740112095B1228807410023B51F582E43A
:105163003DF583E02228F582E422F8E43BF98A82C4
:105173008B83A3A3E8F0A3E9F022C082C083900647
:1051830083E0700479018002790002494BC082C038
:1051930083900683E06004640270047901800279DD
:1051A3000002494BC082C083900683E0640370040D
:1051B30079018002790002494B74F712039E90062D
:1051C30083E0125233126B5A8A828B83E0C2E7F078
:1051D30025E0F8EC1251683DF583A3E493FE1252E7
:1051E30033F5831252496005EE900683F08A828B71
:1051F30083E012523FEC28F582ED39F583E493FC0A
:10520300C4540F25E0F874921251683406F58312E2
:10521300524970051216BC8014EC540F25E0FCE8CB
:105223002CF582E439F58312477A120529024C05DD
:1052330012523F74E528F582741D392225E0F8E403
:1052430033F922900626125CBCE8492274F112035A
:105253009E74FE120999890AEAFEEBFF12534BFA78
:105263007B00121E8A8A088B09EA450960388A8204
:105273008B83E50AF0A3E4F08E0C8F0DF50E780C0A
:10528300120909A80A125358EA2402FAE43509FB61
:10529300121E6074031208CFAA08AB0990067CE0C3
:1052A300F9121E968012851882851983E50AF07912
:1052B3001AAA18AB1912162C74021208CF0233BDA6
:1052C30074F212039E74FE120999890B8A088B09E2
:1052D30012534BF50AFA7B00121E8A8A0C8B0DAE11
:1052E3000CAF0DEE4F604A8E828F83E50BF0A3E483
:1052F300F0A80AEE28F8E43FF98E828F83125175E5
:105303008E828F83A3A3A3A3E4F0F50A780812097E
:1053130009A80B1253581236D0121E6074031208D8
:10532300CFEEFAEFFB90067CE0F9121E967900802F
:1053330014851882851983E50BF0791AAA18AB191D
:1053430012162C791A023BE374C129F582E4343036
:10535300F583E49322749528F582E43430F583E4ED
:1053630093FC7D0022C082C083E990067C023FD378
:1053730074F612039E74FE120999EAFEEBFFEE54D3
:105383002070378040A8A8C2AF900625E0141254BD
:10539300ACF508E8A2E792AF8A828B831254A390FC
:1053A300067F1254C6121644851882851983E06459
:1053B3001560077A7F7B061216687A1F7B06121E1A
:1053C300B4EA4B70C0EF54807012801C90067F12B9
:1053D30054C61216447A7F7B0612166890067CE048
:1053E300F9121EA2EA4B70E4EE5410600E85188287
:1053F300851983742D1249DC121644EEA2E0500E77
:1054030085188285198374241249DC121644EE54DC
:1054130002600E85188285198374251249DC1216E1
:1054230044EE5404600E851882851983742612494C
:10543300DC121644EE5408600E85188285198374B5
:10544300281249DC121644EE544060107401120B0A
:10545300C31264F0742C1249DC121644EE548060BB
:10546300107401120BC31264F0742F1249DC12166C
:105473004490067D1252496020A8A8C2AF90067DD1
:105483001254B690067DE4F0A31254CC1254C51204
:1054930016447A7F7B061216687A007B000250421C
:1054A300E0851882851983F022F0E8A2E7E433222D
:1054B3009006041254BA22E0FAA3E0FB22A3A3A3AA
:1054C300A3A3A3EAF0A3EBF0221254ACFEE8A2E7F5
:1054D30092AF22C082C08390067F125CB8EA6870E4
:1054E30002EB69700790067FE4F0A3F002494B7466
:1054F300F712039EEAFEEBFFEE4F700312189CA215
:10550300AFE433F508C2AF8E828F8312524960280D
:10551300E824FBFAE934FFFB90067F126B5CE86C2E
:105523007002E96D700790067FE4F0A3F08E828F1E
:1055330083E4F0A3F0121F320239A2C082C0839029
:1055430006A674B0F0A37416F0A374C2F0A3741685
:10555300F0A374C8F0A37416F0A37472F0A37415C7
:10556300F0A374CEF0A37416F0A3746CF0A37415B7
:10557300F0A37478F0A37415F09006B474FEF0A34E
:105583007416F0A374D4F0A37416F0A374DAF0A322
:105593007416F0A374E6F0A37416F0A374E0F0A3FA
:1055A3007416F09006A5023FD2C082C083900B7997
:1055B300E064FE7003A3E0F470097C707D0B12209D
:1055C3003480158A828B83A3A3A3A3A3A3A3A37469
:1055D30002F012572E12517702494BC082C08390BA
:1055E3000B83C3E094FEA3E094FF4004790380029D
:1055F300790202494BC082C0831257398C828D8352
:105603001256EE687039740268701C8A828B83129A
:105613005647E06870298A828B83A3125647A3E01A
:1056230068701C7901801A7403687013EC2405FCFC
:1056330050010DEA2405FA50010B12203A80027939
:105643000002494BA3A3A3A3A3E0F88C828D83A3F9
:10565300A3A3A3A32274F612039E7E00740A120B63
:10566300C3E01256E2FF8A828B83A3A3A3A3A3A35F
:10567300A3A3E06F706474026F704E8A828B83C041
:1056830082C08388828983A3A3A3A3A3E0F50888A8
:10569300828983A3A3A3A3A3A3E0FBAA08D083D0F7
:1056A30082E06A7003A3E06B703088828983A3A3CE
:1056B300A3E0FA88828983A3A3A3A3E0F9EA6C7029
:1056C30002E96D70157E01801174036F700CE8247C
:1056D30005FCE439FD12203AE9FEEEF9025FF6F823
:1056E300A3E0F9888289831256EE22A3E0131354B0
:1056F3003F540322C082C0838A828B83A3A3A3A3C4
:10570300A3A3A3A3E06402701412572EE0687003EE
:10571300A3E06970047901800F7900800BEAFCEB48
:10572300FD7A707B0B12202E02494B900B79125C91
:10573300BC8A828B83228A828B831256EEF8227470
:10574300EC12039EEAFEEBFF8C128D13750A008C9C
:10575300828D83A3A3A3A3A3A3A3A3E0F510E9A22C
:10576300E75008750CFF750DFF8006900B7F1259EB
:105773007EE9C2E7F511EE240E1247FF54206007BD
:1057830012595F7408800412595FE4125986540455
:105793006007125967748080051259677410125993
:1057A3008654106006125937E4800B900B8CE0C0CE
:1057B300E0125937D0E0125986A2E05003750A204F
:1057C300540860067410450AF50A8E828F83A3A3DA
:1057D300E024FFF508A3E01247F8C39402E0400B6E
:1057E300640B6005E0141236E07403450AF50A758C
:1057F3000B00900B9FE0640170118E828F83A3A333
:10580300A3A3E0C394674003750B1085110E750FB6
:1058130000740E780E120A9CE50F450BF50B7414F9
:10582300120BC3E0F50EA3E0F50F74026511700EC1
:10583300900B841236DF900B831259758013740317
:10584300651170121259417C937D0BAA08FB12203B
:105853004012594E8004E5116028E5106014E50EEE
:10586300650C7004E50F650D70087440450AF50A70
:105873008010850882850983E50D12598CE50C1289
:1058830036E685100C750D00740A780C120A9CE537
:105893000D450BF50B740265107015851282851387
:1058A30083A31236DF851282851383125975801301
:1058B300740365107012125941AC12AD13AA08FBA0
:1058C30012204012594E8004E5106010850882852D
:1058D3000983E50F12598CE50E1236E6A808A909CB
:1058E300E824FFF508E91247F87005900B6F800371
:1058F300900B7BE0FA04F0EA888289831246D6E5AE
:105903000B12598CE50AF0EE2404F8E43FF9123344
:10591300CCAC088A828B83E0F50A88828983E025F0
:105923000AC39C125CD6ECF0A3E509125E52E4F0C4
:10593300F9023131EE2412F582E43FF58322E508C2
:1059430024F9F508E50934FFF5092212595222E535
:105953000824FFF508E50934FFF50922EE1245B8DE
:105963003FF5832212596B22EE2411F582E43FF5B1
:105973008322E0850882850983F022E0F50CA3E009
:10598300F50D22F012476DE0221236EA850882F502
:10599300832274EE12039E890A8A0B8C108D117573
:1059A3000C1A7416120BC312672FAA08FB121512D6
:1059B3008A0E8B0FAE0EAF0FEE4F60607414120B96
:1059C300C3125A26E8F0A3E91232E2E50AF0850889
:1059D3000C85090D750E00780C1209091236CC12CC
:1059E3001E6074031208CF7412120BC3120711AC9A
:1059F30010AD11A90BEEFAEFFB1216927402120806
:105A0300CFE9F50C7016E50A24F960031470061249
:105A13003753D2E5F0EEFAEFFB121566A90C7F0AB5
:105A230002060F1260CB12476E2274F612039E74A5
:105A3300F7120999EAFEEBFF7801EE242F1247FFD4
:105A430060027805124769E81232DF7404125A863D
:105A5300122034EE242C1232AD242E125A93120942
:105A63000D740212096379031A1AEFFB121692746A
:105A7300021208CFE9F5087007EEFAEFFB1215667C
:105A8300025FEFF0EE2423FCE43FFDAA18AB1922DA
:105A9300F582E43FF5831233F7124F7604F078086A
:105AA3002274F212039E8A088B09ECFEEDFF8A82B0
:105AB3008B837405F0EE24321247FF8A828B83A313
:105AC300A3F0EA2403F50AE43509F50B850A82F508
:105AD3008312597E125C82120B7CE50C12458E35C3
:105AE3000DF583120B70125C8CAA0CAB0D122034D3
:105AF300850A82850B831260C3FAA3E0FB8882893F
:105B030083A3A3A31254C0EE242F1247FFC0E012B5
:105B13005CA1D0E0125CE02415F582E438F583E45F
:105B2300125CE0125C94E4125CEB850A82850B83C1
:105B3300E02416FAA3E03400FB1216AA8E828F83A8
:105B4300A3A3A3A3A3A3A3E0C0E0850A82850B8339
:105B5300125CC5240DF582E438F583D0E0125CCFE6
:105B6300FAA3E0FB850A82850B83125CB8E8240B59
:105B7300FCE439FD8A828B83E08C828D83F0A3E47D
:105B8300125CF8E0F50B8C828D83A3E0450B125C6D
:105B9300D6A3E0FCA30A0AAB83A2E7E433C0E0E8A0
:105BA300240FF582E439F583D0E0F074075C6004D8
:105BB30078018002780075F00374075CA428F8EA82
:105BC30028FAE43BFBE5082405F8E43509F98A8261
:105BD3008B831233F7125CF885088285098312548C
:105BE300C088828983E0F50A540725E0FCE50AC4EE
:105BF300540F5407F50A750B007403780A120A9CB4
:105C0300EC250AF8EA28F8E43BF98508828509833C
:105C1300A3A3A3A3A3A3A3A3A3E8F0A3E9124F728F
:105C2300FA8E828F83A3A3E02AFAA3E03400FBC396
:105C3300EA98EB9940308E828F83A3A3E0F885081E
:105C430082850983A3A3A3A3A3A3A3A3A3E0FA8E9B
:105C5300828F83A3A3A3A3E0C39A2885088285091F
:105C630083A3A3A38010850882850983A3A3A3A389
:105C7300A3A3A31246D4A3A3A3A3A3F0023BE8EEDA
:105C83002425F582E43FF58322EE2413FCE43FFD53
:105C930022125C9822240EF582E438F58322125CEA
:105CA300A522E82410F582E439F58322A3A3A3A354
:105CB300A3A3A3A3A3125CBC22E0F8A3E0F9229060
:105CC3000626125CC922E0F8A3E0C822125EE4A310
:105CD300A3E022125CDA22F08A828B8322F0850A07
:105CE30082850B83125CC922F0125CF022EE240839
:105CF300FCE43FFD22125CDAA3AA82AB832274F593
:105D030012039E8C088D09750A0078081209097C14
:105D13000B7D0002668E0208B7C082C08379181219
:105D2300162C02494BC082C0838A828B83E0C394C2
:105D33000B50031216B602494BC082C083791980F7
:105D4300DE74F712039EEAFEEBFF90067D125249C2
:105D5300601090067D1254B61216C27A7D7B06122D
:105D63001668EEFAEFFB12166290067DEEF0A3EFD3
:105D73008002F0A3F0024C0574F712039E74DE1246
:105D83000999EAFEEBFF8E828F83E024FD601124E4
:105D9300FE601524ED600924FA600D14600A803D4D
:105DA3007416120BC3E480077416120BC37401F04C
:105DB300124390740B120BC3AA82AB83122040745C
:105DC30013120BC3125E57120BC3125177740A12CC
:105DD3000BC3125E63120BC3125177804274161207
:105DE3000BC37402F0125C8C740B120BC3AA82AB4C
:105DF300831220407413120BC3125E57120BC3128B
:105E03005177740A120BC3125E63120BC31232C1B1
:105E1300125CF17417120BC3AA82AB831216AA8504
:105E23001882851983740B125E52E0C0E07401126C
:105E33000BC3D0E0125CEB7417120BC3AA82AB83C3
:105E43001216AAAA18AB191228807422023B511207
:105E53005EE4A3227403F0900B83125CBC740222F1
:105E63007402F0900B7F125CBC74142274F712035B
:105E73009EEAFEEBFF8E828F83A3E0F5087036EE79
:105E8300242C125EEA7003A3E06960037508E8EE50
:105E93002423FAE43FFB12168CE96032EE242FF53B
:105EA30082E43FF583E4F0E508700AEEFAEFFB12B3
:105EB300169EE9F508E50860128E828F83A3E50834
:105EC300125EE47419124B69121644024C05EE2457
:105ED3002F1247FF60D19006A4E070CB7508E880CD
:105EE300D8F08E828F8322F582E43FF583125CBC67
:105EF300900B7FE06822C082C08374F11209997409
:105F030002120BC37404125CD6A3E0C0E074031244
:105F13000BC3D0E0F0EA242CF582E43BF583125C5A
:105F2300B8740D120BC3125177EA2423FCE43BFD32
:105F33007404120BC3AA82AB831220347404120BB1
:105F4300C3AA82AB8312168CE9600E125F69121A20
:105F5300D6900B7974FFF0A3F0740212095B122838
:105F630080740F02405885188285198374FFF0A34B
:105F7300F0AA18AB1979532274F612039E74E8122F
:105F830009998A088B097402120BC37403F0EA247B
:105F930013FEE43509FFEEFCEFFD7404120BC3AAF4
:105FA30082AB83122040123822C0E0740C120BC360
:105FB300D0E0F0E5082408FCE43509FD740D120B6C
:105FC300C3AA82AB831216AAEEFAEFFB12168CE970
:105FD300600E125F69121AD6900B7974FFF0A3F06A
:105FE300740212095B12288074188004A9087409CA
:105FF3001208CF7F0202060F74F612039E74D412A6
:106003000999EAFEEBFF8E828F83A3A31260AFE0B0
:10601300A2E65017900B7F1260C3687003A3E06978
:1060230070099006A5E060411216EC740B12095337
:106033007403120BC31266801216A4851882851985
:1060430083742B1249DC121644900B64E0600874CD
:1060530008120BC3E0600E8518828519837405123C
:1060630049DC122880742C8087900B88E060BC1276
:106073003F6512168CE970B3EE2408F508E43FF58A
:1060830009780812090D75080175090078081209C5
:106093000D900B7F1207117C707D0B7A037906122A
:1060A300169874061208CF80BC9006261260B6A319
:1060B30022A3A31260BA22E0F8A3E0F58388822228
:1060C3001260CB123B46E022E0F8A3E0F9EE22C0D7
:1060D30082C08374EF120999851882851983740924
:1060E300F07401120BC374EE1249DC1228800240D3
:1060F3005674F712039EA2AFE433FFC2AFE9600305
:10610300121AC4121A46900B92E0F9121B12900B4A
:1061130091E0F9121B069006A5E0F9121AEE900B16
:106123007F1254B6121AF4900B831254B6121AFA51
:106133007A937B0B121B007E001261781252496026
:106143000912617812477A1205290EEEC3940740AB
:10615300E81217461216209006BEE4F012150C1230
:10616300166E7A827B0B7952121AD6EFA2E092AFA7
:106173007900024C05EE12523F748428F5827406AE
:1061830039F5832212164A02494BC082C083900616
:10619300BF7416F0A37417F0A37434F0A37417F04C
:1061A300A3743AF0A37417F0A3741CF0A37417F04C
:1061B300A37428F0A37417F0A37422F0A37417F048
:1061C30090069274A6F0A37406F0A374B4F0A374BB
:1061D30006F0A374BFF0A37406F0900681E4F0A365
:1061E300F0121A4002494B0208B774F712039EE9F2
:1061F300FE9006BEE06E6016E07017121638E96076
:1062030011EEF9121C02E96009EE9006BEF0790066
:10621300800279E2024C05C082C0839006BEE06032
:1062230008121BFC9006BEE4F002494B74F71203FC
:106233009EEAFEEBFF8E828F83740712628AE08EE2
:10624300828F83A3A312628AA3A3E08E828F83A388
:10625300A3A3126298A3A3120B7C8E828F83A3A3A2
:10626300A3A3120B708E828F83A3A3A3A3A3A3A3C1
:10627300A3E4F0EC2418125160F8126937A3A3A326
:10628300E8F0A3E9025D7712628FA322126298A35A
:10629300A3A3A3A322F08C828D832274F412039E02
:1062A300EAFEEBFF9006CCE4125E52A3A3A3A3A3E2
:1062B300E0C3940640069006CC74E8F08E828F8388
:1062C300A3A3A3A3A3A3A3E0C3940F40158E828F1C
:1062D30083A3A3A3A3A3A3E0640360159006CC74D4
:1062E300E8F08E828F83A3A3A3A3A3A3E064037028
:1062F3000E900681E0A2E040069006CC74E8F0EE32
:10630300FCEFFD7ACB7B061217108E828F83A3A33B
:106313007808120B54740A780812093A9006DF7849
:1063230008120B368E828F83A3A3A3A3A3A3A3E098
:106333009006E31263D89006E41263DD9006E5123B
:1063430063BE9006E6F0EE240C1247FF9006E7F0DA
:10635300A3740AF0900B92E09006E9F09006DC1229
:10636300494274041263C41209097C0B7D007AEA62
:106373007B06121E6074031208CF9006CCE0702ACD
:106383008E828F83A3E070229006CDE06006900694
:10639300CC74EAF09006CDE0F9121B1E8E828F8337
:1063A3007426F07904121BCC80078E828F837429A4
:1063B300F0EEFAEFFB121644023150F0124DC9E031
:1063C30022F0EE240D1263CC22F508E43FF50975A3
:1063D3000A007808221263E3E0221263E3A3E022B7
:1063E300123CBCA3A3A32274F412039E74F71209F4
:1063F30099EAFEEBFF9006CDE070319006E8E06489
:106403000A6029121B30E9C0E09006E8E0F8900624
:10641300D4E028F8A3E03400F9E824F5F582E93460
:10642300FFF583D0E0F09006D3E004F09006DF7828
:1064330008120B547401780812093A9006DF7808A1
:10644300120B369006E8E004F0E508A2E04006E00F
:10645300C3941E40D7E0641E70030264E77AE87BAE
:106463000679E1121AD67408120BC374021264F18E
:1064730074FFF0A3F09006CDE0600464027009EEAF
:10648300FAEFFB1217228062E06401700679087A42
:1064930080800479077A837508EA750906780812FB
:1064A300090DE4F508F509780812090D7508FF755B
:1064B30009FF780812090D740612096312169874FD
:1064C300061208CFE9F874DB68601474E568600F9E
:1064D30074F368600A74DF68600574E868700BE839
:1064E3009006CCF0124B6312164402314BE4126453
:1064F300F522F08518828519832274F012039E75A4
:106503000801750900750A00750B009006E8E0782C
:10651300081208927808120AF69006CF7808120A31
:10652300769006CDE06403700F12657C120B5478ED
:1065330008790C1202AF8035750801750900750AD8
:1065430000750B009006E3E07808120892908176BC
:106553007808120A3D908182780C120B54780879DE
:106563000C1202AF9006CDE07003121B2A780812BA
:1065730009057AD67B06023532900B8D123136909F
:106583008182780C2274F512039E74D4120999EA5D
:10659300FEEBFF9006CDE06402600DE0640160084D
:1065A300E0640560030266769006CCE4F0740B1297
:1065B30009537403120BC31266801216A49006E4E7
:1065C300E0F89006D3E0C3985077A312672F9006A4
:1065D300D3E0F50A8032850882850983125CAF74A3
:1065E30014120BC3E0687003A3E069700F740B12FD
:1065F3000963AA08AB0912202EE97045150AE508BC
:106603002421F50850020509E50A70CA740B120922
:106613005388088909750A0078081209097C217DC5
:10662300009006D3E08CF0A4F8A9F0A3E028FAA325
:10663300E039FB121E6074031208CF9006D3E00406
:10664300F0900B64E0600E7408120BC3E0700690C8
:1066530006E4E07007AA18AB191228809006E4E05C
:1066630060179006D3E0F89006E4E068700B124BD5
:1066730063800312673B121644742C8013E8F0A363
:10668300E9F0EEFCEFFDAA18AB1922121E607403A9
:106693001208CF7F0302060F74F612039E74FE12D4
:1066A3000999EAFEEBFFEE241B1247FF64037067B0
:1066B300EE24241247FF6403705D126723121AD677
:1066C3008E828F83A3A312672F850882F5831267B7
:1066D3004750020509AA18AB197950121AD6850832
:1066E3008285098312674750020509AA18AB1979F5
:1066F3004B121AD6AA08AB0979E1121AD685088279
:10670300850983A3126752125F73121AD69006CCBF
:10671300E4F0124B63800312673B121644025042AB
:10672300EE2413FAE43FFB794A22F58312673322FE
:10673300E0F508A3E0F509229006CC74E8125EE4C4
:106743007429F022126752F0E5082402F50822E0CA
:10675300FAA3E0F9EA851882851983F0A3E922C038
:1067630082C0837AD67B06121776121B2479041211
:106773001BD89006CDE0640370069006CCE0600958
:106783007AE97B0679E1121AD67ACB7B06024812A4
:10679300C082C08374F5120999EAFCEBFDAA18AB19
:1067A300191217107401120BC374FC1249DC12285E
:1067B30080740B024058C082C083790702618774DA
:1067C300F712039E9006F5E4F0A3F09006F7F0A30A
:1067D300F0901DEF1267E6901DF31267E69006F93D
:1067E300025D75F0A3F0A374FFF0A3E4F02274F448
:1067F30012039E9006F9E4F0A3F09006F5125249B5
:106803006032901DEF7808120B541268981209C475
:1068130050221219C88A088B098C0A8D0B126898AA
:106823001209C45006126898120B369006F51268C6
:10683300911251779006F71252499006F96023128C
:10684300524960131242C57808120B549006F7128E
:10685300689B1209C450109006F712689112517781
:1068630080051252496021901DEF7808120B549055
:1068730006F912689B1209C4500E9006F91242C21F
:10688300120BAC1219DA80031219E0023150125CB8
:10689300BC9006F9229006F5124F8F78082274F007
:1068A30012039EA2AFE433F508C2AF9006F9125269
:1068B30049607412694B120B54901DEF780C120946
:1068C300C4500B12189C9006F912524960591219C0
:1068D300C88A0C8B0D8C0E8D0F12694512087350EC
:1068E30046908142780C120B541269451209C45028
:1068F3000312189C9006F9E0FEA3E0FFEEFAEFFB0B
:106903001217768E828F83A3A3A3A3A3A3A31269D3
:106913003712692FE508A2E092AF120529A2AFE46E
:1069230033F508C2AF809FE508026AD31254BA8ACE
:10693300828B8322A3E0F98E828F83A3A3A3A3A3D5
:10694300A3229006F9E0F8A3124F92780C2274F078
:1069530012039E8A088B098C0A8D0B7410120BC3C9
:10696300801C908142780C120B548E828F83A3A3D8
:10697300780C1209C4500312189C8E828F83123B29
:10698300DB60338E828F83A3A37808120AC2126955
:10699300BC7002EF6970CB908142780C120B548E5D
:1069A300828F83A3A3780C1209C450B68E828F837F
:1069B300A312312A80C402353A9006F91260CB68DB
:1069C3002274F012039EA2AFE433FEC2AF9006F727
:1069D30012672F9006F5120711901DEF780C120B1A
:1069E30054780C120AD5AA0CAB0DAC0EAD0F1217CE
:1069F3005874021208CF8039901DEF780C120B5493
:106A0300850882850983A3A3780C1209C4401590D5
:106A13001DEF780C120B54850882850983A3A37894
:106A23000C120A16850882850983125CB8880889C6
:106A330009E508450970C1901DF37808120B5490BD
:106A43001DEF78081209AF6015901DF3120B7C90AF
:106A53001DEF120B70901DEF120BAC1219C212171F
:106A63004CEE806C74F012039EEAFEEBFFA2AFE4DF
:106A730033F50CC2AFECFAEDFB8C828D838008AA50
:106A83000EAB0F8A828B83E0F50EA3E0F50FE50EC4
:106A9300450F601A850E82850F83A3A37808120B16
:106AA300548E828F83A3A378081209C450D18A829B
:106AB3008B83EEF0A3EF125EE4E50EF0A3E50F1275
:106AC30062981269BF7002EF69700312174CE50CEC
:106AD300A2E092AF02353A74F412039EEAFEEBFF92
:106AE300740C120BC3C082C0831219C88A088B09A5
:106AF3008C0A8D0BD083D0827808120A3D8E828F48
:106B030083A3A37808120B367CF57D06EEFAEFFB20
:106B130012176402315074F712039EECF8EDF98CEE
:106B2300828D838004A882A983126B5C8C828D83FF
:106B3300E58245836014EA65827003EB658370E543
:106B4300126B521254C6790180027900024C05126D
:106B530054BA8882898322F583E0FCA3E0FD227482
:106B6300F712039EEAFEEBFFA2AFE433F508C2AFD0
:106B73007CF57D06121770E9700B7CF77D06EEFA43
:106B8300EFFB1217701269BC7002EF6970031217E2
:106B93004C0239A274F012039E9006F5125249700A
:106BA300089006F7125249604BAEA8C2AF1219D42F
:106BB3008A088B098C0A8D0B1219C88A0C8B0D8CD1
:106BC3000E8D0FEEA2E7E433FAEEA2E792AF9081C7
:106BD30076780C120A3D7808790C120B065011785E
:106BE30008790C1209EEAA08AB09AC0AAD0B800CAC
:106BF3007A0180027A007B007C007D0002353A74C2
:106C0300F012039E74B31209998A088B097F008AD4
:106C1300828B83A3A3E07003026CEB147003026CFA
:106C2300F1147003026CF7147003026D2E147003D9
:106C3300026D74147003026DA3147003026DDD14EE
:106C430070030271AD24FE7003026DE3147003023E
:106C530071AD24FA7003026E6F147003026EE224A6
:106C6300FD7003026E82147003026E8814700302B7
:106C73006EDC24F67003026E37147003026E371451
:106C83007003026E37147003026E1B147003026EDE
:106C930037147003026E4F24E57003026EF814700C
:106CA30003026F3B24FD7003026F61147003026FD4
:106CB3006724FD7003026FE71470030270201470E1
:106CC3000302702C147003026FC224FE700302705F
:106CD3008B24CD700302709114700302710F24A1F1
:106CE300700302719C0271AB121D520271AD121D31
:106CF300580271AD1271C3121E787401120BC3EAEC
:106D0300F0A3EBF07A837B00121FAA8A088B097425
:106D130001120953880A890B780A12090D7808129F
:106D2300090D7C007D007A83026DD08A828B83A358
:106D3300A3E0FE79041271CF121E7EEAF8EBF9ECA0
:106D4300FAEDFB7406120BC3120B707A847B0012EC
:106D53001FAA8A088B097406120953880A890B78BB
:106D63000A12090D780812090D7C007D007A8480CF
:106D73005C8A828B83A3A3E0FE7A617B00121FAA45
:106D83008A0A8B0BE5082403F508500205097808E5
:106D930012090D780A12090D7C007D007A61802D9D
:106DA3008A828B83A3A3E0FE7A627B00121FAA8AE6
:106DB3000A8B0BE5082403F508500205097808122D
:106DC300090D780A12090D7C007D007A627B00129E
:106DD3001FB074041208CF026FE1121D5E0271AD81
:106DE3001220168A088B098C0A8D0B90812A780C45
:106DF300120B547808790C12032F780812090574C2
:106E03000A12095B121EEA74041208CF74061209EF
:106E1300637B047A0902714E8A828B83A3A3E0FA0F
:106E23007401120BC374F5F07402120BC374FFF0F8
:106E3300740180308A828B83A3A3E0FA851882854C
:106E4300198374F51278397B0102714E8A828B8320
:106E5300A3A3E0FA7401120BC374F5F07402120BCE
:106E6300C3E4F0041209637B0202714EEA2403FCBB
:106E7300E43509FD8A828B83E0FB7A1002714E129E
:106E83001D640271ADE580C0E0740A120BC3D0E04B
:106E9300F0E590C0E0740B120BC3D0E0F0E5A0C0A6
:106EA300E0740C120BC3D0E0F0E5FDC0E0740D12EA
:106EB3000BC3D0E0F0E5FEC0E0740E120BC3D0E0CC
:106EC300F0E5FFC0E0740F120BC3D0E0F0740A12B8
:106ED30009637B067A1502714E121D6A0271AD8A2F
:106EE300828B83A3A3A3E0F91210921278327B0161
:106EF3007A1102714E1271E61209097C087D007441
:106F030022120BC3AA82AB83121E6074031208CF32
:106F1300741C12095B122A30741D120BC3E0F8A310
:106F2300E0F97401120BC3E8F07402120BC3E9F029
:106F3300740112096302701B1271C3121E78741D4F
:106F4300120BC3EAF0A3EBF0741C12095B122A3C88
:106F5300741F120BC3AC82AD837B0802714C121DEC
:106F6300700271AD8A828B83A3A3E0FE74011209C0
:106F7300631271CF12277E7403120BC3E9F07023DF
:106F83007401120BC3E0C0E07404120BC3D0E0F031
:106F93007401120BC3A3E0C0E07405120BC3D0E06D
:106FA300F080127C027D0079FF7404120BC3AA8265
:106FB300AB83121E7274031209637B0302714C12BA
:106FC30071E61209097C087D00742C12095B121EFC
:106FD3006074031208CF742912095B1227661278B2
:106FE3003202710B1271D850020509F582850983AB
:106FF300A385820A85830BE0FA850882850983E0ED
:10700300F91229BE850882850983EAF0850A8285FB
:107013000B83EBF0AC08AD097B0202714C1271F6E5
:10702300E0FA7B0012296A80451271D850020509E3
:107033000A0A0AAB09122A60E96006AA08AB0980AA
:10704300047A007B00850882850983A3A3A3A3A3F5
:10705300A3A3A3E0FC850882850983A3A3A3A3A319
:10706300A3A3A3A3E0F9EC2FE439FD1229888A082E
:107073008B09AC08AD09743112095B121D7C7431A4
:107083001209637B1C02714C121D760271AD1271E1
:10709300D850020509741A120BC3E4F0A31271B994
:1070A300E0C0E07419120BC3D0E0F07418120BC3E4
:1070B3007402F0E5082404FAE43509FB121E78741F
:1070C30010120BC3EAF0A3EBF0850882850983E075
:1070D300900BF61271B9A3E0F50A8F0B780A120927
:1070E3000D850882850983A3E0FC741212095B9065
:1070F3000BEEE0F912229E74021208CFE985088292
:10710300850983F0AC08AD097B01803D8A828B83BE
:10711300A3A3E0FEEA2403F50AE43509F50B7A019B
:107123007B00122292E9F50C2401FAE43400FB12ED
:107133001F2C8A088B09EA45097014850A82850B7E
:10714300837401F0AC0AAD0BFBEEFA796780548AC5
:10715300828B83A385820E85830F780E12090D859A
:107163000A82850B83E0F9A3AC82AD837A017B00AD
:1071730012229874021208CFE9850882850983F0E8
:10718300AC08AD097401250CFBEEFA7967121C56A5
:10719300AA08AB09121F3280117C007D007B007AA4
:1071A300E07947121C5680027F02EFF9744D1208F2
:1071B300CF7F0802060FF0850882850983A3A322E7
:1071C3008A828B83A3A3E0FE1271CF22EA2403FAFF
:1071D300E43509FB228A828B83A3A3E0FEEA24031E
:1071E300F508221271F6A982AA8389088A098F0AEF
:1071F3007808228A828B83A3A3E0FE8A828B83A3EF
:10720300A3A32274F012039E74FF120999750A0E48
:107213007E007F00851882851983E4F0901CC5E009
:1072230060046401701CAA18AB191229708A088BB8
:1072330009AE08AF09851882851983E0C333240E8C
:10724300F50AAA0A7B00121F2C8A088B09EA450952
:10725300700302733E8A828B83E4F0A385820C85DC
:10726300830D780C12090D750E08750F00780E1238
:10727300090D7C007D007A017B00121FB674041295
:1072830008CF1211F4850C82850D83A3A3A3A3A3B6
:10729300A3A3A3EA12735AEB12735AA37407F090D1
:1072A3001B59E0C0E0E50C240BF582E4350DF583B2
:1072B300D0E0F0901CC5E060046401706185188221
:1072C300851983E0C0E012734ED0E0F0E50C240D85
:1072D300F50C5002050D851882851983E06048EE90
:1072E300F8EFF97C00851882851983E0FAECC39ADC
:1072F300503588828983E0850C82850D83127D1940
:10730300A3E0850C82850D83A3F0E50C2402F50C24
:107313005002050D0CE82402F850CA0980C7127305
:107323004EE4F0E50C240DAC08AD09AB0A7A007904
:1073330067121C56AA08AB09121F32EE4F6007EE04
:10734300FAEFFB121F3274010271B1E50C240CF544
:1073530082E4350DF58322F0850C82850D83A3A38A
:10736300A3A3A3A3A3A3A32274F012039E74FA12EC
:1073730009997A207B00121F2C8A088B09AE08AF6B
:1073830009EE4F70030275427C207D0079FF121EC7
:10739300728E828F83A385820A85830B780A1209F2
:1073A3000D750808750900780812090D7C007D0029
:1073B3007A017B00121FB674041208CFE9F5086046
:1073C30003750801E50A2408F50A5002050B740247
:1073D300120953880C890D780C12090D750C04756C
:1073E3000D00780C12090D7C007D007A847B00125D
:1073F3001FB674041208CFE96008E508D2E1F50866
:1074030080607402120BC3780C120B547418780C3E
:1074130012093A850A82850B83E50CF07402120B7C
:10742300C3780C120B547410780C12093A850A8233
:10743300850B83A3E50CF07402120BC3780C120BBB
:1074430054E50D850A82850B83A3A3F07402120B06
:10745300C3780C120B54850A82850B83A3A3A3E57F
:107463000CF0E50A2404F50A5002050BA818A91923
:10747300880C890D780C12090D750C02750D0078B6
:107483000C12090D7C007D007A837B00121FB674F9
:10749300041208CFE96008E508D2E2F508801E85EA
:1074A3001882851983E0850A82850B83F08518820B
:1074B300851983A3E0850A82850B83A3F0E50A245B
:1074C30002F50A5002050B780A12090D750C0178B2
:1074D3000C12090D7C007D007A617B00121FB674CB
:1074E300041208CFE9F8850A82850B83A385820AF3
:1074F30085830B6006E508D2E3F508780A12090DC7
:10750300750A10750B00780A12090D7C007D007A4C
:10751300627B00121FB674041208CFE96006E50807
:10752300D2E4F5088E828F83E508F0EEFCEFFD7B55
:10753300207A017967121C56EEFAEFFB121F3274A0
:10754300060271B174F412039E74FF120999EAFEE4
:10755300EBFF8E828F83A3A3E0F50885188285193C
:1075630083E4F0EE2403FE50010FFAEFFB121E78C2
:10757300EB541FF98E828F83A3A3E06048740569DF
:10758300600A74FF6A700374FF6B700C900BF774DE
:10759300FFF0A3F0A3F0A3F0740469600A74FF6A18
:1075A300700374FF6B7008900BEA74FFF0A3F07420
:1075B3000669600A74FF6A700374FF6B704D900B69
:1075C300EC74FF8043740569600A74FF6A70037486
:1075D300FF6B700B900BF7E4F0A3F0A3F0A3F07430
:1075E3000469600A74FF6A700374FF6B7007900B81
:1075F300EAE4F0A3F0740669600A74FF6A70037426
:10760300FF6B7007900BECE4F0A3F0AC18AD197BA3
:1076130001AA087967121C5674011208CF7F04026D
:10762300060F74F612039E74FA120999908108AC3E
:1076330018AD197406120833E5FD85188285198380
:10764300F0E5FEC0E07401120BC3D0E0F0E5FFC02B
:10765300E07402120BC3D0E012783F7044E9600873
:107663001460181460288078750801750900E8789B
:1076730008120A9CE508F452FD8065750801750936
:1076830000E87808120A9CE508F452FE8052750857
:1076930001750900E87808120A9CE508F452FF8096
:1076A3003FE960081460171460268034750801757B
:1076B3000900E87808120A9CE50842FD8022750853
:1076C30001750900E87808120A9CE50842FE80105B
:1076D300750801750900E87808120A9CE50842FF5D
:1076E300E5FDC0E07403120BC3D0E0F0E5FEC0E09B
:1076F3007404120BC3D0E0F0E5FFC0E07405120B75
:10770300C3D0E01278397B067A147967121C567459
:10771300061208CF7F0202060F74F612039E74F757
:107723001209999080C2AC18AD197409120833E597
:1077330080851882851983F0E590C0E07401120BEF
:10774300C3D0E0F0E5A0C0E07402120BC3D0E0F0B8
:10775300E5FDC0E07406120BC3D0E0F0E5FEC0E027
:107763007407120BC3D0E0F0E5FFC0E07408120BFE
:10777300C3D0E012783F7044E960081460181460C5
:10778300288078750801750900E87808120A9CE5D5
:1077930008F452808065750801750900E8780812BD
:1077A3000A9CE508F452908052750801750900E8B7
:1077B3007808120A9CE508F452A0803FE960081497
:1077C30060171460268034750801750900E878088D
:1077D300120A9CE50842808022750801750900E8B9
:1077E3007808120A9CE50842908010750801750913
:1077F30000E87808120A9CE50842A0E580C0E0741E
:1078030003120BC3D0E0F0E590C0E07404120BC385
:10781300D0E0F0E5A0C0E07405120BC3D0E012780D
:10782300397B097A167967121C567409027714E9B1
:10783300851882851983F0AC18AD1922127C69E092
:10784300F98A828B83A3A3A3A3E0F88A828B83A301
:10785300A3A3A3A3E02274EE12039E74E512099975
:107863008A828B83A3A3E0F50AAC18AD19EA24033B
:10787300FA50010B12277E7402120BC3E9F0600366
:1078830002796A7A187B00121F2C8A108B11EA4541
:1078930011700302797C781012090D7508187509A7
:1078A30000780812090D7C007D007404120BC3E0FC
:1078B300FAA3E0FB121FB674041208CFE9600302B7
:1078C3007954851882851983E0F8A3E0F9E875F007
:1078D30009A4F8AAF075F009E9A42AF9747B28FA37
:1078E300741C39FBEA24FBF8EB34EDF9E8FEE9FFFD
:1078F300EA24F7F8EB34EDF98808890985100C853B
:10790300110D750E00780C1209097C107D007406A8
:10791300120BC3AA82AB83121E6074031208CF85B5
:10792300088285098312070D7417120BC3AA82AB51
:1079330083121EEA74041208CF8E828F8312070DFE
:10794300741B120BC3AA82AB83121EEA74041208BF
:10795300CF7C187D007900AA10AB11121E72AA10F9
:10796300AB11121F3280127C187D0079FF74031251
:107973000BC3AA82AB83121E7274021209637B19B2
:10798300AA0A7967121C567C197D007900740212C9
:10799300095B121E72741B1208CF7F0A02060F7452
:1079A300ED12039E74E9120999EAFEEBFF8E828FB2
:1079B30083A3A3E0F50F7C0E7D0079FF7409120900
:1079C3005B121E72740B120BC374FEF0740C120B59
:1079D300C374FFF08E828F83A3A3A3E0F50C8E8282
:1079E3008F83A3A3A3A3E0F87408120BC3E8F0EEFC
:1079F3002405FE50010F740368700DEEFCEFFDAA21
:107A030018AB191220408012EEFAEFFB121E788594
:107A13001882851983EAF0A3EBF08E828F83A3A3E8
:107A2300A3A3A3A3A3A3E0F50D8E828F83A3A3A394
:107A3300A3A3A3A3A3A3E0F50E606425E0F50AE4E2
:107A430033F50BAA0AFB121F2C8A088B09EE240AB2
:107A5300F510E43FF5117512007810120909AC0A0C
:107A6300AD0B121E6074031208CFE5084509602FA1
:107A7300780812090DAD0EAC0D740212095BA90C46
:107A830012180674021208CF8A0A8B0BAC0AAD0BCC
:107A9300740912095B121D82AA08AB09121F327402
:107AA300091209637B0EAA0F7967121C5674171209
:107AB30008CF7F0B02060F74F612039EEAFEEBFF5C
:107AC3008C088D09EC4509700C8E828F8374FEF04F
:107AD300A304027B7E8C828D83127B92127C7712AD
:107AE3007B8CF0EC2402F8E43509F988828983124F
:107AF3007B8D127D18127B98127C7D127B98127CF1
:107B030076127BA8127B85127BA8127C76127BB23D
:107B1300127B85127BB2127C76127BC4127B851298
:107B23007BC4A3F0EC240BF582E43509F583E0C0B4
:107B3300E0EE240BF582E43FF583D0E0F0EE240C75
:107B4300FE50010FEC240CF582E43509F58312078E
:107B53000DEEFAEFFB121EEA74041208CF8E828F29
:107B630083E02404F0E5082410F8E43509F9888259
:107B73008983127B92127D19127B8CF0EE24020210
:107B83007717F08C828D83A322A3127B92A322E02A
:107B93008E828F8322127B9C22127BA022A3127BD4
:107BA30092A3A3A322A3A3A3A3127B9CA3A3221206
:107BB3007BB622A3A3A3A3A3A3127BA0A3A3A3A3E4
:107BC30022A3A3127BB6A3A32274F512039EEC4D4A
:107BD300701E8A828B8374FFF0A3127C6FA314122E
:107BE3007C6504127C65A3127D12F0EA2406806D85
:107BF3008C828D83E08A828B83127C77127C86F061
:107C0300EC2402F8E43DF988828983127C87127D93
:107C130018127C86A3A3127C7DA3127C8EF0EC2425
:107C230005F8E43DF9E8FEE9FF8E828F83127C8E2E
:107C3300A3F0EC2406F508E43DF509750A0078087D
:107C43001209098E828F83E025E0FCE433FDEA24E8
:107C530006FA50010B121E6074031208CF7F030251
:107C6300060F127C6922127C6FA3A322F08A828BF7
:107C730083A322A3F08C828D8322F08C828D83A335
:107C8300A3A322A3E08A828B83A322E08A828B832D
:107C9300A3A3A3A322C082C08374FA120999900BF1
:107CA300F6E0851882851983F08A828B83E0C0E031
:107CB3007401120BC3D0E0127C6FE0C0E0740212B7
:107CC3000BC3D0E0127D12A3A3E0C0E07403120B38
:107CD300C3D0E0F0EA2405F8E43BF988828983E025
:107CE300C0E07404120BC3D0E0127D19A3E0C0E01E
:107CF3007405120BC3D0E01278397B067AE1794719
:107D0300121C5674061208CFD083D0820208B71211
:107D13007C69A3A322A3F08882898322F075E1E220
:107D230075E1FF027E2FA9A8C2AF75C300A8A2AA5E
:107D3300A3E9A2E7E433FCE9A2E792AFE4CAF97B43
:107D43000212024EE8F90208B7C082C0839061A410
:107D5300E0A2E4500312189C759C019061E4740145
:107D6300F075E1E275E1FFA8A8C2AF759B007591BC
:107D7300EFE8A2E7E433FAE8A2E792AFA9A8C2AF1B
:107D8300759B007591F7E9A2E7E433F8E9A2E7925E
:107D9300AF027E2FC082C0831219FE75E1BC75E16C
:107DA300B875E10F75E1D075E1D075E1D075E1D01B
:107DB300805FC082C0831219FE75E1BC75E117753F
:107DC300E18175E11075E1D275E1818044C082C023
:107DD30083900BDFE09061E2F075A1FDA2AFE43385
:107DE300FAC2AF75C300A8A2A9A3900B51E09412E5
:107DF3005008E87005E97002780175C30388A28909
:107E0300A3EAA2E092AF127E93121BF075E1E18028
:107E13001B75E11075E1D275E1D975E10175E109D1
:107E230075E1BA75E10175E1C575E1D2D083D08200
:107E33000208B7C082C0831219FE75E1BC80D874F2
:107E4300F712039E127E93A2AFE433F508C2AF7517
:107E5300C300E5A2AFA4740F5FF8740F98FE90619E
:107E6300E2F0121BDE900BDA7401F075E1E175C3E9
:107E730000E5A2E5A46F600DEEC39402400774FF12
:107E83002E9061E2F0E508A2E092AF7F0102060FB7
:107E93009061A4E0D2E4F0E0D2E3F022C082C08398
:107EA3009061E4E070179061A4E0A2E4500FE0C297
:107EB300E4F0E0A2E35003121A34121C38027E2FBE
:107EC30074F512039E9061A4E0A2E4500312189C7F
:107ED3001219F8E9F50A900B62E0FEC394155003FA
:107EE30012189C74EC250A2EFE75F01484FF75F0AD
:107EF30014A4CE9EFE0F9061E47402F0EF9061E251
:107F0300F0EEC39415400312189C75A1FDA2AFE4D3
:107F130033FAC2AF75C3038E087509007409780874
:107F2300120A9CF8A909900B51E0C394125006E978
:107F33007003087900E8F5A2E9F5A3EAA2E092AF9D
:107F430075E1E275E1FFA8A8C2AF759B007591EFDB
:107F5300E8A2E7E433FEE8A2E792AF75E1BC75E17E
:107F6300B875E1D29061A4E0D2E4F075E1E11219B1
:107F7300F8E9C3950A500A9061E2E06F7003E014D8
:107F8300F07F0302060FC082C0839061A4E0C2E4C5
:107F9300027D1FC082C0839061A4E0C2E3F0121C83
:107FA30050027E2FC082C0839061A4E0C2E4F090AF
:107FB30061E4E07005121C388015E064017005125D
:107FC3001C32800BE06402600312189C121C4402F2
:107FD3007E2FC082C0837A007900121B42D2879021
:107FE30061967406F0D083D0820208B70208B70204
:027FF30008B7CD
:077FF800851A87000208B79B
:10800000FFFFFFFFFFFFFFFFFFFFFFFFFFFFFFFF80
:10801000FFFFFFFFFFFFFFFFFFFFFFFFFFFFFFFF70
:10802000FFFFFFFFFFFFFFFFFFFFFFFFFFFFFFFF60
:108030000000000000000000000000000000000040
:108040000000000000000000000000000000000030
:10805000000000000000FFFFFFFFFFFFFFFFFFFF2A
:10806000FFFFFFFFFFFFFFFFFFFFFFFFFFFFFFFF20
:10807000FFFFFFFFFFFFFFFFFFFFFFAA285C168C3B
:1080800010E00D760EBC229024AC208E20AA22B4E3
:1080900018000000000000000000000000000000C8
:1080A00000000000000000000000000000000000D0
:1080B00000000000000000000000000000000000C0
:1080C00000000000000000000000000000000000B0
:1080D000000000FFFFFFFFFFFFFFFF00080004009C
:1080E000020001FFFFFFFFFFFFFFFFFFFFFFFFFF9A
:1080F000FFFFFFFFFFFFFFFFFFFFFF02050200087A
:10810000017482003A003B00000000000000000003
:108110000000000002000206030000000000FFFF54
:10812000FFFF000000FF96511800E80300006AAE50
:10813000E7FF97511800080000000000FF001F0033
:108140000000000000000A000000FEFFFFFF0048E2
:108150000000102700000400000019E0FCFFF8FFF9
:108160000000E71F0300805101003C000000100EDA
:108170000000E9FFFFFF010000000B000000FA0013
:108180000000300000006400000000000001030057
:10819000000000000000F0FFFFFF11000000F401EC
:1081A000000060EA0000E204000058020000BC0287
:1081B00000003200000000F8FF079F020000E90302
:1081C000000000000000000000000B74F712039E86
:1081D000E9900599F090054EE4F0121E309005B13B
:1081E000E4F0A3F090059AF0A3F0121362901CC57E
:1081F000E06004640170061229F4120CBA121E36F3
:108200009004D5E4F0A3F012285C02B42474EC12BC
:10821000039E74D7120999EAFEEBFF5480606890C0
:108220000599E0F9121EA28A088B09EA4509604FF8
:108230007C0080010CEC75F003A4F8A9F074EB2825
:10824000F582742F39F583E493F4602CE493F88578
:1082500008828B83E06870DCAA08EC75F003A4F850
:1082600074EC28F582742F39F583E493C0E074012F
:1082700093F583D082120529AA08AB09121E90EE4D
:10828000FAEF6480028751EF5420601E1211AC8A0D
:10829000088B09EA4509600A1210C2AA08AB091244
:1082A0001E90EEFAEF6420028751901CC5E0640234
:1082B000705FEEA2E0501F900553E0640F701179DB
:1082C00000121092E96009901E42120BAC1210AA23
:1082D000EE6401028668EF54406036901B59E064FA
:1082E000067028740BF0901E5AE0F97508017509A4
:1082F00000750A00750B00900541E078081208929D
:10830000AA08AB09AC0AAD0B121AE2901CB50287A1
:108310000FEE542070030286397A207B0090059975
:10832000E0F9122004EA4B4C4D701A9005AD120B87
:108330007CE8494A4B700E750C01750D00750E00F6
:10834000750F008061750C00750D00750E00750FBE
:10835000001220168A088B098C0A8D0B9005AD122D
:108360000B7CE8494A4B602A9005AD7808120873E7
:10837000400E750CFF750DFF750EFF750FFF801217
:1083800085080C85090D8C0E8D0F9005AD780C12AB
:10839000096B7401780C12093AE50C450D450E4540
:1083A0000F70030285607C0079047A007B00121153
:1083B000708A088B0902848D85188285198374FF61
:1083C000F07401120BC374FFF07402120BC374FF3C
:1083D00012A344FAA3E0FB740312096312D2211220
:1083E00011D6E96401600302846FE508240D12B020
:1083F000274480F8A3E0F97424120BC3E8F0A3E942
:1084000012C57AA3A3A3E0C0E07426120BC3D0E088
:1084100012D029A3E0540860167424120BC3A3E001
:108420004401128774C0E07428120BC3D0E0F0E559
:108430000812EDC5350912D002601CE508240F12A0
:10844000CCF1A3E0C812C54238F583E0F8741212EB
:108450000BC3E8F0A3E4F090814212070D740412FC
:108460000963740712095B120C1E74041208CF858D
:108470000882850983A3A3A3A3A3A3A3A3A374062C
:10848000128774F9121152850A08850B09E508450F
:108490000970030285607C007904AA08AB091211F7
:1084A000708A0A8B0B850882850983A3A3A3A3E0A6
:1084B000F510A3E0F511E4F512F513780C7910121C
:1084C0000B064023E5082404F8E43509F9850C106F
:1084D000850D1188828983C3E09510F0A3E0951182
:1084E00012F24870A2800E850882850983A3A3A397
:1084F000A3E4F0A3F0850882850983A3A3A3A3A323
:10850000A3A3A3A3A3E06401850882850983A3A391
:10851000A3A3A3A3702BE0540460030283B88508CF
:1085200082850983A3A3A3A3A3A3A3A3A37406F093
:108530007AB78508828509831289571210A40284AC
:1085400087A3A3A3A3E060030283B88508828509FB
:1085500083A3A3A3A3A3A3A3A3A37401F00284876B
:108560001211407C0079017A007B001211708B0996
:10857000EA4509600C7A207B00900599E0F9121E0B
:10858000CC850C0A850D0B7C0079047A007B0012E7
:108590001170EA4B701580558A828B83A3A3A3A325
:1085A00012E704E50898E5099940098A828B83A3BC
:1085B000A31287667C0079041211708B0DA90DEA55
:1085C0004970D5C3E50A9508E50B95095013C3E535
:1085D00008950AF508E509950BF509E508450970C0
:1085E000147A207B00900599E0F9121ECC9005AD1D
:1085F000129B70803FE50825E0F508E50933F50991
:10860000E4F50AF50B78081209057A207B0090053D
:1086100099E0F9121FF274041208CF122016EAC072
:10862000E0EBC0E0ED9005ADFBECFAD0E0F9D0E076
:10863000F8120B70EE6420802FE060076401600385
:1086400002872AEE54106008120CF6EE64108018AF
:10865000EE54406008120D6EEE6440800BEE5480C4
:10866000600B1229D0EE6480FAEF028751EF5401BB
:10867000600B121338EEFAEF6401028751EF5408D1
:108680006047120CC6901CAFE064017034901CB0BF
:10869000E0602EF508E4F509F50AF50B90812A78DB
:1086A0000C120B547808790C1202AF7808120905E5
:1086B0007A007B08900599E0F9121FF874041208FB
:1086C000CFEEFAEF6408028751EF54106012900564
:1086D000ABE06005E4F0120CC6EEFAEF64108071B6
:1086E000EF544060459005D212D0046036901CB91A
:1086F000E06401702E9005D312C926120529900559
:10870000D812D004600612C92612052990812A12B7
:10871000070D7A007B40900599E0F9121FF8740468
:108720001208CFEEFAEF64408027EF5402600A127D
:108730001332EEFAEF64028018EF5404601612CE82
:10874000D8790190054C12CD05120C3CEEFAEF647D
:1087500004FB80047A007B0074291208CF7F0C028E
:10876000060F8E828F83A3A312876C22E0F508A3E5
:10877000E0F5092212C57EA3E022C082C08374EA1C
:108780001209997C167D007900AA18AB19121E7285
:108790007408120BC37402F0900542129B431287B7
:1087A000BA7409120BC312CD147413120BC3E41262
:1087B000D03B12284A741602D5F4E8F0A3E9F090F1
:1087C000054C12D5B72274F712039E74DA12099978
:1087D000EAFEEBFFEE4F602DAC18AD191211D67406
:1087E00006120BC3E0601E7417120BC3E0FD740188
:1087F000120BC3E0FCEEFAEFFB7900121068E9609F
:108800000479A480027900742602B42174F412035E
:108810009EEAFEEBFF8E828F83A3A3A3A3A3A3E014
:108820005440601912E36612CD05121290E96007F8
:108830007AFF7BFF02890112E3660288F4901CC56F
:10884000E06007640160030288E9900539E0A2E175
:1088500040030288E912B46712CE04A3A3A3A3E0E5
:10886000FA88828983A3A312D9838E828F83A3A3DC
:10887000A3A3A3A3A3E0541060047940800279006D
:10888000750AFE750BFF780A12090D128945120749
:1088900011AC08AD0912E36612CD05120CCC7404BC
:1088A0001208CFE5086A7003E5096B600B12BFC3BD
:1088B0006A7003A3E06B703F750A00780A12091111
:1088C00079028E828F8312B528FCA3E0FDAA08AB43
:1088D000091212D274011208CF7508CDAA081289A4
:1088E000531210A4E9604C8057901CC5E0640270DC
:1088F000E890054212CD0574FE6A700374FF6B6048
:10890000D812E36612E1D6121290E98E828F83604C
:108910000B12BCE112F51AE4F0A3800312F508F083
:108920007C987D108E828F8312CD05122850E9F538
:108930000870A9EE4F60097901EEFAEFFB12114CB5
:10894000A908028FF5EE12894A222411F582E43F2C
:10895000F583228E828F8312F4F1E0F92274F612ED
:10896000039EE9FEEAFF7A0F7B00121E8AEA4B6043
:108970001F8A828B83740CF0EEA3A3F0EF8A828BA4
:108980008312B1DD900599E0F9121E967900802FCF
:10899000EEF91211768A088B09A808A909E849603E
:1089A0001C88828983A3A3A3A3A3A3A3A3A3740660
:1089B00012EDCBE0F9120D80EEF91211527910028E
:1089C000C98374F412039E8A088B098C0A8D0B905C
:1089D0000553E0640F702CEA4509450A450B6023F6
:1089E00090054EE064086005E06404701678081293
:1089F00009057A017B00900599E0F9121FF27404D1
:108A00001208CF028FF574F212039EEAFEEBFF8C80
:108A10000A8D0B8908740E120BC312E709850C82AC
:108A2000F583E4F0A312CECDF5838882E0F912122B
:108A30006CE9602612CCF8121290E96402701B8E69
:108A4000828F83A3A3A3A3A3A3A3A3A312BB4E8537
:108A50000C82850D8312CD14800375080012B51F9A
:108A600014602E14604314606414606C1460481425
:108A70007003028AF824FE7003028B121470030242
:108A80008B1B147003028B2E147003028B3C028B21
:108A900052780C12090DAC0AAD0BEEFAEFFB120C7A
:108AA000DE74021208CF028B37AC0AAD0BEEFAEF80
:108AB000FB120CE4028B5C12CCF8121290E96003FA
:108AC000028B52EEFAEFFB120D32028B5CA908EE1C
:108AD000FAEFFB1212D8805F12B9E264027073E5FC
:108AE00008700A12E28C7003A3E069706FEEFAEF6F
:108AF000FBA908121260803F12E28C7003A3E069A8
:108B0000705012B9E264027049EEFAEFFB1212489B
:108B1000804AEEFAEFFB121356804112E28C70038A
:108B2000A3E069702DEEFAEFFB1212E4802EEEFA4C
:108B3000EFFBA9081212F0E9F5088020901CB9E0BB
:108B400064017009EEFAEFFB1212FC800F75080049
:108B5000800A7508007AD37B00122472A908800766
:108B6000A90A74031208CF7F0602060F74F41203D9
:108B70009E74D61209998A088B098A828B83A3A3D3
:108B8000E0F91211768A0A8B0BAE0AAF0BEE4F702A
:108B900003028C9E850882850983A3A882A983E0AD
:108BA000C0E012CCDFD0E012E716E064F16033855C
:108BB0000882850983A3E064CD6027850882850942
:108BC00083A3E0641A601B850882850983A3E0649F
:108BD000E9600F850882850983A3E064E1600302F0
:108BE0008D96901CC5E0600764016003028CBF8E07
:108BF000828F83A3A3A3A3A3A3A3E05408700302BB
:108C00008CBF8E828F83A3A3A3A3A3A3A3A3A374C8
:108C100005F0901CC5E060046401705385088285EE
:108C20000983A3E064E960479005CE12D004600692
:108C300012C9261205299005D012D0046031900582
:108C400039E0A2E1502912D1F7A3A3A312BA2088D8
:108C500082898312CD05121392EA4B601285088235
:108C6000850983A3E0F99005D012E36A1205298EE5
:108C7000828F83A3A3A3A3A3A3A3A3A3E0640270EF
:108C8000108E828F83A3A3A3A3A3A3A3A3A374067D
:108C9000F0850882850983A3A3E0F912115212110D
:108CA00040901CC5E064027011901E48E0F508A3D6
:108CB000E0AA08FBE4FCFD1210AA742A028FF279E4
:108CC0000012114CE97003028D96901CC5E06007FC
:108CD00064016003028D6B900539E0A2E14003025C
:108CE0008D6B12CFFF7003028D6B8E828F8312CD3E
:108CF00005740412096312D2211211D685088285E7
:108D00000983A3E064E97023128EA012091185087B
:108D100082850983A3E0F50A780A120911128EAD43
:108D200012CD0512120C74021208CF740D120BC36F
:108D300012CFF512F17312CD147409120BC3E06057
:108D400004794080027900740F120BC312BA2074A8
:108D50000D120BC312CD05120CD8E9600E8E828F56
:108D600083A3A3A3A3A3A3E04420F0EE2404F50A65
:108D7000E43FF50B8E828F8312B034E0F9850A82CE
:108D8000850B8312CD05121E42850A82850B83EA6C
:108D9000F0A3EB028C11850882850983A3E0C0E073
:108DA0007402120BC3D0E012A82412E172E5082469
:108DB0000B12B027C0E07403120BC3D0E012E9D944
:108DC000E0AA18AB197031120C18901CC5E06004B1
:108DD000640170277402120BC3E0701F12E3661265
:108DE000CD05121290E970399005CE12D004603191
:108DF00012C92612052980031212667402120BC3CF
:108E0000E064E9701C128EA0120911750AE9780A53
:108E1000120911128EAD12CD0512120C7402120835
:108E2000CF901CC5E0600764016003028C6F900561
:108E300039E0A2E14003028C6F8E828F83A3A3A34B
:108E4000A3A3A3A3A3A3E06402703C8E828F83A399
:108E5000A3A3A3A3A3E05404602D12E36612CD05DF
:108E6000121290E98E828F83700F12E36A74FFF002
:108E7000A312A9D47405028C90A3A3A3A3A3A3A3B4
:108E8000A3A37403028C90850882850983A3E06400
:108E9000E96003028C6FEEFAEFFB12130E028C6F87
:108EA0008E828F8312DAB9750A01780A22E50824C6
:108EB0000C12BFE2E0F98A828B83A3A3A3A3A3A32E
:108EC000A3A3A312D97B2274F412039EEAFEEBFF44
:108ED0007508007509008E828F83A3A3A3A3A3E066
:108EE000603B75080812CCF879FF120E828B0BEAF2
:108EF000450B601075082C8E828F83A3A3A3A3A3B8
:108F0000E0D2E0F08E828F83A3A3A3A3A3E0540357
:108F100064016003028FD1430811028FD1EE24183F
:108F200012B9E56049EE241A12B9E56003F4701D28
:108F300012E28C7003A3E0697006750822028FD1DB
:108F400090054EE064046003028FD1801CEE241B68
:108F5000F582E43F12BA2E241A12B9E5FAEE24196A
:108F6000129C00120D44E97068750901806312CCEF
:108F7000F8121290E96402700375080112E28C7015
:108F800003A3E0697006E508D2E1F508E50860157D
:108F90008E828F83A3A3E07006E508D2E58004E506
:108FA00008D2E6F50812CCF8121290E964017006B6
:108FB000E508D2E0F5088E828F83A3A3E060121249
:108FC000B51FF912126CE964016006E508C2E0F50C
:108FD00008901CC5E0600464017012E508A2E1403D
:108FE0000CE509A2E04006E508D2E7F50802894051
:108FF00074181208CF7F0402060F74EC12039E74DB
:10900000C3120999EAFEEBFF85188285198374FE65
:10901000F0A304F0751000751100750900901CC5CF
:10902000E0640270248E828F83A3A3A3A3E060195F
:10903000901E4612D0046011901E46E0F50AA3E08F
:10904000AA0AFBE4FCFD1210AA74051209638E82C1
:109050008F83A3A3A312CFF712CD031211D6E97009
:109060000302943678017407120BC3E0C3940240E4
:109070000278007409120BC3E0C394024002780026
:10908000740E120BC3E064F87003A3E0F4700302E3
:109090009436740E120BC3E064F97003A3E0F4700D
:1090A00003029436740E120BC3E064FA7003A3E05B
:1090B000F47003029436740E120BC3E064FB700369
:1090C000A3E0F470030294367408120BC3E0F99025
:1090D000053CE0696003029436E8A2E04003029494
:1090E00036901CC5E06402700B7429120BC3E0605B
:1090F0000302943612BB457424120BC312BA4F24D8
:109100001C12BB487412120BC312CD14740B120B39
:10911000C3E0601D741C120BC3E0FD7406120BC388
:10912000E0FC8E828F8312CD037901121068E97002
:109130003D740512095B1210BCE9F508740B120BA3
:10914000C3E0702F900536E0602974225508642230
:10915000602174425508644270147422120BC312C9
:109160009B1C600F7422120BC3129B2260057ACFE6
:10917000029438E9A2E6506C901CC5E060046401DA
:10918000701B900539E0A2E150137422120BC31238
:10919000B52812079601010BBB9100369474221278
:1091A0000BC312B52824FD601214600F24FD600B60
:1091B00024FD600724FE60030294367422120BC360
:1091C000129B5B700F7422120BC3A312C926A3E07B
:1091D000640D6010740512095B1212CCE964017011
:1091E00003029B05EE242DF582E43FF58312A3379D
:1091F0007003A3E0697021750A00780A12091178DA
:109200000A120911EE242F129C00129B2812CD0580
:1092100012120C74021208CF740B120BC3E070030D
:109220000292C7129B2812CD051213928A0A8B0B49
:10923000EA450B700302935E7406120BC3E0F88ECE
:10924000828F83A3A3E028F8A3E03400F9E8240D7B
:10925000129B0AF88A828B83A3A3A3E068600EE8BE
:109260008A828B83A3A3A312B1CB129B707904745F
:1092700006120BC312A687E02AF8A3E03400888206
:10928000F583A3AA82AB83121E7E8A0C8B0D8C0EF3
:109290008D0F850A82850B83A3A3A3A3780C1208E4
:1092A000734003029B05908176780C120A3D850A73
:1092B00082850B83A3A3A3A3E50CF0A3E50DF0A384
:1092C000E50EF0A3E50FF0901CC5E0640260030218
:1092D000940B90054EE064046008E06409600302AA
:1092E0009B05E508A2E54003029399EE242F12B9ED
:1092F000E5C0E07402120BC3D0E0129B81C0E074A1
:1093000003120BC3D0E0129B79C0E07404120BC3AC
:10931000D0E0F07416120BC3E064017026741012D2
:109320000BC3129B387003A3E0697017740E120B05
:10933000C312CD05121290E9640270077416120B65
:10934000C3E4F0129B6612070D74061209637409D8
:1093500012095B120C1E74041208CF029B059005C3
:1093600093E0640160030292C77422120BC3129B44
:109370001C7009E508A2E650030292C77412120B92
:10938000C3E0F47003A3E0F4600CEEFCEFFD7405A1
:1093900012095B1210C8029B05A2E64003029B055E
:1093A0007422120BC312D2047016741C120BC3E089
:1093B00064027054740512095B79001212608048CF
:1093C0007422120BC3129B227014741C120BC3E084
:1093D00064047034740512095B121254802A7422DA
:1093E000120BC3129B5B700C7900740512095B129F
:1093F00012D880147422120BC312B52A640C7008A0
:10940000740512095B121308029B05E060076401F2
:109410006003029B05900539E0A2E14003029B0531
:109420007429120BC3E060267410120BC312CD0511
:109430001229A0E9700A7AD37B00122472029B05DC
:109440008E828F83A3A312E36AA3E0C2E5F07416B1
:10945000120BC3E0601DEE2402F8E43FF9E8FAE9DC
:10946000FB12D20A14F012D20AF87416120BC3E8D7
:10947000F07006E508C2E7F508E508A2E35061755B
:109480001110A2E25018740A120BC3E054E3F074F6
:109490000A120BC3E0131313541FF8E0802CA2E44C
:1094A000502A740A120BC3E01313543F5407F86098
:1094B00009740768600B18E87007C3E508C2E7F590
:1094C00008E8333354FCF8E054E348F0740A120B14
:1094D000C3E0C0E08E828F83A3A312B112D0E0F06C
:1094E00090054EE064046008E0640960030295BCE6
:1094F000740E120BC312E2997003A3E069601F742B
:109500000E120BC312CD05121290E96402600F74A3
:109510000A120BC3E0540364016003029B05740745
:10952000120BC3E07041EE242F12B9E5C0E07402C3
:10953000120BC3D0E0129B81C0E07403120BC3D0A6
:10954000E0129B79C0E07404120BC3D0E0129B615F
:1095500012070D7406120963740912095B120C1EBE
:1095600074041208CF80527422120BC312D20470FA
:1095700016741C120BC3E06402703E740512095B82
:10958000790012126080327422120BC3129B227077
:1095900014741C120BC3E06404701E740512095B82
:1095A00012125480147422120BC3129B5B700A793E
:1095B00000740512095B1212D8029B0574615508EC
:1095C00070030296C3E508A2E0506D12BA17740545
:1095D00012095B120D74E9705C121206E9F5097448
:1095E00016120BC3E0700F7410120BC3129B38706D
:1095F00003A3E0696042A90912BA17740512095B56
:10960000120D7AE96024E508A2E3500C85188285E2
:10961000198374FFF0A3800C740E120BC3129B43CA
:10962000E8F0A3E9F0751004800EE508C2E5F5083E
:10963000750900800353089FE508A2E5503FEE241A
:109640002F12B9E5C0E07402120BC3D0E0129B8167
:10965000C0E07403120BC3D0E0129B79C0E0740425
:10966000120BC3D0E0129B6112070D74061209633E
:10967000740912095B120C1E74041208CFE508A2CB
:10968000E64003029998A818A919880A890B780A54
:1096900012090DA909129B1312095B1210B0740272
:1096A0001208CFE9F50970030299987422120BC3CE
:1096B00012B5286401600302999874104510F510E2
:1096C0000299987407120BC3E06401705D74221252
:1096D0000BC312B5286405701EA818A9198808893B
:1096E00009780812090D129B1112095B1210B0744F
:1096F000021208CF029B057422120BC3129B5B70EF
:1097000029740E120BC312CD051229A0E9601BA803
:1097100018A919880A890B780A12090D129B1112CF
:10972000095B1210B074021208CF7416120BC3E05A
:1097300070257407120BC3E06401700C7422120BC5
:10974000C3E0F8129B5B600CEEFCEFFD74051209A0
:109750005B1210C8029B05121146E96003029B05CB
:10976000741D120BC3E070030298117420120BC316
:1097700012BA20741F120BC3E0FA741E120BC3E05E
:10978000F9120D44E9607D741F120BC3E0701E7462
:109790000E120BC3129B4312F52AFAA3E0FB122907
:1097A000948B0BEA450B600302999280517420124E
:1097B0000BC312CD05741F120BC3E0F9120D3E85C9
:1097C000188285198312E1D67808740D120BC3E054
:1097D00060027810740C120BC3E06004740828F85F
:1097E000740A120BC3E0600108088E828F83A3A362
:1097F000E028FAA3E034008A82F583E014F07510C3
:10980000400299927508007808120911790B0299A3
:109810004B740E120BC312CD097409120BC3E06016
:1098200003029966E508A2E35003029966740712E1
:109830000BC3E06401607A79008518828519831270
:10984000CD05120D988A0A8B0BA80AA90BE849606E
:109850001C88828983A3A3A3A3A3E0640160528828
:10986000828983A3A3A3A3A3E064026044EE242D12
:1098700012BA1A85188285198312CD051213928A9D
:10988000828B83E5824583600FA3A3E0F91213B0B6
:10989000E96005C3940840197410120BC312CD057A
:1098A0001229A0E970030299417409120BC37404D0
:1098B000F07800E8F5097809120911741E120BC33B
:1098C000AC82AD83740F120BC312CD05740A120B58
:1098D000C3E0F9120DAA74011208CFE9600F7510E8
:1098E000208E828F83A3A312B528543FF0741D12DB
:1098F0000BC3E06023740E120BC312BA20741E1245
:109900000BC3AA82AB831211D085188285198312EA
:10991000E1D674404510F5107407120BC3E06401E2
:10992000601579007410120BC312BA20740E120B5A
:10993000C312CD05120D4AE508A2E35037794080E5
:109940003575080078081209117902740F120BC3DB
:1099500012BA207411120BC312CD051212D2740167
:109960001208CF029B05E508A2E340030298B178F4
:10997000400298B379007410120BC312BA20740E0F
:10998000120BC312CD05120CD8E9600674204510E5
:10999000F510121206E9F509851882851983E0642D
:1099A000FE7003A3E0F47003750900901CB2E0643C
:1099B000016003029A4BEE241312B9E5F47003A37D
:1099C000E0F47003029A4B740E120BC3C3E094F9D7
:1099D000A3E094FF507512BB457410120BC3E068EE
:1099E0007003A3E06960647410120BC312CD0512FA
:1099F00029948A0A8B0BA80AA90BE849604D888232
:109A00008983A3A3A3A3E06401600D88828983A353
:109A1000A3A3A3E0640270337430120BC374011269
:109A2000E720F8A3E0F9743B120BC312CD14743095
:109A300012095B122A24E960127433120BC3AA8242
:109A4000AB83122982E960031223FAE508A2E740FA
:109A500003029B05E5097003029B058E828F83A399
:109A6000A3A3A3E0FA7B00121F2C8A0A8B0BEA4502
:109A70000B7003029B05EE2404F512E43FF5138EF0
:109A8000828F83A3129B4D1209098512828513834D
:109A9000E0FC7D00121E6074031208CF7407120BE5
:109AA000C3E0C0E0742B120BC3D0E0F0742E120B95
:109AB000C3E4F0A3F0742B120953880C890D780CC1
:109AC00012090D7508007808120911781012090D95
:109AD000E509F508780812091112B9D9120711859C
:109AE0001282851383E0F97408120BC312BA20AAFC
:109AF0000AAB0B1211C474081208CFE96007AA0A56
:109B0000AB0B121F32743D02875AF582E412EF5EEE
:109B100022790012B9DD12BA2474072212B5426408
:109B2000062212B544640722EE242BF582E43FF5A9
:109B30008312BA3412B9DE2212D5B7EE241312BF43
:109B4000CA682212D5B785188285198322A3E0F549
:109B50000CA3E0F50D750E00780C2212B5446403D9
:109B600022F0129B6622EE2425F582E43FF5832243
:109B7000E4F0A3F0A3F0A3F022F0EE243112BFCA68
:109B800022F0EE243012BFCA2274F412039EEAFEC1
:109B9000EBFF8C088D09901CAFE0600F12E28C7017
:109BA00003A3E0697005120CC68052790012CCF84C
:109BB000120D988A828B83E58245836035A3A3A327
:109BC000A3A3A3E05418602AE508241C12CCF112C8
:109BD0000711E508241312CCF1120711EE24181214
:109BE0009C00129C0512CD05120DB074041208CF12
:109BF000800B7900129C0512CD05120CF0028FF536
:109C000012BFCAF9228E828F83A3A3A3A3A3A3A307
:109C1000A3A312BA3412CCE42274F012039E74EAA5
:109C20001209998A0A8B0BEA2402F50EE4350BF52A
:109C30000F0A0AFB12298E8A088B09AE08AF097534
:109C40000801850A82850B83A3E0F509750C01AC38
:109C50000EAD0F740B120BC3AA82AB83122040749B
:109C600013120BC374FEF0A304F07415120BC3742B
:109C700002F07408120BC3E4F0901DDAE0700EEEEF
:109C80004F700AE50970067508C3029E5590054E8F
:109C9000E0640860067508C2029E51850A82850B41
:109CA00083A3A3A3A3A3A3A3A3A3A3E0A2E1500E12
:109CB000A2E35005750C04800C750C038007A2E329
:109CC0005003750C02EE4F7003029D648E828F83E9
:109CD000A3A3A3A3E06404600D8E828F83A3A3A338
:109CE000A3E06403700C7404650C602C7403650CB1
:109CF00060268E828F83A3A3A3A3E06402600D8EEF
:109D0000828F83A3A3A3A3E0640170317402650C66
:109D100060067401650C70188E828F8312CD051257
:109D200012AEE9703F12A9CA120BC312CD148034CF
:109D30008E828F83A3A3A3A3E06402600D8E828F23
:109D400083A3A3A3A3E06401700A8E828F8312CD44
:109D500005120D0EE50A2402FAE4350BFB122982E6
:109D60007E007F007413120BC3E064FE7003A3E057
:109D7000F47046122A18E97040E509601B901DE353
:109D800012CD051212AEE9700F901DE312A9CE128A
:109D90000BC3E8F0A3E98020850A82850B83A3A387
:109DA000A3A3A3A3A3A3A3A3E05402F9120D0274D7
:109DB00013120BC3EAF0A3EBF07413120BC3E064AD
:109DC000FE7003A3E0F470067508C7029E51E50912
:109DD000F50D780D120911850A82850B83A3A3A3C3
:109DE000A3A3A3A3A3A3A3E0F9E50A2402FCE435FB
:109DF0000BFD7414120BC312CD05120C4274011228
:109E000008CFE9704CA90CE50A2402FCE4350BFDEF
:109E10007413120BC312CD051229B28A0E8B0FAE2A
:109E20000EAF0FEE4F601F74026509700D8E828FAA
:109E300083A3A3A3A3A3E0D2E3F07415120BC3E49E
:109E4000F0750800800B7413120BC374FEF0A304AA
:109E5000F0E5097009AA18AB19122832800AFCA98A
:109E60000CAA18AB1912124EE9FCEE4F6053E5092B
:109E700060208E828F83A3A3A3A3A3E0D2E6F07415
:109E8000026509700D8E828F83A3A3A3A3A3E0D2E2
:109E9000E5F0850A82850B83A3A3A3A3A3A3A3A3B1
:109EA000A3A3E0A2E6500D8E828F83A3A3A3A3A356
:109EB000E0D2E7F08E828F83A3A3A3A3A3A3E00441
:109EC000F0E508703BEC60337D007A017B10121ED8
:109ED0003CEE4F600CE50A2402FAE4350BFB122934
:109EE000827413120BC3E064FE7003A3E0F4600BF2
:109EF0007413120BC312CD05120D0E741602D9A5E0
:109F0000FC80C574F712039E74F7120999EAFEEB00
:109F1000FF90054EE06403600DE064016008E064BA
:109F200009600302A0528E828F83A3E0600302A027
:109F3000107C007D007A027B00121E3C12A0578A22
:109F4000828B8312BB4E90053F12CD147953122899
:109F50002690054EE06409600990054C12CD05126B
:109F6000138C851882851983740112D03B794212B3
:109F7000282690054E7404F0740112095B794A1288
:109F8000282074011209637A447B05122040901B3B
:109F900059E0640B70057406F0800B790090054C55
:109FA00012CD05120C3C901CC5E060046401701FCA
:109FB000900542E064FE7003A3E0F4602A79007427
:109FC0000112096390054212CD051229B28018E0F2
:109FD0006402701390053F12BA207A037B00121EB0
:109FE0003C12A8B6121E3C900539E0A2E35004D200
:109FF000F08002C2F012D0317952122826901CC58E
:10A00000E06402704A901E42120BAC1210AA803F0C
:10A01000FC7D007A037B10121E3C901CC5E064029C
:10A02000701B901B59E0640B7003740AF0901CB312
:10A03000E4F0FA7B40900599E0F9121FFE8E828FC2
:10A040008312A06112CD05120C3C90054EE4F01273
:10A050001116740902B421EE2402FAE43FFB22E057
:10A06000F8A3E0F990054C22C082C0839004D51279
:10A07000D004701F90054EE014600924FC600A149F
:10A08000600C800F9004E080349004DC802F9004FA
:10A09000DE802AE84960089004D612A698700C8ADF
:10A0A000828B83A3E0F9120C24801D9004D512D278
:10A0B0000E64027005121326800E9005CC12D00497
:10A0C000600612C92612052902C5F174F412039E16
:10A0D00074FE1209998A088B097A007B049005990D
:10A0E000E0F9121FFEAA18AB1979501228207A0F36
:10A0F0007B00121E8A8A0A8B0BAE0AAF0BEE4F60F2
:10A1000020850882850983A3E0701690054CE0F451
:10A110007003A3E0F4603B12A3317003A3E0696015
:10A1200031850882850983A374EA12A81C122826A7
:10A130007A427B05794B1228267A4C7B057950129E
:10A1400028267A417B0579E1122826EE4F7003021A
:10A15000A1DB8E828F837402F090054CE0F47003D3
:10A16000A3E0F4600A12A3317003A3E069704F8585
:10A17000188285198312A05FE8F0A3E912A81C12C7
:10A18000282090053F12B04512CD147A427B057904
:10A190004B1228207A417B0579E1122820750A00AC
:10A1A000780A120911780A120911901E2912A06268
:10A1B00012AD7B12CD0512120C74021208CF850865
:10A1C0008285098312A1E0A3F090054E7403F0EE9E
:10A1D000FAEFFB900599E0F9121E967402028FF2D5
:10A1E000A3E08E828F832274F412039E74E8120916
:10A1F00099EAFCEBFD8C828D83A3A3A3A3780812BC
:10A200000B547808120AF690054F7808120A767FE8
:10A210007F7E7F790090054F7808120B54E978080B
:10A2200012093AE508A2E05029780090059A8014B6
:10A23000850882850983A3A3E069700108E50824E5
:10A240001412CCF112AA6570E7E8C39F5004E8FF2E
:10A25000E9FE09E9C3941B40BC8C828D83A3A3A3B0
:10A26000A3120B7CE8494A4B6079EC2404F508E41E
:10A270003DF509850882F583120B7C90054F120B82
:10A28000707C187D007900AA18AB19121E7285081F
:10A2900082850983120B7C851882851983120B70C5
:10A2A0007404120BC37401F0900555E0C0E074050E
:10A2B000120BC3D0E0F07407120BC3E412D03B12B0
:10A2C000283E806A90054C12CD05120C728A0A8BCA
:10A2D0000BA80AA90B90054C12A340687003A3E0D9
:10A2E00069602D90059A12AA656025850882850906
:10A2F0008312A3377003A3E069700C850882850977
:10A3000083A3A3E06E60BDE508241412CCF180D6CF
:10A31000EE900541F01210F8E9601390054EE4F05C
:10A320009004E212D004600612C924120529028F9B
:10A33000F085188285198312D5B790054CE0682204
:10A34000E8F0A3E912A34822F0850882850983E09A
:10A350002274F412039E74E81209998A828B83A3F3
:10A36000A3A3A3A3A3A3A3A312DAB57C0090054FD4
:10A370007808120B54EC780812093AE508A2E0506C
:10A380002FECF8EA2812BB3DF8901DE2E0C398508C
:10A390001F750801750900750A00750B00EC780837
:10A3A0001208927808120AF690054F7808120A7679
:10A3B0000CECC3941B40B690054F120B7CE8494A45
:10A3C0004B604E7C187D007900AA18AB19121E72E2
:10A3D00090054F120B7C851882851983120B7074BF
:10A3E00004120BC37401F07407120BC37401F090D4
:10A3F0000555E0C0E07405120BC3D0E0F0740712FD
:10A400000BC3E412D03B12283E90054E7406F08038
:10A410001C90054EE4F0FCFD7A047B10121E3C906B
:10A4200004E212D004600612C924120529028FF03A
:10A4300074F512039E74D11209998A088B098A82D5
:10A440008B8312BCD9741C1209638A828B83A3A3E9
:10A45000A3A3A3A3A312A69012CCFC121128741CD0
:10A46000120BC3E0702C850882850983A3A3A3A3E4
:10A47000A3A3A3A3E0C3940B40188E828F83A3A34E
:10A48000A3A3A3A3A3A3E06402700712CCDFE0F4AC
:10A49000600302A68290054EE06402700302A56785
:10A4A000E06406700302A5679004D512D00460082A
:10A4B00012A698700302A59B90054EE06408600800
:10A4C000E06404600302A682741E120BC312A68706
:10A4D000A3A3A3A312BCD99004D5E0F84960071246
:10A4E000D2146402607790054CE06E7003A3E06FB5
:10A4F000600302A68274016A60167423120BC3AC57
:10A5000082AD837A607B0512203AE9600302A6825D
:10A510007A007B02900599E0F9122004EA4B4C4D39
:10A52000600302A68290054F120B7C851882851964
:10A5300083120B70900555E0C0E07404120BC3D079
:10A54000E0F07405120BC37401F07406120BC374AF
:10A550000212D03B1229E8E9600302A67FEEFAEF6F
:10A56000FB12132002A6829004D512D004702C7521
:10A57000080078081209117808120911EE2410F564
:10A5800082E43FF58312CFF8A3A3A3A3A312BA3D9D
:10A5900012CD0512120C74021208CF8E828F831214
:10A5A000BB4E7407120BC3E8F0A3E912A9D412BB87
:10A5B0004E7409120BC312BA4F12BFD4C0E0740B11
:10A5C000120BC3D0E0F012CCDF128768740F78084A
:10A5D000120B45740C120BC3E508F07420120BC368
:10A5E000E0C0E0740D120BC3D0E0F07422120BC374
:10A5F000E0C0E0740E120BC3D0E0F0741D120BC368
:10A60000E0C0E07410120BC3D0E0F0741E120BC354
:10A61000E0C0E0740F120BC3D0E0F0EE241012B9CA
:10A62000E5C0E07411120BC3D0E0F07421120BC32B
:10A63000E0C0E07412120BC3D0E0F0742E120BC312
:10A64000E0C0E07413120BC3D0E0F07423120BC30C
:10A65000A982AA8389088A09750A0078081209095B
:10A660007C087D007417120BC3AA82AB83121E6094
:10A6700074031208CF740712095B120C36800312A0
:10A6800029E2742F02B6D6E0FA8E828F83A3A3222A
:10A69000A3E0F98A828B832212D21564012274F717
:10A6A00012039E74C912099912133E90054EE0647C
:10A6B00008601F9030FDE493900530F09030FDE489
:10A6C0009390052EF0900557740112A813A304125D
:10A6D000A8137C237D007900741412095B121E728A
:10A6E00090055FE07009741E120BC374018006743C
:10A6F0001E120BC3E412A824740FF0901DE112D0B7
:10A700003B79461228267401120BC3E4F0901E5BBD
:10A71000E0C0E07402120BC3D0E0F090053CE0C052
:10A72000E07403120BC3D0E0F07404120BC3E4F026
:10A730007405120BC3E4F07407120BC3E4F0900528
:10A740005FE0C3940F500CE0C0E07406120BC3D05E
:10A75000E080077406120BC3740FF07C607D0574F3
:10A7600008120BC3AA82AB831220407C037D0079C0
:10A77000FF7410120BC3AA82AB83121E729005984D
:10A78000E0C0E07413120BC3D0E012CC4574011288
:10A79000095B1211227A9C7B057945122826121238
:10A7A0003C900553E0C0E0741C120BC3D0E0F09065
:10A7B0000554E0C0E0741D120BC3D0E0F0900541D9
:10A7C000E0C0E0741A120BC3D0E01287BE741812F6
:10A7D0000BC312CD147420120BC3E4F0900556E0A5
:10A7E000C0E0741F120BC3D0E0F07434120BC3E44A
:10A7F000F07429120BC3E412A81C1228267A427B9B
:10A8000005794B122826741412095B1228447437F8
:10A8100002B421F0A3E4F0A3F0A3F022F07A3F7B8E
:10A820000579532212A82822F085188285198322DF
:10A83000C082C0838A828B83A3E090054E6004E4CB
:10A84000F080707408F090055FE070289004E212C8
:10A85000D0046008790012C92612052990054C120F
:10A86000BA207A057B00121E3C90054C12CD0512D1
:10A87000138C80187900120C3090053F12BA207AA0
:10A88000067B00121E3C12A8B6121E3C9005D21286
:10A89000D004601F901CB9E06401701790812A12E7
:10A8A000070D7A007B40900599E0F9121FF87404B7
:10A8B0001208CF02C5F190054212BA247A047B0037
:10A8C0002274F412039E74EA1209998A088B09EA29
:10A8D0002402FAE43509FB12298E8A0A8B0BAE0A90
:10A8E000AF0BEE4F700302A9C58E828F83A3A3A383
:10A8F000A3E06401602A8E828F83A3A3A3A3E064F4
:10A9000002601D8E828F83A3A3A3A3E06403601063
:10A910008E828F83A3A3A3A3E06404600302A9C56E
:10A92000E5082402FCE43509FD740B120BC3AA826E
:10A93000AB8312204012A9CA120BC312CD14741596
:10A94000120BC37401F07408120BC3E412D03B1253
:10A950002838E9FC7D007A077B00121E3C8E828F2E
:10A9600083A3A3A3A3A3E0C2E012A9D4740112E9B4
:10A97000E85001097A027B0012024EE88E828F8332
:10A98000A3A3A3A3A3A3A3A3F0901CB9E0640170A5
:10A9900034901CB3E06402702C8E828F83A3A3A337
:10A9A000A3E06401600D8E828F83A3A3A3A3E06460
:10A9B00002701212B9D9120B7C12C2C8120B70EEBF
:10A9C000241B12CFEB7416028FF28E828F8312D566
:10A9D000B774132212A9D82212C2FEA3A3A3A322E2
:10A9E00074F212039E74F8120999EAFEEBFF8C0AC6
:10A9F0008D0B890D9080F3AC18AD197408120833D3
:10AA0000750C00EEFCEFFDAA18AB1912203AE970A4
:10AA100003750C0190059A801AEEFCEFFDE5082401
:10AA20000BFAE43509FB12203AE97023E5082414F7
:10AA300012CCF112AA656024E50CA2E040DB850887
:10AA400082850983E0650A7004A3E0650B70DD85EB
:10AA50000882850983A3A3E0650D70D0AA08AB091D
:10AA60007408028B6412876CE508450922C082C015
:10AA70008390059A02C5EE74F712039E90059A1210
:10AA8000F16E800C12D81D12BCDC121F32EEFAEFF0
:10AA9000FBEA4B70EF90059AE4F0A3F002B4247443
:10AAA000F412039EEAFEEBFFEE241312B9E56403F1
:10AAB000700CEE240BFAE43FFB12298E800EE0644A
:10AAC00002707C12CCDF12CD051229948A088B0902
:10AAD000E508450960698E828F83A3E0700F8508C1
:10AAE00082850983A3A3A3A3A3A3E4805164F16097
:10AAF0000A8E828F83A3E064E1702785088285092E
:10AB000083A3A3A3A3A3A3E0640170168508828591
:10AB1000098312CD05120D0EEE240BFAE43FFB1251
:10AB20002982850882850983A3A3A3A3A3A3E06048
:10AB30000E850882850983A3A3A3A3A3A314F0020F
:10AB40008FF574F112039E8A088B09ECFEEDFF89E4
:10AB50000A8A828B8312DC588A828B8312A1E012CC
:10AB6000AC148A828B83A3A3E0C454F0FA88828950
:10AB700083E04A12AC2412A1E012AC1EE03333543D
:10AB8000FCF88E828F83E04812AC1EA3E03333338F
:10AB900054F8F88E828F83E04812AC148508828BBB
:10ABA00083A3A3A3A3A3A3E0A2E0E4331313FA882F
:10ABB000828983E04AF0E5082407F50CE43509F5BD
:10ABC0000D750E00780C1209097C087D00EEFAEF75
:10ABD000FB121E6074031208CFEE2408FE50010F12
:10ABE000E508240FF50CE43509F50D780C12090978
:10ABF0007C037D00EEFAEFFB121E6074031208CF97
:10AC0000E50AC3940F400A12CCED12A1E1A3A3A35D
:10AC1000F002E9BAF0EEF8EFF9A30EAF832212AC1E
:10AC200024A3A322F08508828B83A3A32274F112AC
:10AC3000039EEAFEEBFF890A8C088D098E828F83C2
:10AC4000E08C828D8312C005AE82AF83E012C3B464
:10AC500012C59EC412C3B412ACECE012C3BB12C541
:10AC60009CA2E2E4338C828D8312C59B1313135490
:10AC70001F12C3B412C59AA2E7E4338C828D83A35A
:10AC8000A3A3A312ACEC8E0C8F0D750E00780C12E2
:10AC900009097C087D00E5082407FAE43509FB1260
:10ACA0001E6074031208CFEE2408FE50010F8E0CB4
:10ACB0008F0D780C1209097C037D00E508240FFA3A
:10ACC000E43509FB121E6074031208CFE50AC39431
:10ACD0000F40118E828F83A3A3A3E0C0E012CCEDBE
:10ACE000D0E0800412CCEDE4F002E9BAA3A312C0D4
:10ACF000090EAF832274F512039E8A088B098A829B
:10AD00008B83A3AE82AF83E0F9120C5A8E828F83BD
:10AD1000E064EB6024850882850983A3E064E16038
:10AD200018850882850983A3E064F1600C85088298
:10AD3000850983A3E0641A7009850882850983A3C5
:10AD4000E4F0901E42120BAC1210AA750A01780AA8
:10AD5000120911850882850983A3E0F50878081295
:10AD60000911790090054C12AD7B12CD0512120C21
:10AD700074021208CF12114002B6D912BA249005FB
:10AD80004222C082C083E99005AC7003E480027463
:10AD900001801EE0F902C5F1C082C0837C987D105D
:10ADA0008A828B8312CD0512285002C5F1EAF0A3E6
:10ADB000EBF002C5F174F612039E9005ACE0701B37
:10ADC0007C0079017A007B00121170EA4B600C8ADA
:10ADD000828B8312D004600312109E02C983C0824A
:10ADE000C083790412116AE9F8903116E493C3988C
:10ADF000401079FF12116AE9F8903115E493C39875
:10AE0000500479018002790002C5F174F012039EAA
:10AE10008A088B09890B750C008A828B83A3A3A3F4
:10AE2000A3A3A3A3A3E0F91211768A0E8B0FAE0E93
:10AE3000AF0F750A01EE4F600302AEF685088285FA
:10AE4000098312B034A3A3A3A3A3A312C0C212CD3B
:10AE50000512115E8A0C8B0DAE0CAF0DEE4F700318
:10AE600002B01F8E828F83A3A3A3A3E4F0A3F0E517
:10AE700008240CFAE43509FB8A828B83E0C0E012D7
:10AE8000E9DED0E0F0E508240D12B02C12DC261229
:10AE9000CD1412129CEE240F12E1D0E508241112F9
:10AEA000B02C12894612CD14E508241312B027C025
:10AEB000E012B9D9D0E0F0750C01EE240612BFBA49
:10AEC000E0547FF0A3E054FC12E716E05404600362
:10AED00002AF6D901E54E0F50875090074077808FC
:10AEE000120A9C8E828F83A3A3A3A3A3A3E0450889
:10AEF000F0A3E04509F08E828F83A3A3A3A312875A
:10AF00006674077808120B45E5085407FCE50B60EA
:10AF10006C8E828F83A3A3A3A3A3A3A3A3A3740272
:10AF200012C59F12B2FB600B90053A12B045A3A365
:10AF300012CD14EC700302AFE8EE240612F4BC54F8
:10AF40007FF508A3E054FCF509EC24FFF50EE4348A
:10AF5000FFF50F7407780E120A9CE508450EF8E518
:10AF600009450FF98A828B8312CD14807B8E828FE4
:10AF700083A3A3A3A3A3A3E0448002AEF5EC7005D2
:10AF8000750A0080638E828F83A3A3A3A3A3A3E08B
:10AF90005420600C121E84EA547F7900245F8019CB
:10AFA0008E828F83A3A3A3A3A3A3E05410601A12DD
:10AFB0001E84EA540F7900240A5001098E828F837F
:10AFC000A3A3A3A3F0A3E9800D8E828F83A3A3A3E1
:10AFD000A37401F0A3E412A9D47404F07A207B00D6
:10AFE000900599E0F9121ECCE50CA2E0503412BA9B
:10AFF00039A3A3A3A3A3A3A3A3A3E0F9EEFAEFFBB2
:10B00000121164E9601C12EDC43F12D002600912F3
:10B01000B59712CD05121F32EEFAEFFB121F3275F3
:10B020000A00A90A02D9A812BFE2E02212BFE21266
:10B03000D5B7EE22A3A3A3A3A3A312BA24850882A3
:10B04000850983A32212D5B78E828F83A3A322748E
:10B05000F412039E74F71209997E00121176EA4BDE
:10B06000700302B10B8A828B83A3A3A3A3A3A3A320
:10B07000A3A3E06406600302B10B8A828B83A3A3BF
:10B08000A3A3A3A3A3E0FF8A828B8312B112E0C023
:10B09000E07408120BC3D0E012B53912CD0A1211B8
:10B0A00094EF5408606385188285198312BA207A58
:10B0B000007B001211588B0BEA450B704C12F616F0
:10B0C0001228687C007D007A007B0080288E828FA9
:10B0D0008312B528F47003A3E0F4602D90054C12A0
:10B0E000BA4112CD05122862E9641A601C7C007D09
:10B0F00000EEFAEFFB1211588A0A8B0BAE0AAF0B67
:10B10000EE4F70C9790012286E7E01EEF9740902C3
:10B110008FF212BCE512B119222408F582E438F549
:10B120008322C082C083EA4B70059005B180068AF5
:10B13000828B83A3A312B32F60258A828B83A3A360
:10B14000A3A3A3A3A3E0540860E5EC4D60158A8295
:10B150008B8312B5286C7003A3E06D70D280047AE3
:10B16000007B0002C5F174F212039EEAFEEBFF8938
:10B170000A8C088D097A147B00121F2CEA4B603F61
:10B180008A828B83A3A3A3A3A3A3A3A3A3E412B53F
:10B190002EA3E50A12B1CBA3A312DD938A828B837F
:10B1A000A3A3A3A3E4F0A312B54C12B1DD12E16E88
:10B1B000EA12EDC53BF583E4F012B1C2F0A3F00250
:10B1C0008B67A3F08A828B83A3A32212B1CF2212B2
:10B1D000B1D322F08A828B83A3A3A3A322A3F0126C
:10B1E000F4DD3BF583E4F02274F412039EEAFEEBF7
:10B1F000FF89088C0A8D0BEE4F700302B284740134
:10B2000065087012790112116AE9F890310CE49323
:10B21000C3985022801674046508701479041211C2
:10B220006AE9F8903116E493C398500A7911805670
:10B2300074026508704E8E828F83A3A3A3A3A3A379
:10B24000A3A3A3E50812BA4912DC33E4F0A3F090FB
:10B2500005B112D00460178003E0F8A312CE0BA34F
:10B26000A312B32F88828983A3A370ED8003900576
:10B27000B112E1727A207B00900599E0F9121ECCA0
:10B280007900800279C1028FF5C082C083E9F87924
:10B29000009005B1801D8A828B83A3A3A3A3A3A3DF
:10B2A000A3A3A3E068600574FF687001098A828B1C
:10B2B00083A3A312B32F70DE02C5F174F712039EAD
:10B2C000EA4B70059005B180068A828B83A3A31296
:10B2D000B32F60208A828B83A3A3A3A3A3A3A3A3DA
:10B2E000A3E06970E4EC60108A828B83E012B2FB09
:10B2F00070D780047A007B0002B42412F512E05467
:10B300000422C082C0839005B180068A828B83A309
:10B31000A312B32F60128A828B83A3A3A3A3A3A338
:10B32000A3A3E06970E580047A007B0002C5F112F6
:10B33000D239EA4B2274F712039EEAFCEBFD90052A
:10B34000B180068A828B83A3A312B32F60248A82E2
:10B350008B8312B5286C7003A3E06D70E68A828B34
:10B3600083A3E0C812BCD212D994A2E0E43370D314
:10B3700080047A007B0002B42474F212039E8A0ACD
:10B380008B0B8C0C8D0D750800750900EA450B6060
:10B39000309005B180068E828F83A3A312BCDCEEB1
:10B3A0004F601EAC0CAD0DEEFAEFFB850A82850BEB
:10B3B00083120529E9640170DDEEF8EFF988088948
:10B3C00009AA08AB09028B6779000208B774F71263
:10B3D000039E9005B112BB4E7C007D00800DE8FC01
:10B3E000E9FD88828983A3A312BB4EE8496030EA55
:10B3F000687002EB6970E79005B112CD05E86A70DC
:10B4000002E96B88828983A3A3700812BB4E900562
:10B41000B1800912BB4E8C828D83A3A312CD148000
:10B42000031208CF7F0102060F74F712039EEAFE93
:10B43000EBFFEE4F602F12118E12B46712CD051282
:10B440001F328E828F8312CD05121F3212EDC43F40
:10B4500012D002600912B59712CD05121F32EEFA12
:10B46000EFFB121F3280BD12D00AF5832274F61250
:10B47000039E8A828B8312B528F508A3E0F5099014
:10B4800005B112BB4E7D007C00802F88828983A38A
:10B49000A3A3A3A3A3A3A3A3E0640570140C12DCCD
:10B4A0004FF5838E82E065087004A3E065097001A2
:10B4B0000D88828983A3A312BB4EE84970CD9031D9
:10B4C00013E493F8EDC398500890311212EF4C40FA
:10B4D0000F8A828B83A3A3A3A37401F0A3E480103B
:10B4E00090053AE0F812A690A3A3A3A3E8F0A3E97D
:10B4F00012B54C740512B52EE0440812B539F4703B
:10B5000003A3E0F4601190054C12D97712CD051217
:10B510002862E9641A7005790112286E02C983EE67
:10B52000241DF582E43FF583E0F812B5442212B5FC
:10B53000322212B1D3A3A3A322F08A828B8312B545
:10B540004222E0F8A3E0F5838882E02212B532A31C
:10B55000A32274F612039E9005B112BCDC802A125D
:10B56000876212B46712CD05121F328E828F83124A
:10B57000CD05121F3212B59712CD05121F32EEFA09
:10B58000EFFB121F32AE08AF09EE4F70D29005B13B
:10B59000E4F0A3F002C983EE12CDF022C082C08392
:10B5A000EAFCEBFDEC4D6017EC24FBF582ED34FF7B
:10B5B00012D002700712B5F6E0F46007121E9079FF
:10B5C000058030900599E0C0E012B5F6D0E0F0902B
:10B5D0003106E493F97AB37B05121EC6E964017063
:10B5E000107A007B20900599E0F9121ECC7900803A
:10B5F00002790402C5F1EC24FFF582ED34FFF583F6
:10B600002274F412039EA2AFE433F508C2AF900592
:10B61000B312BCDCEE4F603AEE24FBF582EF34FF50
:10B6200012D0027A007B209005996007E0F9121E83
:10B63000CC8005E0F9121ED2E4F50AF50B780A1267
:10B64000090DEEFCEFFD7AB37B05121EC0740212E9
:10B6500008CFE508A2E092AFEEFAEFFB028FF57497
:10B66000F512039E8A088B09750A009005B112DC59
:10B6700053805A8E828F8312B52865087004A3E028
:10B680006509703D8E828F83A3A3A3A3E4F0A31268
:10B69000C30F540460118E828F83A3A3A3A3A3A31B
:10B6A000A3A3E0F9120D808E828F83A3A3A3A3A38B
:10B6B000A3A3A3A37406F07AF01289531210A40571
:10B6C0000A8E828F83A3A312BB4EE8FEE9FFEE4FE2
:10B6D00070A1A90A80031208CF7F0302060F74F03D
:10B6E00012039E74D4120999EAFEEBFF750B0075E4
:10B6F0000A007508FE7509FF121146E9600302B9D8
:10B70000CCEE241512B9E56044901E71E0C43354A8
:10B71000E0F8E0333354FC48C0E012D7A6D0E01282
:10B72000BA4912CD0579FF120E828B0DEA450D60E4
:10B730000F750B017508FF12CFEF12CEC5D2E0F0E6
:10B74000901CC5E0600464017003750A408E828F0E
:10B750008312CD03121290E9600312B9F1EE2413A3
:10B7600012B9E5700D903105E493C0E012B9D9D05B
:10B77000E0F08E828F83E0A2E7500454038019EE3C
:10B78000241412B9E5701290052BE0C0E012F4B257
:10B79000D0E0F090052BE004F012F4CE7016901E6D
:10B7A0005DE0600D900536E0700A8E828F83E07058
:10B7B0000312CDE0901CC5E060046401704B90055D
:10B7C00039E0A2E15043E50BA2E040218E828F8355
:10B7D00012CD03121290E960308E828F83E0600DEB
:10B7E000EE240B12B522F912126CE9601C12B9FD9D
:10B7F000700302B97EEE241312B9E56401600302FE
:10B80000B97E12B597E054FBF08E828F83E064011D
:10B81000700DEE240B12B5226402700312BA0A12E4
:10B82000B9FD600302B8E4E50BA2E0500302B8E4FE
:10B83000901CC5E060076401600302B8E49005391C
:10B84000E0A2E1400302B8E4E50AF50B780B120927
:10B8500011EE2406FCE43FFD8E828F8312CD03EEB1
:10B860002412129C00120DAA74011208CFE960067E
:10B8700012B9F112BA038E828F83A3A3A3A3A3A349
:10B88000E0603CEE2402F50CE43FF50D850C8212DD
:10B89000BA2E2407FAE43FFB1211D08A088B0985DF
:10B8A0000C82850D83E065087004A3E06509700CC7
:10B8B0008E828F83A3A3A3A3A3A3E4F012BA0A8E5C
:10B8C000828F83E06401600BA90A12BA3D12CD0396
:10B8D000120D4AA90A12BA3912CD03120CD8E96026
:10B8E0000312BA03AC18AD19EEFAEFFB1211CA8AB3
:10B8F0000A8B0B74FE6508700474FF6509700312EF
:10B900008762EA450B700302B9D08E828F83E0C054
:10B91000E07401120BC3D0E0F07404120BC312E107
:10B9200072EE241E12BB487402120BC312CD1474A3
:10B9300001120953880C890D780C12090DEE242090
:10B9400012B9E912091112B597120711EE240E125D
:10B95000B9E912091190053F1207117408120BC3BF
:10B96000E0F9AC08AD091211C474081208CFE9FE61
:10B9700074106E705DAA0AAB0B121F328054EE2455
:10B980001312B9E5C0E07417120BC3D0E012F5230F
:10B99000740F120BC312BA4F240412F4C112BB4E1F
:10B9A0007411120BC3E8F0A3E912C02AC0E07418A6
:10B9B000120BC3D0E012E9D412A69112BA20740679
:10B9C00012095B120D7AE9600302B809791180044B
:10B9D0007E10EEF9742C02D9A512B9DD22EE12CE3A
:10B9E0002822EE241712BFCA2212BFCAF50C780C07
:10B9F00022EE2412F582E43FF583E4F02212BA111C
:10BA000054402212BA114420F02212BA114440F0DC
:10BA100022EE12CDF4E022EE2413F582E43FF5830A
:10BA200012BA242212BA2822E0FCA3E0FD22F583F8
:10BA300012BA342212BA28EE228E828F83A3A3A3D5
:10BA4000A312BA248E828F832212DC3F22A3A3E8A2
:10BA5000F0A3E9F0EE22C082C08374D71209999056
:10BA60008030740312096374261208338A828B8330
:10BA7000A3A3A3A312BB4E740E120BC3E8F0A3E959
:10BA800012D5B0740C120BC312BB52240D12BB3D65
:10BA9000C0E0741A120BC3D0E0F012D82712BB4CCE
:10BAA0007420120BC312BB52241512BB3DC0E074AC
:10BAB00008120BC3D0E0F0EA241CF582E43B12BB71
:10BAC0004C7412120BC312BB52241112BB3DC0E0C6
:10BAD0007409120BC3D0E0F0EA241212BB3DC0E09F
:10BAE0007407120BC3D0E0F0EA241EF582E43B1287
:10BAF000BB4C7424120BC312BB52242012BB3DC09A
:10BB0000E07426120BC3D0E012A82474FFF0740175
:10BB1000120BC374FFF07402120BC374FFF0908118
:10BB20004212070D7404120963740712095B120CA8
:10BB30001E74041208CF7900742902D5F4F582E44A
:10BB40003BF583E022EE2413F582E43FF58312D522
:10BB5000B722E8F0A3E9F0EA2274EE12039E74EC37
:10BB60001209998A0E8B0F8C088D09890C750A10A1
:10BB70007A217B00121F2C12D5FAE849700302BC0F
:10BB8000CB750B007C217D00790085188285198397
:10BB9000E0FA121E727429120BC312BCDC901CC591
:10BBA000E060046401703EAA08AB091229948A106F
:10BBB0008B11A810A911E849602388828983A3A367
:10BBC000A3A3E06401600D88828983A3A3A3A3E0FB
:10BBD00064037009EE5440700474044FFFEF540482
:10BBE0006003750B0190054C12CD058518828519EF
:10BBF0008312BCE12409F582E43812E1D4742612E0
:10BC00000BC312BB4E7411120BC3E8F0A3E912BCB4
:10BC1000EA12F4D412BCEA12B119740212F52EF829
:10BC2000A312C92612DEFD12BCEA12F4E4E50CF000
:10BC30007428120BC3E0F50885188285198312F465
:10BC4000EDE50812BCEA12BCD2F583E50EF0A3E5DF
:10BC50000FF07406120BC312E1727408120BC3E5E5
:10BC600008F0742C120BC312E36AC082C083740CF8
:10BC7000120BC3AC82AD83D083D08274051208331B
:10BC8000742B120BC3E0C0E07413120BC3D0E0F0AE
:10BC9000A90BAA18AB1912114CE964017021901C70
:10BCA000C5E0600464017012E50BA2E0500CA90825
:10BCB000121176EA4B600312119A750A00800C8506
:10BCC000188285198312CD05121F32A90A74140235
:10BCD000C315241FF582E43822A3A3A312DC53FF6B
:10BCE0002212BCE52212D614C82212D609C8227428
:10BCF000EE12039EEAFEEBFF8C088D098E828F8385
:10BD0000A37408F0EE241612B9E560088E828F83C2
:10BD1000A37410F012B9E260098E828F83A3E0242D
:10BD200008F0EE241512B9E560088E828F83A3E037
:10BD300004F08E828F83A3A3A3A3A3A3E060198E34
:10BD4000828F83A3A3A3A3A3A3A3E0C3332402F8F6
:10BD50008E828F83A3E028F012BFC36005750B0E9F
:10BD60008003750B00901CC5E06402701E901CB926
:10BD7000E0640170168E828F83E06401600D901C78
:10BD8000B3E0600712BFB07401800412BFB0E412C8
:10BD9000C005E012BFD228250B8C828D83F012BF24
:10BDA000C36013900537E0F912106EE9F885088238
:10BDB000850983E029F0850882850983E0C39475AD
:10BDC000400975080075090002BFA9E0FA7B00125E
:10BDD0001F2C8A088B09EA4509700302BFA98E82CD
:10BDE0008F83E0FA90053C12BFFE7402780C120AB1
:10BDF0009CEA450CFAAB0DEE241212B9E55403F59A
:10BE00000C750D007406780C120A9CEA450CFCEBCC
:10BE1000FDEE241512B9E56004780180027800EE89
:10BE20002416FAE43FFBE8F9ED49FD12BFC3F50C17
:10BE30007409780C120A9CED450DFD8A828B8312E1
:10BE4000BFFE740B780C120A9CED450DFDEE241715
:10BE500012BFF8740C780C120A9CED450DFD8E8211
:10BE60008F83A3A3A3A3A3A312BFFE740A780C120B
:10BE70000A9CED450DFDEE242312BFF8740D780CDD
:10BE8000120A9CECF8ED450DF9E8850882850983D6
:10BE9000F0E9A3F0EE240212BFBA12C0CC12C02007
:10BEA000F0EE240412BFBA12BFEA12C020A3A312FC
:10BEB000CE1E12BFEAA3A3A3A312C02A85088285BF
:10BEC0000983A3A3A3A3A3A3A3F0750A088A828B63
:10BED00083E06015EE241812BA1AE5082408FAE483
:10BEE0003509FB122040750A1012B9E26019EE24E0
:10BEF0001A12BA1AA80AE50828FAE43509FB122032
:10BF0000407408250AF50A8E828F83A3A3A3A3A3F6
:10BF1000A3E06057EE2407F510E43FF51185108289
:10BF2000F583E0C0E012BFD9D0E012C010E0C0E05D
:10BF30000812BFDBD0E012C010129B4D1209098518
:10BF40001082851183E025E0FCE433FDA80AE508B2
:10BF500028FAE43509FB121E6074031208CF85101D
:10BF600082851183E0C333250AF50AEE241512B940
:10BF7000E56008C0E012BFD9D0E0F012CCDF129B20
:10BF80004E12090912BFD3FC7D00A80B8E828F834D
:10BF9000A3E0FAE5082AFAE43509FBEA28FAE43BCB
:10BFA000FB121E6074031208CFAA08AB0902C31863
:10BFB000EE2423F582E43FF58322F8E43FF98882FA
:10BFC00089832212BFC722EE2411F582E43FF58354
:10BFD000E022F8EE12DC2AE022A80AE5082812BFC7
:10BFE000E222F582E43509F5832212BFEE22E085D4
:10BFF0000882850983A3A322F582E43FF583E0F557
:10C000000C750D002212C00922F08E828F83A322AC
:10C01000F0050A8E828F83A3A3A3A3A3A3A3A322C5
:10C02000A3A312E72612BFEEA322F0EE241412BF40
:10C03000CA2274F412039E74FD1209998A088B09AE
:10C04000ECFEEDFF7401120953880A890B780A127D
:10C05000090D7402120963EEFAEFFB120D26740249
:10C060001208CFE9705385188285198312C0CCF06D
:10C070007401120BC3E0F812C0C2A3A312F52A6028
:10C080002914850882850983A312F52E12DAAE746D
:10C0900001120BC3E028F8A3E039F9E824FEF58289
:10C0A000E934FFF58312F16E800C850882850983DF
:10C0B000A3E4F0EEFAEFFB80047AFE7BFF74030248
:10C0C0008FF2A3E0F985088285098322E085088242
:10C0D0008509832274EE12039E8A0A8B0B8910EC69
:10C0E000FEEDFF750F017C267D007900EEFAEFFB77
:10C0F000121E72E510C39408500302C2618E828F33
:10C1000083E510F0EEFCEFFD850A82850B8312C5F6
:10C110006C1211DCE96003750F0012C54E8E828F20
:10C120008312C5A6EE12C5423F12C590C0E0128927
:10C1300045D0E012C588C0E0EE2412F582E43FF558
:10C1400083D0E012C005740812C2F6A3A3E0601801
:10C15000E50A2408F8E4350BF912B9D912CD148E8A
:10C16000828F83A3E02408F08E828F83A3A3A3A3EE
:10C17000A3A3A3A3E060178E828F83A38582088583
:10C18000830912C56112D7A612A3402408F0EE2439
:10C190001912B9F4EE241B12B9F4A312C2F6E0602E
:10C1A0000F12C2DD8E828F83A3A3A3A3A312C309A0
:10C1B000EE241812B9E5700302C25112C2DDFAEE84
:10C1C0002419F582E43FF583EA12C309F8E50A2849
:10C1D000F582E412F610F812DD67E812C309E8C32D
:10C1E0009AEE5068241912B9E5F8903108E493C327
:10C1F00098500575110C8008EE241912B9E5F51157
:10C200008E828F83A3E0F8E50A28F50CE4350BF560
:10C210000D750E00780C120909AC11EC2CFCE433FE
:10C22000FD7A1A7B11121E6074031208CFEE241BD4
:10C23000F582E43FF583741AF0A37411F0E511C39D
:10C2400033F8850882850983E028800412CDD7E47D
:10C25000F08E828F83A3E0F88E828F83E0C39850A4
:10C260000479008061A3E0FAE50A28F8E4350B12AE
:10C27000C2D2E8F0A3E912C59FC39AC0E012C2C8B7
:10C28000D0E012C30F603DEE2417F8E43FF98808B0
:10C2900089098882F583E024F2F0EE241D12BFBAEA
:10C2A000E0240EFAA3E03400FB8882898312E1D6F1
:10C2B000900537E0F912106EE9F885088285098348
:10C2C000E0C398F0A90F8050EE2417F582E43FF503
:10C2D0008322F9EE241DF582E43FF583228E828FBE
:10C2E00083A3858208858309E0F8E50A28F582E4BE
:10C2F000350BF583E02212C2FA2212C2FE22F08E22
:10C30000828F83A3A3A3A3A32212A34804F0221223
:10C31000C2FAA3E0221208CF7F0A02060F74F412B9
:10C32000039E8A088B09EA12C3BBA3A3F0EA131386
:10C33000543F12C3B4A3A3A3F0EAC4131312C3BBA4
:10C3400012C3CE7409780A120B4512C3C2A3A3A369
:10C35000A3A3A3F0EB12C3C412C3CD740A780A12CC
:10C360000B45E50A5401C0E0EC2418F582E43DF5E4
:10C3700083D0E012C3D2740B780A120B4512C3C2E9
:10C3800012C3CB740C780A120B4512C3C2A312C39A
:10C39000CB740D780A120B45E50A5401C0E0EC2479
:10C3A00024F582E43DF583D0E0F0740E7808120B9A
:10C3B00045028940540F8C828D832254038C828DD8
:10C3C0008322E50A54018C828D8322A3A3A3A3A315
:10C3D000A3A3F08A0A8B0B22C082C08379008A82D1
:10C3E0008B83A3A3A3A3A3A3E0900536600EE07004
:10C3F000238A828B83A3A3E0701A8016E060158ADB
:10C40000828B8312CCFC90053FE06A7003A3E06B43
:10C410006002790102C5F174F212039E8A0A8B0B45
:10C42000890C8C088D098A828B8312C56C1211DCF1
:10C4300012C54E85088285098312C5A6E50812C576
:10C4400042350912C590C0E0E508241112CCF1D0A4
:10C45000E012C588C0E012CCEDD0E012D01874080C
:10C4600012C57AE06017E50A2408F8E4350BF9E50F
:10C4700008241312C54612D018E02408F08508825B
:10C48000850983A3A3A3A3A3A3A3A3E0601785089F
:10C4900082850983A312C55DE508241512C54612DD
:10C4A000C59F2408F0850882850983A3A3A3A3A3BD
:10C4B000E06019850882850983A3AE82AF8312C22A
:10C4C000E885088285098312C59A04F0AA08AB0999
:10C4D0001211E2E9F50D7064850882850983A3A332
:10C4E000A3A3A3A312C0CCA3701AE0FAE50A2AF80A
:10C4F000E4350BF9E508241D12CCF112CD14E50C3E
:10C50000C39A802C12C55DE8240EF8500109E50895
:10C51000241D12CCF112CD14900537E0F912106EE3
:10C52000E9F88E828F83E0F9E50CC39924F2C39871
:10C53000C0E0E508241712CCF1D0E0F0A90D028B81
:10C5400067EA12F4DE2212BFE2E8F0A3E922850ACC
:10C5500082850B83A3A312C5BCE0F9EA22AE82AFA9
:10C5600083E0F8E50A28F8E4350BF922E0FAA3E0C5
:10C57000F8E4C8F9EA28E439FB2212C57E2212D079
:10C5800020A3A3A3A3A3A32212C5CFA3A3A3E02206
:10C59000F583E812C5C8A3A3E022A3A3A3A3A3F035
:10C5A0008E828F83E022A3A3A3A3A3A3A3A3A3129A
:10C5B000C5C812C5BCA3A3E0F9EAF822E0FA850ACF
:10C5C00082850B83A3A3A322F0A3E912C5CF22F097
:10C5D000850A82850B83A3A3A3A322C082C0837A8A
:10C5E000C17B0579E21228207AC17B05800312CD38
:10C5F00005D083D0820208B7C082C08390053F80F7
:10C60000EDC082C08390054280E4C082C083794A35
:10C6100012282080DC74F612039E9005C9E0FE0407
:10C62000F0EEF91211768B09EA450970EDEE60EA39
:10C63000F902C98374EE12039EEAFEEBFF8C0E8DA5
:10C640000F890C750A00750B001213928A088B096A
:10C650007412120BC3E0F50D7413120BC3E0F51046
:10C66000EA45097017E510600302C756A90CAC0E25
:10C67000AD0FEEFAEFFB1213B602C855E5107003CA
:10C6800002C721901CC5E060046401700E9005CEC5
:10C6900012D004600612C926120529E50D700E8518
:10C6A0000882850983E4F0750B0102C779901CC5E7
:10C6B000E060076401600302C779900539E0A2E1F8
:10C6C000400302C7799005D012D004600CA90DAACE
:10C6D00008AB0912C926120529850882850983E05D
:10C6E000FA12E9C9500109C3EA98E499A2D265D0C7
:10C6F000335009850882850983E004F08508828526
:10C700000983E0F8903102E49368706D750A01EED8
:10C71000FAEFFB120DB6850882850983A3E4F08049
:10C7200058E50D701CEA240212B027A80C28F8E482
:10C73000340013E813F070098A828B83A3A3740179
:10C74000F08A828B83A3A3E0F8901E29E0C398505F
:10C7500052750B01804D74016510701DE50D601957
:10C76000901CC5E060046401700F900539E0A2E1FF
:10C770005007EEFAEFFB120DB6901CC5E064027094
:10C780002274016510701CE50D9005E06013E00453
:10C79000F0901E55E0F89005E0E0C3984005750A5A
:10C7A00001E4F0E50BA2E092F0E50AA2E072F040AD
:10C7B0000302C855901CC5E06004640170419005F7
:10C7C00039E0A2E15039EEFAEFFB1229948A088B86
:10C7D00009A808A909E8496026E50BA2E0500D88E0
:10C7E000828983A3A3A3A3A3E0C2E0F0E50AA2E0A9
:10C7F000506388828983A3A3A3A3A3E0D2E0F0E5DA
:10C800000AA2E05050901CC5E060046401701D90C5
:10C810000539E0A2E15015EEFAEFFB1229A6E96016
:10C820000BEEFAEFFB7900120C548029900542E0E0
:10C830006E7003A3E06F701DEEFAEFFB7901120C2E
:10C8400054901CC5E06402700C7A017B009005993D
:10C85000E0F9121FFE02C31874F412039E8A088BBB
:10C86000098C0A8D0B90817678081209AF700E7AC8
:10C87000017B00900599E0F9121ECC8035901E4294
:10C880007808120B36EA4509450A450B6018780806
:10C890001209057A017B00900599E0F9121FF274E4
:10C8A000041208CF800C7A017B00900599E0F91200
:10C8B0001FFE028FF5C082C083901E4602ADADC040
:10C8C00082C083901E4802ADAD74F612039E7508B7
:10C8D0002B750905780812090D7C6E7D007A217B85
:10C8E00000121FA474021208CFE9F508122A00E909
:10C8F0004208901CC5E060046401700612294CE9EE
:10C90000420890070412D004600912C926120529B2
:10C91000E94208120EA6E9FE122790E9F8E5084E52
:10C9200048F9805F79C4E0F58388822274F61203A7
:10C930009E121E3675082B750905780812090D75AB
:10C94000086E750900780812090D7C007D007A21B7
:10C950007B00121FB074041208CF1229FA901CC574
:10C96000E060046401700312294690070612D004A7
:10C97000600612C926120529120EAC1227A28003E6
:10C980001208CF7F0202060F74F612039E74FF1284
:10C9900009997E0075082B750905780812090D7C28
:10C9A0006E7D007A217B00121FA474021208CFE969
:10C9B000600302CA6D780812090D75086E8E097839
:10C9C0000812090D7C007D007A217B00121FB674CD
:10C9D000041208CFE9600302CA6D90053FE064FECF
:10C9E0007003A3E0F4700302CA6D7E0190054EE06F
:10C9F00064086005E06404706F851882851983EE11
:10CA000012D03B79421228267A567B0579431228A8
:10CA1000267A537B0579471228267A447B05794A82
:10CA20001228267A427B05794B1228267A4C7B0500
:10CA300079501228267A3F7B0579531228267A549A
:10CA40007B0579541228267A417B0579E112282644
:10CA5000900539E0A2E35004D2F08002C2F012D077
:10CA60003179521228268005121E367E00122A12B3
:10CA7000901CC5E06004640170031229349007081B
:10CA800012D004600612C926120529120EB8EEF95A
:10CA9000740102C98074F612039EE9FEA2E05026DA
:10CAA00075082B750905780812090D75086E75094A
:10CAB00000780812090D7C007D007A217B00121F8E
:10CAC000B074041208CFEEA2E35003122A06901CA1
:10CAD000C5E0600464017008EEA2E1500312292E43
:10CAE000EEA2E2500E90070A12D004600612C92688
:10CAF00012052902C98374F612039E74EC12099977
:10CB00007401120963901DE1E0F97A9C7B05121112
:10CB1000287405120BC3E4F07407120BC3E4F07A17
:10CB200004F91229BE9030FDE493F8C3EA98EB941F
:10CB3000005058122A18E970529030F512CBE76075
:10CB4000197A0479031229BE8A088B099030FDE412
:10CB500093F89030F512CBF150087405120BC374A2
:10CB600001F09030F712CBE760197A0279011229AF
:10CB7000BE8A088B099030FDE493F89030F712CB11
:10CB8000F150087407120BC37401F0901DE1E0F935
:10CB90007C9C7D05740112095B1211227A9C7B0535
:10CBA00079451228267407120BC3E0701174051220
:10CBB0000BC3E07009851882851983E48008851805
:10CBC000828519837401F0901DDBE0F8901DDAE096
:10CBD00058F8851882851983E05812D03B794112A4
:10CBE0002826741402C980E493F8740193F9E84983
:10CBF00022E493FA740193FBE8C39AF8E49BF9C327
:10CC0000E50898E509992274F712039E74ED12095C
:10CC100099E9FE900598F0AC18AD19901DE1E0F986
:10CC20007A9C7B051211287412120BC3EE12CC45AC
:10CC3000AA18AB191211227A9C7B05794512282675
:10CC4000741302B421F0901DE1E0F97C9C7D052273
:10CC500074F412039EEAFEEBFF901DE3E064FE70A5
:10CC600003A3E0F470767A167B00121E8A8A088B82
:10CC700009EA450960668A828B83740112C30F8AB0
:10CC8000828B83A36004740280027401F0EA240A98
:10CC9000F8E4350912C2D212F173A312DD71F0A2C9
:10CCA000E3400912CCDF12CD051211B2EE241512A9
:10CCB000BA1AE5082402FAE43509FB122040E50817
:10CCC000241312CCF1E4F0AA08AB09900599E0F91D
:10CCD000121E9612CCDF12D5A912CD14028FF512B6
:10CCE000CCE322EE240BF582E43FF58322E5082411
:10CCF00012F582E412BFE5228E828F83A3A3A3A341
:10CD0000A3A3A3A3A312D23922E0F8A3E0F98518C4
:10CD100082851983E8F0A3E9F02274F212039E746D
:10CD2000FD1209998A088B09890A8C0B7401120B70
:10CD3000C3740412D03B1212728A0C8B0DAE0CAF6E
:10CD40000DEE4F700302CDC812CDFD740712DD77D2
:10CD5000E5082413FAE43509FB8A828B8312CE138B
:10CD60008A828B8312CE12E508241512CCF112DDD3
:10CD70007112DD7EE508240BF8E43509F912CDD6F1
:10CD8000E8F0A3E912DF111211EE12DD5F12CE1EE0
:10CD90007401F07403650A60067401650A70071275
:10CDA000CDE77404800412CDE7E4F0901DE312B0E7
:10CDB0004512CD147401650B700312CDE0EEFAEF4D
:10CDC000FB122A2AE9F980027910901DE374FEF023
:10CDD000A304F0028B62EE2418F582E43FF583226F
:10CDE000EE12894AE4F02212CDEF7440F0A322EE55
:10CDF00012CDF422240FF582E43FF58322EE12F4E3
:10CE0000DE3FF58312CE0822E0F8A3E0F98882899C
:10CE10008322A3E088828983F0A308A9832212CE0B
:10CE20002222F0EE12CE28222413F582E43FF5836D
:10CE30002274F412039EEAFEEBFF7A007B04900555
:10CE400099E0F9121FFE12CED890054E7409F01227
:10CE500011EE8A088B09AC08AD0912B9D912CD05BB
:10CE600012203AE96401705A7A0F7B00121E8A8AF6
:10CE7000088B09EA4509604A8A828B83740212CEC4
:10CE8000CDF988828983A3E0FC88828983A3A3E00B
:10CE9000FBEC8A82850983A3A312E1D78882898368
:10CEA000A3A3A3E08A82850983A312CEC5FAA3E0D7
:10CEB000FB794A122826AA08AB09900599E0F912D5
:10CEC0001E96028FF5F0EE241512BFCA22F0EE2452
:10CED0001D12BFCAF8A3E0229004D712D5B7901E46
:10CEE00048E8F0A3E9F09004D912D5B7901E46E8BF
:10CEF000F0A3E9F02274F412039E74FD1209998ADA
:10CF0000088B097401120BC3740212D03B12127207
:10CF10008A0A8B0BAE0AAF0BEE4F700302CFE312FF
:10CF2000F4FDE412D018A3A3A3E064017008888282
:10CF30008983A37420F0850882850983A3A3A3A312
:10CF4000A3E06401700988828983A3E0D2E6F085BA
:10CF50000882850983A3A3A3A3A3A3E06401700AA5
:10CF600088828983A3E0D2E7800512B9D9740112BF
:10CF7000D029E064017021850882850983A3A3126A
:10CF8000D004600312CFE8850882850983A3A31229
:10CF9000B02F12CDD712CD14850882850983A3A3A3
:10CFA000A3A3A3A3A3E06401700712F06EF0A3E4AF
:10CFB000F085088285098312CD05121290E960047C
:10CFC00012CFEFF0EE241712CFEB1211EE12DD5F4D
:10CFD00012A34412CFF612BA4DFAEFFB122A2AE935
:10CFE000F98002791002C0BDEE241612DD862212ED
:10CFF000BA11440422E0F8A3E0F98E828F83221252
:10D00000D00AF58312D5B7E849228E828F8312BCED
:10D01000E5241FF582E4382212D01C2212D02022EF
:10D02000F0850882850983A32212D01CA3A3A3A3A1
:10D0300022A2F0E433851882851983F0AA18AB196F
:10D040002274F512039E74F3120999890AEAFEEB21
:10D05000FF7508007509007C0D7D007900AA18ABEA
:10D0600019121E7212C2D312D1F0741F58600C7ABA
:10D07000D37B00122472790002D140E8A2E5500867
:10D08000740C120BC37401F0E8A2E75008740B1281
:10D090000BC37401F0E8A2E6740A5008120BC374C3
:10D0A00001F08008120BC3E0640170138E828F833D
:10D0B000A3A3A3A3A3A3A3E06032EE241380128E44
:10D0C000828F83A3A3A3A3A3A3A3A3E0601EEE2444
:10D0D00015F582E43FF58312AA656010AC08AD092E
:10D0E0007402120BC3AA82AB8312204012CCDF124F
:10D0F000CD09740A120BC3E06401703B12CCF81224
:10D100001290E97039EE240B12BB48900542E0689A
:10D110007003A3E0697027E5084509601A1211EE53
:10D120008A088B09AC08AD097402120BC3AA82AB42
:10D130008312203AE96007AA18AB19120C4EA90A0B
:10D14000740D02B6D674F712039E74CD120999EAD3
:10D15000FEEBFF8E828F8312D20EA2E0400302D13B
:10D16000EB12D1F7E054FE12EDD6740D12096312E2
:10D17000D2211211E8E97073742A120BC312D2047F
:10D1800070697C0D7D007900AA18AB19121E7274AB
:10D1900016120BC312CD09742A120BC312D1F0A2BE
:10D1A000E55008740B120BC37401F0E8A2E75008B5
:10D1B000740A120BC37401F0E8A2E65004742080D4
:10D1C000027422120BC312BA207402120BC3AA8279
:10D1D000AB831220408E828F83A3A3E0C0E0740C47
:10D1E000120BC3D0E012D03B120C48743302B421AE
:10D1F00012E36EA3E0F8228E828F8312D99BA3A341
:10D20000A3A3A32212B5426404228A828B83E0F88E
:10D2100012D21422A3E0C82406F582E438F583E094
:10D2200022EA241EF582E43BF583E0F9EA241FF5A7
:10D2300082E43BF58312D2392212F16EFB22E9F827
:10D240007900740468600A740A6860057403687081
:10D250000279010208B774F612039E8A828B8374E6
:10D2600024F0A3A37401F0122A0C8A088B09AE08DB
:10D27000AF09EE4F60108E828F8312DF0F1211EE16
:10D28000EE241A12E1D0EEFAEFFB02C983C082C08D
:10D290008390053C02AD93C082C083901DE202AD35
:10D2A00093C082C083E9901DE202ADB1C082C08309
:10D2B0009005B57401F0E9A2E350037403F0E9A20C
:10D2C000E15004E0D2E2F002C5F174F612039E7957
:10D2D000007C008A088B0978081205C9F8FF07FF4F
:10D2E000D2FDD2FDD2FDD2FDD2F5D2F9D2FFD2F1DC
:10D2F000D27C01800A7C0480067C0280027C08903B
:10D3000005B5E05C600479028005EC6002790102F9
:10D31000C98374F412039EEAFEEBFF890812298E7A
:10D320008A0A8B0BA80AA90BE84960418882898385
:10D33000A3A3A3A3E06036C394055031740165082C
:10D34000601A88828983A3A3A3A3E06401600D8887
:10D35000828983A3A3A3A3E06402700A88828983DD
:10D3600012CD05120D0EEEFAEFFB122982028FF597
:10D3700074F612039E8A828B83E07014A3A3A31217
:10D38000D004600C8A828B8312CD02120F068004B7
:10D390007A007B0002C983C082C08390054EE0649E
:10D3A0000870031212B402C5F1C082C0837C00EC85
:10D3B00075F003A4F8ADF0EDF912D47F7003A3E08B
:10D3C0006B7018903100E493C0E074B828F5827453
:10D3D000053DF583D0E0F079C580620CECC3940381
:10D3E00040CD7C00EC75F003A4F8A9F074B928F5E1
:10D3F000827405129B0D64FE7003A3E0F4600F0CB1
:10D40000ECC3940340DE7C00EC12D4407026EC7533
:10D41000F003A4FCADF074B82CF874053DF98882D3
:10D420008983A312E1D6903100E49388828983F046
:10D43000790080090CECC3940340CD79C702C5F193
:10D4400075F003A4F8A9F074B828F582740512EFFA
:10D450005E22C082C0837C00EC75F003A4F8A9F0C2
:10D4600012D47F7003A3E06B700912D44760047973
:10D470000180090CECC3940340DE790002C5F1740D
:10D48000B928F582740512EF5E6A2274F212039EC7
:10D4900074DD120999EAFEEBFF750800901CC5E0E7
:10D4A00060076401600302D5A290053FE06E70033F
:10D4B000A3E06F7010EE4F700302D596750801124D
:10D4C00012BA02D5A21229948A0A8B0BEA450B7074
:10D4D0000302D5968A828B83A3A3A3A3E064016091
:10D4E000108A828B83A3A3A3A3E06402600302D506
:10D4F00096851882851983E412D5B0740B120BC37C
:10D50000E8F0A3E912D03B122A24E9700302D59671
:10D51000850A82850B8312D5A912CD147900120DCC
:10D5200002850A82850B8312DAC4120BC3AC82AD6A
:10D53000837418120BC3AA82AB83122040850A821F
:10D54000850B8312BB4E7420120BC312CD147422B0
:10D55000120BC3E4F07C02850A82850B83A3A3A38C
:10D56000A3E0F9740D12095B12124E850A82850B35
:10D570008312BB4E7401120BC3E8F0A3E912D03B37
:10D58000122A1E750801E50A240CF582E4350BF514
:10D5900083129B70800C90054C12BA30FAEFFB128C
:10D5A000137AA9087423028B6412D5B7901DE32265
:10D5B00012B1C312D5B72212D614F922C082C08389
:10D5C00074FE120999901CC5E0600464017023790F
:10D5D00001120D0812D5FA90053FE8F0A3E912D028
:10D5E0003B795312282685188285198312CD05129E
:10D5F000238E74021208CF02C5F185188285198323
:10D60000EAF0A3EB12D609F922F085188285198376
:10D6100012D61422E0F8A3E02274F412039E74F3ED
:10D620001209998A088B09ECFEEDFF750A12EA458A
:10D63000097005790002D70590053FE06508700480
:10D64000A3E06509701D1211EE8A0A8B0BAC0AADBE
:10D650000BEEFAEFFB12203AE97005750A01800320
:10D66000750A00851882851983E4F004120BC31231
:10D67000DEFD12D03B122A3CE9602A7403120BC370
:10D68000AA82AB83122A60E964017019750A0174D9
:10D6900003120BC3AC82AD83EEFAEFFB12203AE922
:10D6A0006003750A00901CC5E06004640170177483
:10D6B00012650A7011EEFCEFFDAA08AB091229AC45
:10D6C000E96003750A00EEFCEFFDAA08AB0912132E
:10D6D00098E9F8740A687005750A01801D74A068DD
:10D6E0007012EEFCEFFDAA08AB091213AAAA08AB50
:10D6F000091213BC7401650A70097900AA08AB0904
:10D700001212C6A90A740D028FF274F612039EEA71
:10D71000FEEBFF8908901CC5E060046401701E12D6
:10D7200012B4E508F5097809120911790DEEFCEF3C
:10D73000FD7AFC7BFF1212D274011208CF02C9835A
:10D7400074F712039EEAFEEBFF8E828F83A3A3A3DE
:10D75000A3A3A3A3A3E0601612D7A6129C1212CD16
:10D76000051212C0E96401700512CCDF80298E8297
:10D770008F83A3A3A3A3A3A3A3E0602512BA1712C8
:10D78000CCF81212C0E9640170178E828F83A3A3B4
:10D79000A3A3A3A3A3A3A312CD051212A87901806A
:10D7A00002790002B424EE2415F582E43FF58322C9
:10D7B00074F212039E74FD1209998A088B09ECFE1B
:10D7C000EDFF890B750A017401120BC3740412D0AA
:10D7D0003B121272EA4B60427411120BC3E06014E8
:10D7E00012DE76E412E3768A828B83E0D2E7F012CF
:10D7F000D81DE4F012D82712CE02740312DACEEE4E
:10D8000088828983A3A3F0EF88828983A3A312B1BE
:10D81000C212DD93122A2AE9F50A028B60EA241467
:10D82000F582E43BF5832212F4DD3B2274F012030F
:10D830009EEAFEEBFF890A750B01EE12DB903F12A8
:10D84000D994F50C88828983A3A3E0FA888289831E
:10D8500012D98312B9E26404600A7AD37B001224DD
:10D860007202D973E50C1207960200027ED8030BF0
:10D870002BD9030C11D90DE9D80E2BD928D9901C1E
:10D88000C5E060076401600302D92B900539E0A26E
:10D89000E1400302D92B7900AB09120D98EA4B60E5
:10D8A0003D8A828B83A3A3A3A3A3A3E05418602E75
:10D8B00012CCDF1207118A828B83A3A3120711797E
:10D8C000008E828F83A3A3A3A3A3A3A3A3A312D990
:10D8D0007712CD05120DB074041208CF802E790195
:10D8E000AA08AB09120C608042901CC5E060046479
:10D8F000017038900539E0A2E15030AB091212A254
:10D90000AA08AB091212A8E964C5701F750B008044
:10D910001A901CC5E0600464017010900539E0A203
:10D92000E150081223B28003750A00EE2409F50EB7
:10D93000E43FF50FAC08AD09A90C850E82F5831202
:10D94000CD05120C78850E82850F8312CD0512123B
:10D9500090E9601F12BFC3C39402401712CCDF12BC
:10D96000E2997003A3E069600AE50BA2E05004A904
:10D970000A80027900803112D97B2212BA288A8269
:10D980008B8322A3A3A3E0F8E4C8F9EA28F508E40E
:10D9900039F50922F58312D99BE02212D614F988B1
:10D9A000828983A3221208CF7F0802060F74EE1229
:10D9B000039E74F51209998A0A8B0B890D8C0E8DC2
:10D9C0000F7E01EE120BC3740AF0741D120BC3E03C
:10D9D000F50CE9700FE50CC333240AC0E0EE120B1E
:10D9E000C3D0E0F0AA18AB191212728A088B09EAA8
:10D9F0004509700302DAA612C541350912DC4474E8
:10DA000009F0A3E50DC43354E0450C12DC5DAC0E07
:10DA1000AD0FEEFAEFFB122040EE2408FE50010F8E
:10DA2000E50D702F7C00741E120BC312DAB5801D39
:10DA300012DAADEA28F8EB39F98882898312DC58CA
:10DA40008882898312A1E0F0A30EAF830CECC3950A
:10DA50000C40DDE508241712CCF17401F01211EE30
:10DA6000E508241AF582E4350912DAC2120963AA1C
:10DA70000AAB0B122A54E96019E508241612CCF1FE
:10DA80007401F07403120953E508241812CCF11242
:10DA9000CD14850882850983A3A312DACCAA08AB2A
:10DAA00009122A2AE9FEEEF9740B02C315EC25E0EF
:10DAB000F8E433F92212DAB92212D614F9E8FAE9B5
:10DAC000FB22F583EAF0A3EBF0740322E50AF0A34E
:10DAD000E50BF02274F012039E74F81209998A087B
:10DAE0008B0912DB8F350912DCD8F8741F58F50A40
:10DAF000880BA3AE82AF83EEFCEFFDAA18AB191220
:10DB00002040EE2408FE50010FAC18AD197A607B5E
:10DB10000512203AE9607374E0550B7066AA0AEAB0
:10DB20002AFA7B00121F2C8A0C8B0DEA450D605AD5
:10DB30007C00801D8E828F8312C56C12DAADE50CDD
:10DB400028F582E50D3912E1D4EE2402FE50010FD2
:10DB50000CECC3950A40DD780C12090D780A120905
:10DB60001174031209637900E508240B12CCF11239
:10DB7000CD051212EA74031208CFAA0CAB0D121FC6
:10DB80003280077AD37B00122472740802D9A5EA86
:10DB9000241DF582E42274F012039E8A0A8B0B89FD
:10DBA0000D8C088D09901BE512D00460757410125D
:10DBB0000BC3E0F50C12DAAEE8240EFAE439FB12DE
:10DBC0001E8A8A0E8B0FAE0EAF0FEE4F60548E8200
:10DBD0008F8374D4F012DC33A3A3E50DF0AC08AD51
:10DBE00009EE2405FAE43FFB12204012DC25E50C87
:10DBF000F07411120BC312E35F7808120909AC0C20
:10DC0000EC2CFCE433FDEE240EFAE43FFB121E6024
:10DC100074031208CFEEFAEFFB901BE512E36A12D1
:10DC2000052902D9A8EE12DC2A22240DF582E43F50
:10DC3000F58322A3A3E50AF0A3E50B12DC3F221231
:10DC4000C009A322F58312DC53FF8E828F832288C2
:10DC5000828983E0FEA3E022E08E828F83F0A3AE70
:10DC600082AF832274F612039E74F8120999890810
:10DC700012DB8F3B12DCD8F9741F59F88909A3AE67
:10DC800082AF837401687042EEFCEFFDAA18AB19F5
:10DC9000122040EE2408FE50010FAC18AD197A6036
:10DCA0007B0512203AE9602974E05509701C8E82C8
:10DCB0008F83A3E0FA8E828F83A312C56E8E828F2C
:10DCC00083E0F912131AA90880097AD37B00122481
:10DCD000727900740802C980F583E02401FEA3E094
:10DCE0003400FF8E828F83E02274F012039E74FD55
:10DCF0001209998A0A8B0B8C088D09890D750C0104
:10DD00007401120BC3740312D03B1212728A0E8B71
:10DD10000FAE0EAF0FEE4F603F12CDFD740BF0A3B0
:10DD2000E50D12DD777413120BC312DD7112DF11D2
:10DD30001211EE12DD5F12DD7EEE2418F582E43F53
:10DD400012DD918E828F83A3A3E50AF0A3E50B1267
:10DD5000DF04122A2AE9F50CA90C740302D9A512D2
:10DD6000DD67EAF0A3EB22EE241AF582E43FF583A7
:10DD700022E08882898322F0A3A882A98322F0EE80
:10DD8000241612DD8622F582E43FF5837401F02229
:10DD900039F58312DEFDF02274EF12039EEAFEEBEA
:10DDA000FF751000EE12DB903F12DFE4F508A3E0F0
:10DDB000F50912D7A612CD0512298EEA4B7003027F
:10DDC000DE718A828B83A3A3A3A3E0700302DE71BA
:10DDD000C39403400302DE71E508C3940F5004E5C9
:10DDE0000960057510018079EA2412F582E43BF59B
:10DDF00083E4F0E5087022902FAF7808120A5012E1
:10DE0000DE767808120B36902FAF7808120A50127F
:10DE1000E7CD7808120B368039750900740278084E
:10DE2000120A9C74AF2508F582742F12CCF4780C7A
:10DE3000120A5090816A7808120B54780C790812F3
:10DE400002AF12DE76780C120B3612E7CD780C1288
:10DE50000B36EA241BF582E43BF5837401F01223B0
:10DE6000FA901CB3E0FCA91012CCDF12CD051213FE
:10DE7000027F0902060FEA2417F582E43BF58322AC
:10DE800074F012039E74F51209998A088B09890BA4
:10DE90008C0C750A017401120BC3740312D03B126F
:10DEA00012728A0E8B0FAE0EAF0FEE4F604812CD7E
:10DEB000FD740C12DACEA3E50C12DF111211EEEE96
:10DEC000241AF582E43F12DAC2120963AA08AB09E8
:10DED000122A54E9600E12CFE8740312095312CDCE
:10DEE000D612CD148E828F83A3A312DEFD12DF041F
:10DEF000122A2AE9F50AA90A740B02D9A5E508F045
:10DF0000A3E5092212CE227401F0EEFAEFFB22748F
:10DF100001F0EE241712DD862274F012039E12DB4C
:10DF20008F3B12DFE4F8A3E0FEE8600302DFE17458
:10DF3000016E600874026E600302DFE1EE901CB3B4
:10DF4000F07508B375091C780812090D750801757C
:10DF50000900780812090D7C007D007A517B0012BF
:10DF60001FB074041208CF74026E7075901E69E0C1
:10DF7000700A902FAF7808120A508028F5087402B2
:10DF80007808120A9C74AF2508F582742F12CCF41D
:10DF90007808120A5090816A780C120B547808792C
:10DFA0000C1202AF90818E780C120B547808790C09
:10DFB00012032F90812A780C120B547808790C12D6
:10DFC00002AF901CB57808120B36901CB512070DE5
:10DFD0007A007B40900599E0F9121FF8740412084A
:10DFE000CF02D9A8F583E02401F8A3E03400F98832
:10DFF000828983E02274F612039E74DA120999EA88
:10E00000FEEBFF12CFFF60508E828F8312CD05ACE6
:10E0100018AD1912D2211211D67409120BC312E2D3
:10E02000997003A3E069603012E366120711750866
:10E03000FE7509FF780812090D741C120BC3E0F974
:10E04000740D120BC312BA20740F120BC312CD053C
:10E05000120DB074041208CF742602C98074F7122E
:10E06000039EE9FD7A007B00901CC5E0600464011A
:10E0700070407C00800B12E109E02AFAA3E03BFB30
:10E080000C9030FD12EF4C5029EC75F01CA4F8AE4A
:10E09000F0EEF912EF6EF460E7740E28F582740C5E
:10E0A0003912D00260DAED60CD12E109E4F0A3F09C
:10E0B00080CE7C00800B12E0F6E02AFAA3E03BFB66
:10E0C0000C12EF49502DEC75F017A4F8AEF0EEF9F4
:10E0D00012F0ED7003A3E0F460E6745F28F582743B
:10E0E0000E3912D00260D9ED60CC12E0F6E4F0A354
:10E0F000F080CD02B424EC75F017A4F8EEF9745F4B
:10E1000028F582740E39F58322EC75F01CA4F8EE24
:10E11000F9740E28F582740C39F5832274EC12031D
:10E120009E890CEAFEEBFF900598E0C3950C503BEE
:10E130001212429005CA12E172900532E0F508E42D
:10E14000F509F50AF50B9081867810120B547808C2
:10E1500079101202AF78081209057A007B02900547
:10E1600099E0F9121FF274041208CF02875D8A82C7
:10E170008B83EEF0A3EFF02274F612039EEAFEEB1F
:10E18000FF9005B6801388828983E06E7003A3E058
:10E190006F603A88828983A3A312D00470E87A045E
:10E1A0007B00121F2C8A088B09A808A909E849607E
:10E1B0001C8882898312E1729005B612CD0588828F
:10E1C0008983A3A312E1D69005B612CD1402C983A8
:10E1D000F582E43FF583EAF0A3EBF02274F4120336
:10E1E0009E7E009005B680070E8A828B83A3A312C1
:10E1F000B32F70F4EE25E0FAE433FB121F2C8A08EB
:10E200008B09EA4509607F7C009005B680228A82EE
:10E210008B83E0F50AA3E0F50B12DAADE50828F5EB
:10E2200082E50939F58312DACC0C8A828B83A3A3A9
:10E2300012B32F70D990059412E2997003A3E0698C
:10E240007808701C12090DEEF50A780A1209117C83
:10E25000607D05790090059412CD051212EA801AAE
:10E2600012090DEEF50A780A1209117C607D057914
:10E270000090059412CD051212DE74031208CFAA85
:10E2800008AB09121F321229E2028FF58E828F83AA
:10E29000A3A3A3A3A3A3A3A3A312D5B790053FE071
:10E2A0006822C082C08380128A828B83A3A312BBA0
:10E2B0004E9005B612CD14121F329005B612B32F30
:10E2C00070E602C5F174F512039E90054C12BCDC99
:10E2D0009005CA12A05F12CD147ACA7B057950123C
:10E2E00028269005CA12E35F801312EC167004A36F
:10E2F000E06509600612EC23121386050A903109C5
:10E30000E493F8E50AC3985020E50A75F017A4F8DD
:10E31000A9F012EAC46E7003A3E06F70CD745428A4
:10E32000F582740E12DD9080D29005CA12BCDC908A
:10E330001BE712D00460257A067B00121E8AEA4B86
:10E34000601A8A828B8374D5F0A3A3E412E71104C8
:10E3500012E376901BE712E36A12052902B6D9127E
:10E36000876C750A00228E828F8312E36E2212D68A
:10E3700014F58388822212B1CFEEF0A3EFF022C011
:10E3800082C08390053FE064FE7003A3E0F4600E5A
:10E39000900539E0A2E1500612139E12134402C503
:10E3A000F174F012039E90058DE06053F50CE4F5D6
:10E3B0000DF50EF50F90812A7808120B54780C7920
:10E3C000081202AF121E848A088B09A808A90990B6
:10E3D00030F9E49358F508A3E49359F509E4F50AF4
:10E3E000F50B780C7908120AAF780C1209057A003F
:10E3F0007B01900599E0F9121FF874041208CF020E
:10E40000D9A874EE12039E7E007F008E0A8E0B1236
:10E410002964750D00803BAA0D7B0012296A8A08C9
:10E420008B09A808A909E849602688828983A3A3E3
:10E43000A3A3E060046404701788828983A3A3A364
:10E44000A3A3A3A3A3A3A3E0F91213B0E960010F50
:10E45000050D9030FDE493F8E50DC39840B9121313
:10E46000748A0E8B0F750C008023AA0C7B0012138C
:10E47000808A088B09A808A909E849600EE8240FDA
:10E48000129B0AF91213B0E960010E050CC3E50CEA
:10E49000950EE4950F40D3EF2EFE700302E5988EA3
:10E4A0000875090074027808120A9CAA08AB0912C0
:10E4B0001F2C8A0A8B0BEA450B700302E596750C3C
:10E4C000008E0875090074027808120A9CAC08AD29
:10E4D0000979FF121E72750D00805EAA0D7B001275
:10E4E000296A8A088B09EA4509604C8A828B83A3D2
:10E4F000A3A3A3E060046404703D8A828B83A3A37A
:10E50000A3A3A3A3A3A3A3A3E0F91213B0E9F96003
:10E5100026050C780A12090DEEFD8508828509830F
:10E52000A3A3A3A3A3A3A3A3A312E62912CD051219
:10E53000134A74021208CF050D9030FDE493F8E5FC
:10E540000DC3985006E50CC39F4090750C00C3E5C1
:10E550000C950EE4950F5040AA0C7B001213808A94
:10E56000088B09EA4509602AEA240F12B027F9123C
:10E5700013B0E9F9601C780A12090DEEFDE50824D4
:10E580000E12CCF112E62912CD0512134A740212B2
:10E5900008CF050C80B87E007F62900537E0600BE5
:10E5A000F912106EE9F87454C398FF75F003EF8404
:10E5B000F50D94204003750D1F850A08850B09751C
:10E5C0000C00EF6005750C207F00E50DC39E500523
:10E5D000850D0F80088E0FE50CD2E6F50CAC08AD6A
:10E5E00009AA0CA90F121350E9F50EE50CA2E6409A
:10E5F0001D150F7800800BE5082404F5085002056E
:10E600000908E8C3950F40EFE50FCEC39EFEE97001
:10E6100006E50CA2E650A8E50A450B6007AA0AAB7E
:10E620000B121F32A90E02C318E0FC85088285096F
:10E63000832274F212039EEAFEEBFF89088C098D97
:10E640000A7C007D00740E120BC312CD05750B0001
:10E65000800DEAFCEBFDEA2404FA50010B050BE502
:10E660000BC3950A400302E7018A828B83E0F470B2
:10E6700003A3E0F4607AEC4D600C8C828D83C3E0E0
:10E680009EA3E09F50CC8A828B8312E704EE98EF22
:10E690009950BFEAF8EBF988828983E0F47003A30C
:10E6A000E0F46010E82404F8500109050BE50BC301
:10E6B000950A40E3E8FCE9FDE824FCF8E934FFF9B9
:10E6C0008882898312E7098C828D83E50CF0A3E5AB
:10E6D0000D12E7208C828D83A3A312E716A3A3A3B8
:10E6E000E08C828D83A3A3A3F0C3EA98EB9940C486
:10E6F00012E16E8A828B83A3A3E50912E711E50874
:10E70000F0028B6712D5B7C322E0F50CA3E0F50D3C
:10E710002212B1C3A32212E71A22F088828983222F
:10E7200012E726A3E02212E71AA32274F212039E34
:10E7300074FD12099989088A09ECFEEDFF750A013A
:10E7400075F003E9A42402C0E07401120BC3D0E009
:10E7500012D03B121272EA4B607012D82712CE020E
:10E760007408F0741F55084509A3F0E82402F85016
:10E770000109750A0080338E828F8312DD7112DDEC
:10E78000778E828F8312CE128E828F83A3A3E05462
:10E7900007C4FC8E828F83A3A3A3E054074C12CE40
:10E7A00014EE2404FE50010F050AE50AC395084043
:10E7B000C68A828B83A3A374FCF0A374FFF012E7D4
:10E7C000CD7401F0122A2AE9F50A028B60EA2413BB
:10E7D000F582E43BF5832274F112039E8A0A8B0BC7
:10E7E0007508007AFE7BFF7CFE7DFFE50A12DB9058
:10E7F000350B12D994F509741F5509F50CE824025C
:10E80000F8500109E509A2E74065E50A2417F582F9
:10E81000E412F610FE75F003E50CA424026E704FAE
:10E82000E50C600612DC4FFBEEFA750D00801DE072
:10E830005407F50EA3A882A983EEFC90053FE06E75
:10E840007003A3E06F7003850E08050DE50DC395F9
:10E850000C502612DC4FFCE4CCFDEE2CE43DFFE82E
:10E860002402F850010988828983E0548860C07AC4
:10E87000D37B0012247202E9BAE508700BA90912D1
:10E88000135CE9700302E9BA12E9BF12CD0512293F
:10E89000948A0C8B0DAE0CAF0DEE4F605A8E828FAA
:10E8A00083A3A3A3A3A3A3A3E4F090310293F88EC0
:10E8B000828F83A3A3A3A3A3A3A3A3E0C39840240D
:10E8C00012E9C95001097A027B0012024EE88E82D9
:10E8D0008F83A3A3A3A3A3A3A3A3F0E508C39407D3
:10E8E000500205088E828F83A3A3A3A3A3A3A3A38F
:10E8F000A3E508F002E9BA7CFF7DFF12E9BF12CD63
:10E90000051213688A0C8B0DAE0CAF0DEE4F704FD5
:10E9100012136E8A0C8B0DAE0CAF0DEE4F7003020E
:10E92000E9BA7C177D007900121E7212E9BF12CF7E
:10E93000F51287BA8E828F83A3A3A3A3A3A3A3A355
:10E9400012BA4D12B59874AA12E9E85001097A0278
:10E950007B0012024E12DC25E812E9D47401F0901B
:10E960003102E49312BFD2C398401912E9C9500191
:10E97000097A027B0012024E12F074E508C3940774
:10E980005002050812F060E50812E9D9E4F012A07F
:10E9900057122A60E97023850A82850B83A3A3A3FB
:10E9A000A3A3A3A3A3E06012E50A2415F582E4352E
:10E9B0000B12BA2E12A0581220407F0702060FE554
:10E9C0000A12F4DE350BF58322903102E4937900CC
:10E9D0002401F822F012F06422F012E9DE22EE2483
:10E9E0000CF582E43FF58322F0903102E493790044
:10E9F0002401F82274F712039EE9FE74FE6A700384
:10EA000074FF6B603474605E6460602DEEA2E5405C
:10EA10001CA2E690053F500DC3E09AA3E09B50195D
:10EA2000790002B424C3E09AA3E09B40F390053F31
:10EA300012E704EC98ED9940E7790180E574F7124C
:10EA4000039E7E008008EE12EC1C1213860E12EA62
:10EA50007E40F37E00EE75F003A4F8A9F074B828A8
:10EA6000F8740539F988828983A374FEF0A304122F
:10EA7000E716E4F00EEEC3940340DA02B4249031BA
:10EA800009E493F8EEC3982274F712039E7E008087
:10EA9000010E12EA7E5026EE12EAD46A7003A3E059
:10EAA0006B70EE12EAC46C7003A3E06D600A74FF31
:10EAB0006C700374FF6D70D912EC2380047A007BB4
:10EAC0000002B42412EAC822745428F582740E3964
:10EAD000F583E02275F017A4F8A9F012EADF2212FC
:10EAE000EF3EE02274F612039E7CFF7DFF7AFE7BF0
:10EAF000FF121368EA4B703C7508008032E5087518
:10EB0000F017A4F8A9F0745928F582740E129B0D21
:10EB1000600512EF637016744A28FE740E39FF8E7A
:10EB2000828F8312CD05120DB6EEFAEFFB050812A7
:10EB3000EB3740C902C983903109E493F8E508C373
:10EB40009822C082C0837A007B007C00801012F083
:10EB5000E57003A3E0F460050AEA70010B0C12EF04
:10EB60004940EB02C5F174F412039E8A088B09EC4C
:10EB7000FEEDFF800B121386EEFCEFFDAA08AB0939
:10EB8000121368EA4B70EE028FF574F712039E7D44
:10EB9000007C0080020D0C12EF49501C12F0E57051
:10EBA00003A3E0F460F0EDF8EA684B70E8EC75F070
:10EBB00017A4F812EC2380047A007B0002B42474BA
:10EBC000F712039EEAFEEBFFEE4F60187C177D0004
:10EBD0007900121E728E828F8374FEF0A30412F0ED
:10EBE0007BF0A3F002B42474F612039E8A088B090A
:10EBF0007E00801AEE75F017A4F8A9F012EC1670DA
:10EC000004A3E06509600612EC231213860E12EAD3
:10EC10007E40E102C98312EAC865082275F017A494
:10EC2000F8A9F0744A28FA740E39FB2274F412031E
:10EC30009E8A088B09ECFEEDFF901CC5E060046421
:10EC400001702090054CE06E7003A3E06F70141209
:10EC500029948A0A8B0BA80AA90BE8496005E824C5
:10EC600008801AEEFCEFFDAA08AB091213688A08A7
:10EC70008B09A808A909E8496009E8240DFAE439D4
:10EC8000FB80047A007B00028FF574F412039E8AE5
:10EC9000088B09ECFEEDFF750A00750B00802FE56F
:10ECA0000B12F0D5122A60E96022E50B12EAD46556
:10ECB000087004A3E065097003750A0AEEFCEFFD15
:10ECC00012F0DC12203AE96003430AA0050B9031F0
:10ECD00009E493F8E50BC3985004E50A60C1A90A5A
:10ECE000028FF574F612039E7E00805AEEFA7B00C6
:10ECF00012296A8A088B09A808A909E84960468888
:10ED0000828983A3A3A3A3E06401603988828983F5
:10ED1000A3A3A3A3E06402602CE82407129B0AFAD1
:10ED200074012AF090058EE0C39A50198882898375
:10ED3000A3A3A3A3A3A3A3A3A3A3E412EDCBA31212
:10ED4000EDD6120DB60E9030FD12EA81409E7E0087
:10ED50008059EE75F017A4F8AAF0EAF912F0ED70F8
:10ED600003A3E0F46044744A28F8740E39F9E824E7
:10ED70000C129B0AF8740128F090058EE0C398509D
:10ED800029EE75F017A4F8EAF9744A28F8740E39D8
:10ED9000F9E812EDC539F583E4F0E8240EF582E4D4
:10EDA00039F583E412EDD6120DB60E12EA7E40A2BA
:10EDB0007A00EA12D440600214F00AEAC3940340D5
:10EDC000F102C983EE240FF582E42212E726A3A301
:10EDD000A3A3A3A3A32212E71A12D2392274F11219
:10EDE000039E8A0A8B0BECFEEDFF750E007A007B0A
:10EDF000017508FE7509FF740F120BC312E7098035
:10EE000011121E84E50EF5F0EA84E5F0FA750E00A5
:10EE10007B007C00800712EF3E1287680C12EF49DE
:10EE2000505CEC75F017A4F8ADF0EDF912F0ED7050
:10EE300003A3E0F460E612EADB650A7004A3E06570
:10EE40000B60D912F0D07003A3E06F60CF12EADB41
:10EE5000650C7004A3E0650D60C212EF6360BDC372
:10EE6000940850B8E0640760ADEB050E70AEE50E97
:10EE7000C39A40A8744A28F582740E02EF08901CC9
:10EE8000C5E060076401600302EF107C0080071298
:10EE9000EF7E1287680C9030FD12EF4C5072EC75CB
:10EEA000F01CA4F8ADF0EDF912EF7964FE7003A345
:10EEB000E0F460E112EF79650A7004A3E0650B608D
:10EEC000D412EF796E7003A3E06F60C912EF796519
:10EED0000C7004A3E0650D60BC12EF5360B7C394DF
:10EEE0000850B212EF6E640160ABE0640260A612DB
:10EEF000EF5364076099EB050E709AE50EC39A40D4
:10EF00009474FE28F582740B3DF58312CD05802B99
:10EF1000E50E6011EA700E7401650E600302EE01E9
:10EF20007A0102EE0D74FE6508700474FF650960D5
:10EF300006AA08AB0980047AFE7BFF02E9BA744A8C
:10EF400028F582740E39F58322903109E493F8ECA8
:10EF5000C39822740728F582740C12EF5E2239F5EB
:10EF600083E022745828F582740E12EF5E22740238
:10EF700028F582740C12EF5E2212EF7EE02274FEFE
:10EF800028F582740B39F5832274F512039E8A08E2
:10EF90008B09ECFEEDFF750A008002050A9031092D
:10EFA000E493F8E50AC3985022EEFCEFFDE50A125F
:10EFB000F0D512203AE960E3E50A75F017A4F8A944
:10EFC000F0744A28F582740E12DD9002B6D9E9F881
:10EFD0007907C3940D400479018019E8C394074070
:10EFE000047903800FE8C39403400479058005E8A1
:10EFF000700279000208B774F012039E8A088B0928
:10F000008C0A8D0B890C12136E8A0E8B0FAE0EAF0D
:10F010000FEE4F60487C177D007900121E728E82C1
:10F020008F8312DEFD12F07B12DACCE50C60071242
:10F03000B597E50C800312F06EF0900593E0640143
:10F04000700612F060E4800512F060740712E9E8BF
:10F050005001097A027B0012024E12F07402D9A804
:10F0600012F06422EE240EF582E43FF5832212CDE5
:10F07000EF740122EE12DC2AE8F02212A9D8A322B2
:10F0800074F712039EEAFEEBFF750800803AE5086C
:10F0900075F017A4F8A9F012F0D07003A3E06F6028
:10F0A0001474FF6E700374FF6F701B12F0ED700329
:10F0B000A3E0F4601112F0DC122A60E97008E508A0
:10F0C00012EC1C121386050812EB3740C102B4245F
:10F0D00012EADF6E2275F017A4F8A9F0744C28FA32
:10F0E000740E39FB22EC75F017A4F8A9F012EADFD0
:10F0F00064FE22C082C0837AFF7BFF1213BC02C56C
:10F10000F1C082C0839005CC74CEF0A37413F0904C
:10F1100005CE74D4F0A37413F09005D074DAF0A384
:10F12000741302ADB174F712039EEAF8EBF9900480
:10F13000D512F16ECA2406F582E43AF583E0702B0D
:10F1400088828983A3A3A3A3A3A3A3A3A3120711C4
:10F150009004D512F173120BAC88828983A3E0F975
:10F16000120C6C74021208CF1229E202B424E0FAE5
:10F17000A3E02212F16EF5838A8222C082C08390BE
:10F18000059612F23FF090059612D00470057901B1
:10F1900012131402C5F174F612039E74FC1209993D
:10F1A000E9FE903101E493700874E16E600302F2AD
:10F1B0003AEA2408F8E43BF98882898312F23F1284
:10F1C000F248700E900596E4F0A3F0790112131442
:10F1D0008068901E7DE06062F890059612CD05C3B0
:10F1E000E89AE49B505479001213148A088B09ACF6
:10F1F00008AD09ECF8EDF9E875F064A4F8AAF0752B
:10F20000F064E9A42AF990059612CD05120256E899
:10F21000941AE994004023901BDF12D004601B90E5
:10F22000059612CD097402120BC3ECF0A3ED12D0B7
:10F230003B901BDF12E36A120529740402C980E0C7
:10F240002401F0A3E034002212E71A12D5B7E849EE
:10F2500022C082C08374F81209999080CBAC18AD9B
:10F26000197408120833AC18AD1912203AE9640178
:10F270007004790080027901740802D5F474F612E2
:10F28000039E740C120BC312BCDC743A6E7001EF57
:10F290006006743B6E4F7023740A120BC312071181
:10F2A0008C088D09780812090DEAFCEBFDEEFAEFE7
:10F2B000FB121FB674041208CF8002790A02C983B8
:10F2C000C082C0839005D2745EF0A37429F09005CB
:10F2D000D47458F0A37429F0901CB3E06401703228
:10F2E0009005D674F8F0A37413F09005D874FEF06E
:10F2F000A37413F09005DA7404F0A37414F090056D
:10F30000DC740AF0A37414F09005DE74F2F0A374B8
:10F3100013F09005D612D004600612C926120529F2
:10F3200002C5F174F412039E74E61209998A088BDF
:10F33000097404120BC37402F00412095B121272F6
:10F340008A0A8B0BAE0AAF0BEE4F700302F4AD12BC
:10F35000F4FD746012CE1E12DF0F1211EE12DD5F8B
:10F3600012BA4912DEFD12C02A701290052BE0C0BD
:10F37000E012F4B2D0E0F090052BE004F012F4CEED
:10F380007016901E5DE0600D900536E0700A8E826A
:10F390008F83E0700312CDE0AC18AD19EEFAEFFBED
:10F3A0001211CA8A088B09EA4509700302F4A67A89
:10F3B000217B00121F2C7406120BC312E1D67406B7
:10F3C000120BC312D004700302F49F7C217D0079DC
:10F3D000007406120BC3E0FA121E72740112095B6C
:10F3E00079501228207401120BC312BB4E740612FE
:10F3F0000BC312F16ECA2409F582E43AF58312CDEB
:10F400001490053F12BB4E7417120BC312CD147427
:10F4100006120BC312BCE112F4D4F07406120BC333
:10F4200012B112740212F5237406120BC312F17397
:10F4300012CD147406120BC312F50812F52EC0E09B
:10F440007406120BC312BCE112F4E4D0E0F0EE2417
:10F450000E12F4BCC0E07406120BC312F4EDD0E03F
:10F46000F07406120BC312BCE112BCD212DD91EE95
:10F47000240F12BB48740C120BC312CD148A828B5A
:10F4800083E0C0E0740E120BC3D0E0F074061209E2
:10F490005B12113A7406120BC312CD05121F32AA69
:10F4A00008AB09121F32EEFAEFFB121F32741A0278
:10F4B0008FF2EE2414F582E43FF5832212F4C1E0CA
:10F4C00022F8E43FF9E8FAE9FB8A828B832212BF33
:10F4D000C764012212F4DE38F583740222EA240B99
:10F4E000F582E422241EF582E438F5832212F4F139
:10F4F0002212BCE5240CF582E438F5832212CCE319
:10F5000012CE087404F0A322E012F5127401F0A3E5
:10F51000E422F8A3E0C812F51A22240DF582E4389B
:10F52000F5832212DC3F12D5B722E8F0A3E912A836
:10F5300028E02274F612039E7E0080187C047D0071
:10F5400079FF8E088D0974027808120A9C12F76EF2
:10F55000121E720E90310712EA8140E002C98374D4
:10F56000F412039E74F71209997508008022850829
:10F570000A750B007402780A120A9C74E9250AF5D0
:10F5800082741112F61024FFF0A3E034FFF0050896
:10F5900090310712EB3A506D85080A750B00740222
:10F5A000780A120A9C12F608F47003A3E0F460DEF5
:10F5B00085080A750B007402780A120A9C74E92502
:10F5C0000AF5827411350B12D00270A27408120B66
:10F5D000C37402F085080A750B00780A120A9C743D
:10F5E000E7250AFE7411350BFF8E828F8312CD0939
:10F5F00012F6161228687C047D0079FFEEFAEFFB04
:10F60000121E72808902B10D74E7250AF582741109
:10F61000350BF583E02212F7872274EE12039E74F5
:10F62000F7120999EAFEEBFF750CFF7408120BC381
:10F6300012F779122862E9641A700302F6EC750E6B
:10F6400000741B120BC37808120B54800B74FF65F7
:10F650000C7003850E0C050E903107E493F8E50E4F
:10F66000C3985048850E1075110074027810120A64
:10F670009C12F6F0F47003A3E0F460D1850E1075CF
:10F68000110074027810120A9C12F6F06E7003A337
:10F69000E06F70C2750F007402780E120A9C74E954
:10F6A000250EF5827411350FF5838030E493650ED5
:10F6B000702D74FF650C602E850C0E750F007402A2
:10F6C000780E120A9C74E7250EF87411350FF9882C
:10F6D00082898312E17288828983A3A312DD9379E0
:10F6E00001740902C31512F616122868790080F118
:10F6F00074E72510F58274113511F583E02274F456
:10F7000012039E74F7120999EAFEEBFF7408120BBC
:10F71000C312F77912286875080080020508903135
:10F720000712EB3A504585080A750B007402780AF7
:10F73000120A9C12F608F47003A3E0F460DE850858
:10F740000A750B007402780A120A9C12F6086E7091
:10F7500003A3E06F70C67C047D0079FF8D097402FD
:10F760007808120A9C12F76E121E7202B10D74E72D
:10F770002508FA74113509FB22740212A828EEF04C
:10F78000A3EFF012F7872290054C12BA28AA18AB03
:10F79000192274EE12039E8A088B09ECFEEDFF75A8
:10F7A0000A00EE65087003EF6509600C121FAA8A53
:10F7B0000C8B0DEA450D7006750A0102F84EEEFA43
:10F7C000EFFB121FAA8A0E8B0FAC0EAD0FEC4D6033
:10F7D00007EEFAEFFB121FBCE4F50EF50F780E12E0
:10F7E000090DAC0CAD0DEEFAEFFB121FA474021262
:10F7F00008CFE96059AA0CAB0D121F2C8A0E8B0F93
:10F80000EA450F6046780E12090D780C12090D7C3E
:10F81000007D00AA08AB09121FB674041208CFE9D4
:10F82000701D780E12090D780C12090D7C007D00F8
:10F83000EEFAEFFB121FB074041208CFE9600375F3
:10F840000A01AA0EAB0F121F328003750A10A90A13
:10F8500002C31874F712039EE9901BC2F07A157B5D
:10F860008012267C7A387B00901BC2E0F912267C3D
:10F87000901BE374BAF0A37424F0901BE174C0F001
:10F88000A37424F0901BDF74B4F0A37424F0901BD5
:10F89000CC7402F0901BC474FEF0A304F07F01024C
:10F8A000060F74F212039EEAFEEBFF54807003020F
:10F8B000F9C6805279001213148A0A8B0B750C005A
:10F8C000780C120911780812090D780A12090D90A6
:10F8D000059612FD49901BC3E0F91224A874051285
:10F8E00008CF901BDAE060179081B212070D7A08FA
:10F8F0007B00901BC2E0F9121FF274041208CFAA19
:10F9000008AB09121E90901BC2E0F9121EA28A08D1
:10F910008B09E5084509700302F9BE85088285094F
:10F9200083E024CF603E14607E245F70D2E508241B
:10F930000CF582E43509F583E0F50AA3E0F50B78D0
:10F940000A12057D0000020038005BF9158052F9AB
:10F95000FFF8AA08AB0912249C80A4AA08AB0912DC
:10F960002496809B901BCFE0C39404509290055541
:10F97000E0F99081B6120BAC120C12E97081850887
:10F980008285098312FEC6901BD112FC2E85088247
:10F99000850983A3A312FEC6901BD312FC2E901BD5
:10F9A000DA74FFF002F8FF901BDAE0F4600302F86B
:10F9B000B4AA08AB091224A2901BDAE480E5EEFA9F
:10F9C000EF648002FA54EEA2E05025901BDEE09036
:10F9D0000541F07ADE7B1B79E11228261223D690AE
:10F9E0000596E4F0A3F07901121314EE640180622D
:10F9F00054026039901BCD12FEC8E8496025901B67
:10FA0000CDE024FFF0A3E034FFF09081A212070DB7
:10FA10007A027B00901BC2E0F9121FF274041208F4
:10FA2000CF8005901BCFE4F0EE64028025EE5408F1
:10FA30006025901BDAE06017901BD9E0F9901BD588
:10FA4000120BAC120C12E97006901BDAE014F0EE07
:10FA50006408FAEFFB80047A007B007F0602060F41
:10FA600074F412039E74F7120999EAFEEBFFAC18C6
:10FA7000AD191225BC7404120BC3E0C39406505A8E
:10FA800012FC1B600302FBFD7405120BC3E0700344
:10FA900002FBFDC39406400302FBFD7404120BC37A
:10FAA000E0F9851882851983120BAC120C12E960FB
:10FAB0000302FBFD12FC07901BC312FECE12FC2BAF
:10FAC0007405120BC3E014F08518828519837CD568
:10FAD0007D1B740912083302FBFDE064FE7077742D
:10FAE00006120BC312FC12400302FBFD7406120B3C
:10FAF000C3E0F912124279008518828519837808CB
:10FB0000120B54E9780812093AE508A2E040070907
:10FB1000E9C3941B40E2900541E069700302FBFDDC
:10FB2000E9901BDEF0900532E075F064A4F8AAF0CD
:10FB3000E42A8808F5093395E0F50AF50B780812F0
:10FB400009057A017B00901BC2E0F9121FF27404D0
:10FB50001208CF02FBFDE0F4705C7406120BC312B6
:10FB6000FC12400302FBFD7406120BC3E0F91212F3
:10FB700042851882851983120B7CE8494A4B60271D
:10FB80008518828519837808120B5490054F7808E0
:10FB90001209AF6012851882851983120B7C9005BB
:10FBA0004F120B701223D67407120BC3E0FAA3E0B6
:10FBB000FB1224AE804712FC1B70428E828F83A3FF
:10FBC000A312FC267508007808120911780812099A
:10FBD00011E4F509780812090D780812090D780862
:10FBE00012090D90814212070D7D007C807AC47B42
:10FBF0001B12FC07F9122676740C1208CF74091236
:10FC000008CF7F0402060FEE240FF582E43FF58350
:10FC1000E022E0F8900598E0C39822EE240BF582EC
:10FC2000E43FF583E022E0F8A3E0F9901BC4E8F09C
:10FC3000A3E9F02274F712039E74FD120999EAFEFB
:10FC4000EBFFAC18AD191225AA851882851983E03F
:10FC500070187401120BC3E05440600E8E828F83C3
:10FC6000A3A3E0FAA3E0FB1224AE74031208CF02B0
:10FC7000F89D74F212039E8A0C8B0D7A00850C821B
:10FC80008B83A3A3A37808120B54900541E0780856
:10FC900012093AE508A2E05014E0F8E50C28F582D4
:10FCA000E43BF583A3A3A3A3A3A3A3E0FA7B00856E
:10FCB0000C82850D83A3A3A37808120B54EB78085C
:10FCC00012093AE508A2E05076EBF8E50C28F58237
:10FCD000E4350DF583A3A3A3A3A3A3A3E0C39A5084
:10FCE0005E90059412FC26750810780812091178A8
:10FCF0000C12090D901BD3120711901BD112FD4954
:10FD000079001224A874051208CF901BD07401F05A
:10FD1000901BCFE07020901BCD743CF0A3E4F090DA
:10FD200081A212070D7A027B00901BC2E0F9121F1C
:10FD3000F274041208CF901BCFE004F002FA5B0BC0
:10FD4000EBC3941B50F602FCAFE0FCA3E0FD7AC4C9
:10FD50007B1B2274EC12039E89118A128B13ECFE1A
:10FD6000EDFF7510007508007509007A0074161211
:10FD70000BC3E0F50AA3E0F50B850A82850B83A38C
:10FD8000A3A3780C120B54EA780C12093AE50CA2E2
:10FD9000E0500205100AEAC3941B40DDE510605AEA
:10FDA000FA7B00121F2C8A088B09EA4509604B7BFD
:10FDB000007A00850A82850B83A3A3A3780C120B1B
:10FDC00054EA780C12093AE50CA2E05026EAF8E56C
:10FDD0000A28F582E4350BF583A3A3A3A3A3A3A369
:10FDE000E0C0E0EBF8E50828F582E43509F583D0BA
:10FDF000E0F00B0AEAC3941B40B9750C00780C12B2
:10FE000009117419120BC3E0F50C780C1209117862
:10FE10000812090D7418120BC31207118E0C8F0DE6
:10FE2000780C12090D850A82850B83A3A3A3120700
:10FE30000DAD10850A82850B83A3A3E0FCAA12AB4B
:10FE400013A911122676740C1208CFE50845096033
:10FE500007AA08AB09121F327F0C02060FC082C02E
:10FE600083900594E06A7003A3E06B600B900594A7
:10FE7000EAF0A3EBF01223D6D083D0820208B77445
:10FE8000F612039EEAFEEBFF7A067B00121E8AEA58
:10FE90004B602E8A828B837431F08E828F8312FEA8
:10FEA000C88A828B83A3A3E8F0A3E912FECE8A82DC
:10FEB0008B83A3A3A3A312FC2E901BC2E0F9121EF6
:10FEC000967F0202060FA3A3E0F8A3E0F922F08ECA
:10FED000828F83A3A3E0F8A3E0F92274F412039EB7
:10FEE0008A088B097A227B00121E8A8A0A8B0BAE43
:10FEF0000AAF0BEE4F60628E828F837432F08508FA
:10FF000082850983E08E828F83A3A3F08508828592
:10FF10000983A3120B7C8E828F83A3A3A3120B7081
:10FF2000850882850983A3A3A3A3A3E0F508A3E022
:10FF3000F509750A0078081209097C1B7D00EE247A
:10FF400007FAE43FFB121E6074031208CFEEFAEFCB
:10FF5000FB901BC2E0F9121E9602FC02C082C08315
:10FF6000901BD0E060238A828B83A3A3A3E0701947
:10FF70008A828B83A3E07011900596E4F0A3F07958
:10FF800001121314901BD0E4F002FE78C082C083EB
:10FF9000851882851983E0F8A3E0F9E84960128AA0
:10FFA000828B83ECF0A3E824FF18E934FFF9487052
:10FFB000F2D083D0820208B7C082C0831228E080CA
:10FFC00010C082C0831228E68007C082C083122935
:10FFD00016D083D0820208B7C082C08312291C8049
:10FFE000F0C082C083900736E0F9D083D082020847
:0AFFF000B70208B70208B70208B70D
:020000040001F9
:10000000C082C0831217F49004F874F2F0A3740D48
:10001000F09004FA74F8F0A3740DF09004FC74FEF0
:10002000F0A3740DF09004FE7404F0A3740EF002BB
:10003000B79274F712039EE9FE9004EAE4F0EE90A2
:1000400004E9F0901E6E12AB2E12B47D7CBA7D1CBA
:100050007AED7B04122040901E70E09004F5F09041
:1000600004F6749FF0A3741C028F6974F012039E4F
:100070008A088B09EB548070030281C39004E9E085
:10008000F9121EA28A0A8B0BAE0AAF0BEE4F700359
:100090000281BA12A903707EEE241F12AC78641399
:1000A0007002A3E070708E828F83A3A3E0F50EA38D
:1000B000E0F50F90050812B17E750A00750B0080FF
:1000C0000D128DE012B47D121F32AA0CAB0DEA4B5B
:1000D00060448A828B83E0650E7004A3E0650F7034
:1000E000288A828B83A3A3A3A312A916E50A450B32
:1000F0008A828B83A3A3A3A360C7129E4D850A8225
:10010000850B83A3A3A3A380BB8A0A8B0B8A828B54
:100110008312B17A80B8EE242A12AC78F912C2D5D3
:1001200090050812925BA3A3A3A3A3A3A3A3E064D7
:100130000270378A828B8312B17E80078C828D8316
:100140001294BBEC4D60208C828D83E06A7003A317
:10015000E06B70E88C828D83A3A3E06970DE901E53
:100160007612A29BF0804C120E2E8E828F83E0645A
:10017000017034EE241812822C120911129BE31222
:10018000070DEE241212822C120911129BD71209AC
:100190000D12BD4F120711EE2417129BEB1217A080
:1001A000740A1208CF800CE064027007EEFAEFFBCD
:1001B000120F84EEFAEFFB121E90AA08E509648084
:1001C000FB8066901CC5E0600464017019EAA2E03F
:1001D000501490050012B095600612C80A12052945
:1001E000E5086401803AEA5402600C901DDF740156
:1001F000F0EA6402FA8032EA54086029120E288B71
:100200000BEA450B701690050AE4F0A3F0A3F0A3E7
:10021000F07A08FB9004E9E0F9121FFEE508640893
:10022000FAAB0980047A007B0002962112A984F5BA
:100230000A780A2274F412039EEA4B9005006026A5
:10024000ECF0A3EDF08A088B09E4F50AF50B7808C9
:100250001209057A017B009004E9E0F9121FF2749B
:10026000041208CF800FE4F0A3F07A01FB9004E9B8
:10027000E0F9121FFE028CB074F412039E8A088B00
:10028000098A828B8312BFC9129ADB38F583E02476
:1002900009FA7B00121E8A8A0A8B0BAE0AAF0BEE9C
:1002A0004F700302833C8E828F837402F0A3E412AA
:1002B000C9B8A3A3A3A3E8F0A3E912C2FDA3A3A313
:1002C000A3A3A3A3F0E5082403F8E4350912B4209E
:1002D000129ADB3AF583129254F0EE2409FAE43FC5
:1002E000FB8E828F83A3A312BB30F5838882E0A2AA
:1002F000E58E828F83A3A3A3A3A35004740180017E
:10030000E4F0E5082403F88882898312B17EEA12BA
:100310009ACF3BF583128341120909EA241012BDDA
:10032000578E828F8312B17C121E6074031208CF25
:10033000EEFAEFFB9004E9E0F9121E96028CB0A3EE
:10034000A3E0F508A3E0F509750A0078082274F225
:1003500012039E8A088B09ECFAEDFB740E120BC394
:10036000E0FC1218248A0C8B0DAE0CAF0DEE4F6022
:1003700030AC08AD09121812E96026AC08AD09EEE0
:10038000FAEFFB121818E970148E828F83129D7E8B
:10039000FAEFFB12180CAA08AB0912183C7900807E
:1003A0000279B480031208CF7F0602060F74EE12A2
:1003B000039E74F71209998A0A8B0BECFEEDFF7508
:1003C0000CB3750D00750E008002050E90310AE425
:1003D00093F8E50EC39840030284BCAA0E7B00127A
:1003E00018608A088B09EA450960DF8A828B83A33B
:1003F000A3A3A3A3E0250DF50DF8C3E50A98E50B2B
:10040000940050C67C157D007900EEFAEFFB121EB9
:1004100072850882850983A3A3A3A3A3E0F8E50A54
:10042000C3950D2825E0F8E433F9E50828F582E5C1
:100430000939F58312902A12B47D1211EE8A0A8BC3
:100440000BAC0AAD0BEEFAEFFB122040850882855B
:100450000983A3E06401700B129BE3740112D8447A
:10046000A3803DAC18AD1985088285098312B17C43
:10047000121848E9602D7408120BC3E0C0E0129B0B
:10048000E3D0E0F07408120BC3E06403700CAC1806
:10049000AD1912924C12204080098518828519836B
:1004A00012B471850882850983129603A3A312C929
:1004B0000EC0E0129812D0E0F0750C00A90C74097F
:1004C00002CE0774F712039EE9FE8A828B83A3A3F0
:1004D000A3A3A3A3E0540860338A828B83A3A3A3BE
:1004E000A3A3A3E0540260218A828B83A3A3A3A3C6
:1004F000A3A3A3A3A3E06406600F74E96E600A746B
:10050000CD6E600574F06E7003120E1002A51174AA
:10051000E812039E74F81209997406120BC312A90B
:1005200055ECFEEDFF891775150012878112183002
:100530008A0A8B0BEA450B700302872EEE241012F9
:10054000AC78FAA90A120C8A8A128B13EA45137046
:100550000302872EEE2403F50CE43FF50DEE24068E
:10056000F508E43FF5097C00850882129B2F1218DC
:10057000368A108B11850C82850D8312877612B115
:10058000FF851282851383A3A3A3A312AD651287EF
:1005900076A3A3A3A312B0A5851282851383A3A378
:1005A000A3A3A3A312CDFF12C8F3120909EE129A56
:1005B000DB3F12BD5B851282851383A312B17612D5
:1005C0001E6074031208CF7428120BC3129E4DE5EF
:1005D0001212A28D351312B47B742A120BC3E0C021
:1005E000E0E512129ACF3513F583D0E0F0751400D0
:1005F0007423120BC3E0F5167424120BC3780C128B
:100600000B540286B585108285118312B17C1218B5
:100610004E850882850983A3EAF0A3EB128798A38D
:10062000A312C3BE128792A2E6500F8508828509E5
:1006300083A3A3A3A3A3E0D2E1F0E5157066850828
:1006400082850983129E4C90053FE0687003A3E009
:10065000697051850882850983A3A3A31293EB7562
:1006600010007810120911780C120905E516F51022
:1006700078101209117426120BC312071190054C41
:1006800012071179007410120BC312C2DD120FDEB3
:10069000740A1208CF850882850983A3A3A3A3A3A4
:1006A000E04405F074012514FC1287811218368A83
:1006B000108B110514E5104511604EC3E514950A21
:1006C000E4950B5044E51475F006A4F8A9F0E51282
:1006D00028F8E51339F9E8240FF508E439F5098518
:1006E0000882F583E412DC64E0640160030286059D
:1006F000751501850882850983740112879812ABEC
:10070000D8A3E8F0A3E902861CAA12AB13120C903E
:10071000781212090DAD167424120BC3E0FCA91750
:10072000EEFAEFFB120E0A74021208CF803E8E82A0
:100730008F83A3A3A3E0C0E07403120BC3D0E0F047
:10074000EE241212AC78C0E07404120BC3D0E0F0B7
:10075000E50A450B70097405120BC374B980077460
:1007600005120BC3741012BD64120FD8740812085E
:10077000CF7F1002060FE0851282851383A3A3A307
:10078000228E828F8312B1828E828F83A3A3A3E0F5
:10079000F922A312C536E02212DC68A32274E81203
:1007A000039E74F2120999E9851882851983F08AEB
:1007B0000C8B0D8C168D177426120BC312B063AA06
:1007C00008FB120C7EE9F514AA08AB09120C84E9A7
:1007D000F515E5147003028A64751300800F8E828C
:1007E0008F83A3A3A3A3A3E0D2E3F0051312981C65
:1007F000E0F8E513C3984003028A5BE51470030236
:100800008A5BE51375F006A4F8A9F0E50828F8E579
:100810000939F9E8240FFEE439FF8E828F83A3A300
:10082000A3A3A3E0A2E040C3750E00901CC5E06046
:10083000046401704A8E828F83E0704312B17D128E
:1008400029948A0A8B0BA80AA90BE849603188828F
:100850008983A3A3A3A3E06401600D88828983A395
:10086000A3A3A3E0640370178E828F83A3A3A3A323
:10087000A3E0D2E7F0750E01E51570030287EB7572
:100880000F00750A08750B00E5176003750F207CD3
:10089000087D007900740112095B121E728E828F2E
:1008A00083E0604490058FE06401701CE50FD2E3A3
:1008B000F50F750B10129E487401120BC3E8F0A3DC
:1008C000E9129FCD74FF803E430F0C750A0C8E8297
:1008D0008F83A3128A77A3A3A3A312B47D740112FA
:1008E0000BC374FFF0A3801E851882851983E06016
:1008F00009E50FD2E6F50F750A0A129E4874011237
:100900000BC3E8F0A3E9F07403120BC3E50FF01278
:100910009AD9350DF583E0C0E07405120BC3D0E021
:10092000F07406120BC37401F012095B120F8A7483
:100930000D120BC3E06003028A367409120BC31256
:10094000B1EB8E828F83A3A3A3A3F07409120BC310
:1009500012A93EE50AF0A3E50BF012A8F9E516127C
:100960008793601190058FE0C0E07409120BC312E9
:10097000A92ED0E0F07409120BC312982CA3A3A3E4
:10098000128A69241C12A94F12D0CE128A6912A8A9
:10099000F0EAF0A3EB12C837C0E012A8E6D0E012EC
:1009A000C8FFC0E07409120BC312A42DD0E012C01E
:1009B0001FC0E07409120BC312A421D0E0F0740927
:1009C000120BC3128A7712A410128BB8128A6924F0
:1009D0002C12A94FE50C12A26D350DF583E0C0E095
:1009E00012A408D0E0F07409120BC312B17E850C7A
:1009F00082850D83128A6E2428F582E43B12B47B33
:100A0000E50C129ACF350DF58312CE1775120078CA
:100A100010120909129AD9350D12BD5BEA12BF9E58
:100A20003BF58312B17E121E6074031208CF74016D
:100A300012095B120F908E828F83A3A3A3A3A3E05E
:100A4000D2E0F0740D120BC3E060030287DEE50E06
:100A5000A2E05002151515140287EB7900AA08AB25
:100A600009120E16740E02876E12B188E822A3A333
:100A7000A3A3129E51EA22129E51850C82850D83FA
:100A80002274EE12039E74E91209998A088B09896F
:100A90000A8A828B83A3A3A3A3A3A3A3A3E0F9122F
:100AA0000CA88A0C8B0DEA450D7003028B4712B01F
:100AB0002F1294D6E50A6003028B4C7C04850882D1
:100AC000850983A3A3A3A3A3A3A3A3E0F9120CAE58
:100AD000EE4F60738E828F83A3A3A3129E4C740685
:100AE000120BC312BB13129E4C7408120BC312B923
:100AF00076C0E07410120BC3D0E0128BB8129E4C7B
:100B0000740E120BC312B47D7411120BC3E412B134
:100B1000F0C8241FF582E438F58312AE2CC41313F9
:100B20005403FC70027C048E828F83E0F9780C12EF
:100B3000090D742059FD744059F9740212095B12B1
:100B40000E0A74021208CF741702CE077C088508BB
:100B500082850983A3A3A3A3A3A3A3A3E0F9120CF3
:100B6000AE8B0FEA450F7003028AD0EE4F60D8E5D6
:100B70000AF50B780B120911850C82850D83A3A34E
:100B8000A3A3A3A3A3E0F50B780B1209118A828B10
:100B900083A3A3A3E0FB8A82850F831294BE8A827B
:100BA000850F83E0FA8E828F83A3A3E0F912179A50
:100BB00074021208CF028AD4F0850C82850D83A3BB
:100BC000A3A3A3A3A3A3A32274F712039E74FA12F0
:100BD0000999E9FE7C017D017F0080037D000F12F1
:100BE000AC6DE0F8EFC3985028EF75F006A4F885D7
:100BF000F008A908EA28F8EB39F9E8241412B60B32
:100C0000A2E050D8540C60D4E0A2E250D17C008025
:100C1000CD8A828B83A3A3A3A3A3A3E0703DEDA2FF
:100C2000E0400574016E70338A828B83A3A3A3A373
:100C3000A3A3740112A2D5E0C0E07403120BC3D0C9
:100C4000E012A2CDE0C0E07404120BC3D0E0F07457
:100C500005120BC3EC12BD64120FD8740602A50E68
:100C6000C082C0837901120E1602B79274F4120387
:100C70009EEA4B901DDF6022E4F08A088B09F50A9A
:100C8000F50B78081209057A027B009004E9E0F977
:100C9000121FF274041208CF800F7401F07A027BE5
:100CA000009004E9E0F9121FFE800574021208CFDB
:100CB0007F0402060F74E812039E74FC12099974F3
:100CC00002120BC3E4F0A3F09005081294D6851825
:100CD00082851983E4F0A3F0751401900539E0A230
:100CE000E35003028D6C1220168A088B098C0A8D42
:100CF0000B8A0C8B0D8C0E8D0F90050A780C120947
:100D00006B128DE77810790C120B0650077A017B75
:100D100000028DDB850C14850D15850E16850F17C9
:100D20007814791012032FA814A915901E76E0C329
:100D300098E4995003E08001E8F514128DE7780CEF
:100D4000791012032FE4F512F513780879101209BF
:100D5000EE90050A7808120B368011128DE012B45D
:100D60007DEEFAEFFB121F32AE08AF09EE4F606363
:100D70008E828F83A3A3A3E0F8E514C3985029EED5
:100D80002403F582E43FF583A814E0C398F06021C2
:100D90007402120BC3129FC412A9AFEEF0A3EF129C
:100DA000C024FEA3E0FF80C48E828F83A3A3A3E4AC
:100DB000F08E828F8312B05F85188285198312B0FE
:100DC000958E828F83A3A3A3A3609012C2EF12B467
:100DD0003B808B7402120BC312B17E740402876EC7
:100DE000129E5190050822901E74E0F510A3E0F5C4
:100DF00011E4F512F5132274F212039E8A0A8B0B8A
:100E0000E9FE7A007B0090050812B0639005081295
:100E1000B095601E0A850882850983A3A3A3A31247
:100E2000B095600E0AEA70010B88088909E8450947
:100E300070E3901E77129E4DC3EA98EB994003022F
:100E40008EEA7A067B00121F2C8A0C8B0DA80CA947
:100E50000DE8497003028EEA88828983E50AF0A3CF
:100E6000E50BF0EE88828983A3A3F0901E7612B67C
:100E70007DA3A3A312A2FDA3A3A3E4F0A3F0900576
:100E800008129E55600F850882850983A3A3A3A33A
:100E900012B47D801F90050812B47D900539E0A240
:100EA000E34011122016EAF8EBF9ECFAEDFB90059D
:100EB0000A120B70900539E0A2E3502E7A087B00ED
:100EC0009004E9E0F9122004EA4B4C4D701C901E8E
:100ED0007412D6A878081209057A087B009004E9F4
:100EE000E0F9121FF874041208CF0283A8C082C070
:100EF00083E9901DE0F0900502744CF0A3740EF0AD
:100F0000900504745EF0A3740EF09005067470F002
:100F1000A3740EF002B79274F712039EEAFEEBFF81
:100F20008908EE4F700312189C90050E12B0957050
:100F30000890050E8022129E4D88828983A3A3A368
:100F4000A3A3A3A3A3A3129E5588828983A3A3A3CB
:100F5000A3A3A3A3A3A370DEEEF0A3EF12C3DAA3AF
:100F6000A3A3E4F012C3D9E508F002A51174F712A7
:100F7000039E90050E800D8E828F83A3A3A3A3A34F
:100F8000A3A3A3A31294D6EE4F60348E828F83A3C3
:100F9000A3A3A3A3A3A3E06970DD8E828F83A3A381
:100FA000A3A3E06A7003A3E06B70CC8E828F83A34F
:100FB000A3A3A3A3A3E06C70BEEEFAEFFB80047AB8
:100FC000007B0002A51174F712039E90050E129487
:100FD000D690050E128A72687002EB69701EE0C826
:100FE0002409F582E438F583129E4D90050E12B463
:100FF0007D90050E1294D680271294C9EE4F602082
:101000008E828F83A3A3A3A3A3128A6E687002EBC0
:101010006970E68A828B83A3A3A312902A12B47DFF
:10102000121F32EEFAEFFB02A511A3A3A3A3A3A301
:10103000129838A3A3A3A3A32274F012039E74FAF8
:101040001209998A088B098A828B83A3A3A3A3A37D
:10105000A3A3A3E060336401602F8A828B8312B163
:101060007E121290E97022850882850983A3A3A3CA
:10107000A3A3A3A3A3E0640370147404120963AAD6
:1010800008AB09120F00E970167902029235850843
:1010900082850983129E4D7404120BC312B47D1213
:1010A000CBE6243412BAFE121F2C8A0A8B0BAE0A2E
:1010B000AF0BEE4F70030292337C347D0079001247
:1010C0001E72740212095B850882850983A3A3A39B
:1010D000A3A3A3A3A3A3E0F91217E87402120BC3FE
:1010E000E0C0E0129244D0E0F0EE242EF50AE43F96
:1010F000F50B7403120BC3E0850A82850B83F0792C
:1011000001EEFAEFFB120E3A85080C85090D750EFB
:1011100000780C1209097C1E7D0012924C121E6090
:1011200074031208CFEE24321295F92434F8E43F08
:10113000F98A828B8312B47DE5082411F8E435091D
:10114000F9E8FCE9FD8C828D8312A94A243012B49F
:10115000771295F112D95B1209098C828D83129254
:101160005B12B17E121E6074031208CF7404120B5E
:10117000C312983412B47D9004EA129254A3A3A32C
:10118000F09004EAE004F01220168E828F8312A9F8
:1011900099242C129B04750D00850A82850B83E02F
:1011A000780C120A9C8A828B83E50CF012923AE545
:1011B0000C12A9AFE4F0E508241512CBEAA2E07402
:1011C000015007120BC374018004120BC3E4F0EE4C
:1011D000242912B056AA18AB191217CAE924FE85A1
:1011E0000882850983F0EE2430F8E43FF9E8FCE951
:1011F000FD129263120256E88E828F83A3A3A3A3EB
:10120000A3A3A3A3F01292631202568B09EA450925
:10121000600F8E828F83A3A3A3A3A3A3A3A3E00441
:10122000F0EE242012AC784408129B50121ECC79A8
:101230000080027910740602961EEE242BF582E4DB
:101240003FF58322EE12BF9E3FF58322EE240BFA78
:10125000E43FFB2212C305A3A3A3221294C38A82F4
:101260008B83228C828D8312ABDCE0FA7B002274AC
:10127000F412039EEAFEEBFF1220168E828F831279
:10128000A955901E6AE0F8EE242D12AC78C3984060
:10129000030293D0129B107012EE242D12AC78042E
:1012A00012ACABC0E012923AD0E0F0EE242A12ACBD
:1012B00078FC7900800109EE242E12AC78F8E9C39D
:1012C000985026750801750900E97808120A9C12E1
:1012D0009B10550860E0E92CFC750801750900E9D0
:1012E0007808120A9CE04508F0EE242912AC78FA3E
:1012F000EE2430F582E43FF583EC8AF0A4F8ABF0FD
:10130000E42BF9E098F8A3E099F9C3E89AE994008E
:10131000EE4031242912AC78F8129B10602C129206
:10132000441293EBA3E4F0EC7047EE242012AC7867
:10133000442012B97AC0E012AC99D0E012ACA3FA02
:10134000A3E0805212923B74FFF090052FE0FA90D8
:101350001E6D1293E2ABF075F064A4FAADF075F077
:1013600064EBA42DFB8E828F83A3A3EAF0A3EB8012
:10137000B5EE242012AC7854DF12AC94ECF0FAEE07
:101380002429F582E43FF5831293E2FAABF0EE12E2
:10139000A8E03F129B26FB12C8D7EAF0A3EB12C3CA
:1013A000E9C0E0EE2425F582E43FF583D0E012A900
:1013B00066E812B0A590051012B095600BECF9121A
:1013C000C80A120529E9701712924C120ED6800F26
:1013D0007BE912960F121794EEFAEFFB120E4602FB
:1013E0008CB0E0F508EA8508F0A42212C305A3F04A
:1013F0002274F412039E90050E1294D61220168ABF
:101400000A8B0B78FF79FF8020E0C39AFCA3E09B56
:10141000FDC3EC98ED99500E8E828F83A3A3E0C399
:101420009AF8A3E09BF91294C9EE4F605C8E828F0C
:101430008312B17EE50AC39AFAE50B9BFB8E828F7D
:10144000831294BDC3EA9CEB9D8E828F83A3A3403D
:10145000B8A3A3A3A3E06402701AEE240B129B139B
:101460006009129AEF12B17E121E90EEFAEFFB1293
:101470000E468007EEFAEFFB120E527A017B0090C7
:101480001DE0E0F9121ECC802974FF68700374FF20
:1014900069601F88088909E4F50AF50B78081209C4
:1014A000057A017B00901DE0E0F9121FF27404122E
:1014B00008CF028CB0A3A3A3A3A3A3A3A3A3A312A7
:1014C00094C322E0FCA3E0FD228E828F83A3A3A31A
:1014D000A3A3A3A3A3A3E0FEA3E0FF2274F012033F
:1014E0009E8A088B09ECFAEDFB890A7C0112CBE697
:1014F000F9120E408A0C8B0DAE0CAF0DEE4F70033F
:101500000295E5E50A60030295E51295F11296074A
:101510006860030295E51295F1E0FAEE242E12AC14
:1015200078F8EA28FAE43400FB8E828F83A3A3A321
:10153000A3A3A3A3A3E0F8EA98EB9400C365D03378
:10154000401CE508241412CBEAF470127B001296BA
:101550000F121794EEFAEFFB120E460295E5E5081E
:10156000241412CBEAF47042EE242B1295F9242EA7
:10157000F8E43FF9E8FCE9FD7508FF7509008C8285
:101580008D83E07808120A9C8A828B83E508F0122A
:1015900095E7E508F08C828D8312960728F0EE24FB
:1015A0002DF582E43FF583E4801BE5082414F8E47C
:1015B0003509F9E0C0E01295E7D0E012BB25C0E0A4
:1015C00012923AD0E0F01220168E828F8312A999DF
:1015D000129245129603A312B0A57A01FB901DE06A
:1015E000E0F9121ECC803AEE242CF582E43FF5831C
:1015F00022E508241312982422F8E43FF9E8FAE9D6
:10160000FBEE2212C30522E0F8EE12B622E022EE33
:10161000242212A984FAEE241412A984F9221208B1
:10162000CF7F0802060F74EC12039E74FE12099914
:101630008A0A8B0B8C0E8D0F89108A828B83A3A351
:10164000E0F91217BE8A088B09AE08AF09EE4F7099
:10165000077A007B000298087A127B00121F2C8AFE
:10166000088B09EA450970030298047C127D007911
:1016700000121E72AA18AB19850A82850B83A3A3D8
:10168000E0F91217E8E508240FF50CE43509F50D2B
:101690007401120BC3E0850C82850D83F07902AAD8
:1016A00008AB09120E3A850E82850F8312982C1210
:1016B000984A129AC312C3B5F07512FF75130085CC
:1016C0000C82850D83E07812120A9C12D0CEE512AE
:1016D00012A43912C808E0C0E012981CD0E0F01241
:1016E0009AE5F50CE508240D12D0D2E50CF0E50AD8
:1016F000129AF7850CF0A4A9F02427FAE439FB121A
:101700001E8A8A0C8B0DAE0CAF0DE50812C7E0EEF9
:10171000F0A3EFF0EE4F70030297F78E828F837481
:101720001A12B0A58E828F83A3A3F0A31298501231
:10173000983412B47DAC0EAD0F12C8E11217E285D9
:101740000A82850B83A3A3A3E0C0E012AE22D0E0FF
:10175000F090054C12A94A241012984412A9383569
:101760000B12A94812BD46E8F0A3E9129850A3A3B2
:10177000A3A312A94A241212B477850A82850B8387
:10178000A3A3E0C0E0129812D0E0F0E50A12A28D07
:10179000129ACAE0C0E012C0D5D0E0F07416120B65
:1017A000C312C810C0E012CBD4D0E012C3D4C0E042
:1017B00012C7E6D0E012C819C0E012C7F0D0E0129C
:1017C000A95BE510F07418120BC3120B7CEE241AFF
:1017D000F582E43FF583120B70EE2427F8E43FF91D
:1017E000EE242212984412BAEA129ACAE0C0E01219
:1017F000C8E9D0E0F0800DAA08AB09120E467508C2
:1018000000750900AA08AB0974021208CF7F0C0208
:10181000060FEE2414F582E43FF58322129820226D
:10182000E508240BF582E43509F5832212ABDCA32D
:10183000A3A3A3221298382212C54B8E828F83A3B2
:10184000A3A3A322F582E43FF58312A9C7E50A22E8
:10185000F0850A82850B83A3A3A3A3A3A32274ED1F
:1018600012039E8A0A8B0B8C108D11891275090048
:10187000EA129AF7F50890051012B095600EA908C3
:1018800012C80A120529E96003029ABE7C0285107B
:101890008285118312B17EE50A129AC3E0F9120E15
:1018A000408A0C8B0DAE0CAF0DEE4F7054850A8242
:1018B000850B83A3E0A2E04003029ABE7415120BCD
:1018C000C312070D7417120BC3120711A912AC1023
:1018D000AD11AA0AAB0B120E6474061208CF8A0C63
:1018E0008B0DAE0CAF0DEE4F7003029ABE8E828F41
:1018F00083A3A3A3A3A3A3A3A3E508129B50121E33
:10190000CCA8088E828F83A3A3A3A3A3A3A3A3E041
:1019100024FFFAE434FFFBEA684B7003750901EE1B
:10192000240B129B137003029A73850A82850B8322
:10193000A3E0A2E05003750800129B3DE5089AE47D
:101940009BC365D033401CE0F8EE240E12AC78281F
:10195000F0750CFF750D00E8780C120A9C12B89611
:10196000E50CF0E50A129ACF129ACA12C98F120931
:1019700009E50A129ADB350B12BD5BEE240D12ACA1
:1019800078F50CE508850CF0A4FAABF0129AEF128A
:10199000BFCC2422F582E438129B26FB121E607411
:1019A000031208CF750C01129B18780C120A9C12B6
:1019B000AC75450CF0E509A2E05063EE240C129BD7
:1019C00004129B1804780C120A9C8A828B83E045CF
:1019D0000C12A97985080C850CF0A4F8A9F0129ACC
:1019E000E5FCE82CFCE439FD129AEF12BFCC242070
:1019F000F582E438F583ECF0A3ED12A9A0F4701E93
:101A0000EE240BF50CE43FF50DEE129ADB3F129B32
:101A10002F121E96850C82850D8374FF8054122030
:101A2000168E828F8312A95590052FE0FA901E6DB5
:101A3000E0F50CEA850CF0A4FAABF0F8EBF9901E97
:101A40006AE0F50CE8850CF0A4F8ACF0850CF0E940
:101A5000A42CF9EA28F8EB39F9E875F064A4F8AA9F
:101A6000F075F064E9A42AF98E828F83A3A3E8F0CD
:101A7000A3E9F0A808129B3DEA24FF1AEB34FFFB10
:101A8000EA687001EB600EEE240C129B136006E511
:101A900009A2E05029E50A129AFCECF012AC75C0DC
:101AA000E0E50A2414F582E4129ACAD0E0F0AC0A08
:101AB000AD0B85108285118312B17E120EC47F0B8F
:101AC00002060F12A26D129ACA22350BF58322125A
:101AD0009AD322240EF582E422E50C129ADF222406
:101AE00010F582E422E50A129ADF129ACAE022EE89
:101AF000129ADF3FF58322129AFCE02212A2673588
:101B00000BF58322F8E43FF9E8FAE9FB750CFF22B4
:101B1000EE242B12A984F422750D0012A981F5F090
:101B2000E50884E5F022F583E02AFAA3E03B22F5FC
:101B30008312B188850C82850D83E0F922EE240E94
:101B400012A984FC12A981FAEC2AFAE43400FB22DF
:101B5000F07A017B00901DE0E0F922C082C0839002
:101B60001DE0E0F9121E9602B79274F412039E8AE9
:101B7000088B09EB5480703BEAA2E05053120E58D8
:101B8000E5086401FAAB09804B8E828F83E0640123
:101B9000701A129BE312070D129BD712090DEE2447
:101BA00012129BEB120E6A74061208CFEEFAEFFBCC
:101BB000121E90901DE0E0F9121EA28A0A8B0BAE55
:101BC0000AAF0BEE4F70C2AA08E5096480FB8004DF
:101BD0007A007B00028CB0EE240FF50AE43FF50B8F
:101BE000780A22EE12A2673FF5832212A984F9EE49
:101BF0002402FCE43FFDEE2419FAE43FFB2274F1D9
:101C000012039E890A8A088B098A828B8312B17E0D
:101C1000120E828B0DEA450D600579B8029CA61262
:101C20000EA0E9F890310DE493F9E8C399400479E6
:101C3000B280737A157B00121F2C8A0C8B0DAE0CB0
:101C4000AF0DEE4F70047910805C8E828F83E4F0CC
:101C5000A312C531A3E50A12C82A1209097C127D14
